:1000000000400020895F0000C95F0000CB5F000056
:1000100000000000000000000000000000000000E0
:10002000000000000000000000000000CD5F0000A4
:100030000000000000000000CF5F0000D15F000062
:10004000D35F0000FD46000005640000D35F0000A0
:10005000D35F000000000000D35F0000D35F00000A
:10006000D35F0000D5660000D35F0000D35F0000BF
:10007000D35F0000D35F0000D35F0000D35F0000B8
:10008000D35F00006D680000D35F0000D35F000005
:10009000D35F0000D35F0000D35F0000D35F000098
:1000A000D35F0000D35F00000000000000000000EC
:1000B0000000000000000000000000000000000040
:1000C00010B5064C2378002B07D1054B002B02D02E
:1000D000044800E000BF0123237010BD4C02002043
:1000E0000000000030D00000044B10B5002B03D0FE
:1000F0000349044800E000BF10BDC04600000000F6
:100100005002002030D00000164B002B00D1144BC1
:100110009D46402292029A1A924600218B460F4633
:100120001348144A121A0AF03FF90F4B002B00D063
:1001300098470E4B002B00D0984700200021040068
:100140000D000D48002802D00C4800E000BF0AF066
:10015000EBF82000290006F073F90AF0BFF8C0465A
:100160000000080000400020000000000000000027
:100170004C020020A42F002000000000000000001E
:100180000123034010D104280CD90268120909D0B8
:10019000531E9B001A1DC1180979002902D0013392
:1001A0009342F8D1180070470023FBE70378002B37
:1001B00003D05AB2002A01DB013070473F2293433B
:1001C000C03B59424B41C01803789343802BF4D174
:1001D0000130F9E710B500240378002B01D120008D
:1001E00010BDFFF7E3FF0134F6E770B5002204000D
:1001F0000D00411C092002F0DBFE002806D001237F
:100200006200134343600023A34200DB70BD9A00E9
:10021000A958821891600133F6E770B5012803DC14
:100220001C2000F091FE70BD01230D6811201D42BD
:10023000F7D04868184206D1042804D90F23026871
:100240001340042B01D00E20EBE702F027FD6D10C8
:100250000400002D03DDFFF7BDFFA84206DA1220DF
:10026000DFE72000FFF7A2FF0400013D012DF8D1D8
:1002700020787F2809DDDF280BDCF8233F22DB0014
:10028000800118406378134018430123400018434D
:10029000C9E7EF280BDCFC22637812019B011340B5
:1002A0003F220007000C0343A0781040ECE7F7283A
:1002B00012DCFC22637892021B031340E0228004CC
:1002C000520310403F221843E3781340FC220343BB
:1002D000A07812018001E8E701204042D5E7F0B59F
:1002E000070085B00D001C20012F06DD4C6801239E
:1002F00022001A40019203D10D2000F025FE54E0A7
:10030000022F02D08A681A42F6D001232E681E42BC
:1003100000D07EE0042E00D87BE01C41002C00DCE5
:100320001C000F2332681340092B29D173685B101E
:100330000193022F05D0AB68019A5B109A4200DD51
:100340000193019B01221F1B0137FB43DB171F4059
:10035000791C092002F02CFE061E09D001237F0023
:100360001F4303002A68083347600199A14202DA5B
:10037000300005B0F0BD0134A100515802C3F4E7CC
:10038000042B46D1300002F089FCFFF723FF0290D6
:10039000022F04D0AB685B10984200DD0293029BF1
:1003A0009C4204DD002002F06FFE0600E0E7300012
:1003B00002F074FC0700019B9C4222DC3000019794
:1003C00002F06CFC03903800FFF7F0FE029B013452
:1003D0000700A342F7DA019BC71A380002F054FE67
:1003E000061EC5D002F05AFC0400286802F056FC34
:1003F000039A019B991A41183A00200009F0B8FFAE
:10040000B6E73800FFF7D2FE019B070001330193E6
:10041000D1E7212071E7F8B54D680F00EB0706D44E
:10042000042D04D90F232E683340092B03D00B2051
:1004300000F08AFDF8BD6B6836095C10731EA3429C
:100440000FD80321200007F06BFE6421642803DC31
:100450000100032800DA03212800891902F0D8FDE1
:1004600005002B6800201B09013B9C42E2D23A6840
:10047000A31C9B005A510123013464001C436C608F
:10048000D8E7F0B585B0012803DC1C2000F05CFD46
:1004900029E001254F682A00022806D08B682B42EC
:1004A00003D05D10002D00DC15000124274200D090
:1004B00074E0042F00D871E00F223B680E681340EF
:1004C000042B25D1264205D1042E03D933681340CD
:1004D000042B01D00E20D9E73800FFF751FEA842C7
:1004E00003DA0120404205B0F0BD380002F0D6FB2F
:1004F0000700300002F0D2FB013D010078190AF03C
:10050000F2FA0028EDD0C01B013040002043EAE79A
:10051000092B43D17B685B1000939D42E1DC3000E6
:1005200020402ED1042E2BD90F22336820001340F7
:10053000042B26D1300002F0B1FB0F2325000290DE
:100540000393631C01939B00F858864202D1640018
:100550002800DBE728420ED104280CD90368039A4F
:100560001340042B07D102F099FB010002980AF016
:100570008DFA0028EBD0019C009B9C42E1DDB0E7A6
:100580002000431C9A00BA58B24202D14000012414
:10059000BCE71800009B9842F3DDA2E7212075E735
:1005A00010B502F05FFB43000120184310BD0000AE
:1005B00010B57F2902DC0170013010BD1A4B994241
:1005C0000CDC40238A115B42134303703F230B4032
:1005D00080214942194341700230EEE7134B9942A2
:1005E00010DC20230A135B4213433F248022037054
:1005F0008B1152422340214013430A4343708270BF
:100600000330DAE70A4B9942D7DCF0230370603BF2
:100610004370113B8A11FF3B1A4382703F22114005
:100620001943C1700430C8E7FF070000FFFF000056
:10063000FF0F0100F0B50D0085B0002803DC1C2081
:1006400000F082FC0DE009680122080010400AD089
:1006500002AC11412000FFF7ABFF011B200002F0AC
:100660001FFD04001AE004293FD90F230C68234022
:10067000092B3AD14B685B10019303239C46019BE5
:100680009A420EDD02F000FD041E07D02E680125FF
:1006900002F004FB2F00019B9D421DDD200005B0F0
:1006A000F0BD01329300CC580123234001D10D202D
:1006B000C6E764107F2C0DDD0D4E0223B44209DD28
:1006C0000C4E6346B44205DD00270B4EE30FA642F5
:1006D0007B419B00C018D2E70135AB00F15839428D
:1006E000E5D04910FFF764FFD5E72120A8E7C04611
:1006F000FF070000FFFF0000FF0F010010B504001E
:100700000120084010D104290DD90F230A68134095
:10071000042B08D1080002F0C1FA010020000AF001
:10072000B5F94342584110BD0020FCE7F7B50F0072
:10073000012803DC1C2000F007FCFEBD01264D68EB
:100740002E4006D1042D04D90F222B681A40092A05
:1007500001D00B20EFE76A681B095410A34200D8B0
:100760005C1E39681E48FFF7C9FF0123019000286D
:1007700013D139681B48FFF7C1FF002811D0002CA6
:100780000DD00123621C013C9C4092005351234335
:100790006B6004E00136B200AB50B442FADA0020DC
:1007A000CBE73B680D20DA07C5D55B10002B11DDC8
:1007B0009C420FDB9B00A200291DEB188918043313
:1007C000994209D10123013C9C40AA181C43536063
:1007D0006C60E4E71220AEE758681860EFE7C046A7
:1007E00003BA000007BA0000002310B50C000B701C
:1007F000C30705D50D49421020000AF019F908E099
:100800000B49002802D0042804D10A4920000AF02C
:100810002FF910BD0428FCD90F2302681340042BC4
:10082000F7D102F03BFA04490200E5E768C2000094
:100830000CBA000012BA000017BA0000F0B593B06D
:100840000390030002911C20012B1DDD029B01255A
:100850001B681C002C4000D0A8E0042B00D8A5E0A9
:100860001A680F231A40092A48D10194019A029963
:1008700092008A5816002E4005D1042A03D9106828
:100880001840092804D0222000F05EFB07002CE06D
:1008900052685210A418019A013201920199039AE8
:1008A0008A42E3D1611C012202F082FB071E01D1C2
:1008B00000271AE064002543456005000835029AC8
:1008C000B300D1584B680A685B1012099A4200D8ED
:1008D000531E002293420BDCDA43D21713409B00D5
:1008E000ED18019B01369E42E9DB380013B0F0BDE4
:1008F00090000C18A46801322C50EBE7042A55D163
:100900002F0026001D00029AB300D058384237D17C
:10091000042835D903682B40042BB4D1FFF730FCF1
:10092000039B01362418B342EDD1200002F0ACFB4A
:10093000071EBDD0039B029D9B00EB18041D029374
:1009400001232E681E4222D1042E20D90F223368A3
:100950001340042B0DD13000FFF712FC0190300042
:1009600002F09CF9019A0100200009F001FD019BB1
:10097000E418029B0435AB42E2D100232370B4E7B4
:1009800005A9FFF731FF05A80AF092F8C8E705A905
:100990003000FFF729FF05A80AF08AF806000200D8
:1009A00005A9200009F0E4FCA419E2E7212000F0E9
:1009B000CBFA7DE7F0B50D0095B0002806DC1C20D1
:1009C00000F0C2FA0400200015B0F0BD0C6801214F
:1009D00023000B40009306D1042C04D922680F3366
:1009E0001A40092A01D00B20EAE7626852100392EC
:1009F000002A03DC009802F047FBE3E73F4A01923C
:100A000001280BD06868084208D1042806D902687A
:100A10001340042B02D102F041F9019001980AF031
:100A200047F806000F27039B0834013B04935E43FD
:100A3000039B02909B001B19059301232068184219
:100A400051D104284FD903683B40042B52D1FFF702
:100A500097FB059B04343618A342EED1300002F018
:100A600013FB041EAFD02B680593029B002B03D011
:100A7000686802F013F90190200002F00FF90500F8
:100A8000009B059A9B00D3189F68380002F006F976
:100A9000012306001F4201D1042F04D807A9380002
:100AA000FFF7A2FE07AE30000AF002F807000200CE
:100AB0003100280009F05CFC029BED19002B0AD0E4
:100AC000049B009A934206DD2800029A019909F0DE
:100AD0004FFC029BED18009B01330093009A039B8F
:100AE0009342CDD16FE707A9FFF77EFE07A809F073
:100AF000DFFFAEE702F0D2F8F9E7C04667BD0000BD
:100B000010B50224002806DD0B68DA0703D55C1057
:100B1000022C00DA0224611C0122092002F048FAAA
:100B2000002803D0012364001C43446010BD0B68FF
:100B300070B518000125284032D1042B30D90F247C
:100B40001A6849681440092C16D15C6812092C41B6
:100B5000A24200D8541E844205DC02200132904299
:100B600006DB00200FE085005D19A9600130F2E787
:100B7000840019510130F2E7032C11D1294203D12D
:100B8000132000F0E1F970BD4910FF29F8D81209CF
:100B9000043392009A189A42E3D919700133FAE7A4
:100BA0000B2000F0D1F9DCE70123F7B500264D68F2
:100BB0000F002B400093B3420DD11E00042D0AD923
:100BC0000F222B681A40092A0FD16A681B09561098
:100BD000B34200D85E1E3968CB0713D54C10002CE9
:100BE00001DDA64219DA12202EE0042A04D12800E1
:100BF000FFF7C6FA0600EEE7009E032AEBD11E09B6
:100C0000B600E8E72E48FFF779FD002814D009F078
:100C1000ABFE310007F06AFB4C1C009B002B4CD153
:100C2000042D4AD92A680F331340092B10D10134FF
:100C3000A40064592000FEBD39682248FFF75EFD1C
:100C400034000028E9D1113000F07EF90400F1E70A
:100C5000042B2AD1280002F021F80600FFF7BAFA87
:100C6000A042C0DB012C1ADC280002F017F800902B
:100C70003000FFF79BFA851B280002F005FA041EDE
:100C8000D8D002F00BF80190786802F007F8009BCA
:100C90002A00F11A4118019809F06AFBCAE73000EE
:100CA000FFF784FA013C0600DCE7032B05D12C1981
:100CB000E478023B64001C43BCE70B20C4E7C04659
:100CC000FCB9000007BA0000F7B54C680F0001201E
:100CD000210001402AD1042C28D90F222368BE68A4
:100CE0001A40092A13D162681B0955100191AB42C1
:100CF00000D85D1E39682848FFF700FD002829D07C
:100D00000F2322681340092B19D1012313E0032A72
:100D10000CD1064203D1132000F016F9FEBD72106B
:100D20000192FF2AF7D81D09AD00E3E70B20F3E796
:100D300001339A00A6509D42FADA0020EEE7032B19
:100D4000FBD1230001331A1BAA42F6DC6A46127952
:100D5000DA70F7E73968CB0706D54910002901DDBD
:100D60008D4209DA1220D7E70C48FFF7C7FC2900AB
:100D7000002801D11130CFE70F2322681340092B3F
:100D800003D1013189000E51D7E7032BD5D16B4632
:100D90001B796418E370D0E703BA000007BA0000BB
:100DA00010B501240868204216D1042814D90F2256
:100DB00003681A40092A01D1406810BD032A03D1F3
:100DC0001809C0002043F8E7042A05D101F066FFA6
:100DD000FFF700FA4000F5E70B2000F0B5F8ECE76C
:100DE00010B5034A0A21034803F080FD10BDC04638
:100DF000ACB90000A4B9000002000120104001D0ED
:100E0000501070470D22014B1A70FAE78C02002037
:100E1000F0B585B00393019002912C4E2C4B002A23
:100E200002D002223270013A00251A601B68F55484
:100E3000019B9D4201DB05B0F0BD029AAB00D0588A
:100E4000234B1C68C8239B0037191C1B0123184225
:100E500006D0204A43102100380009F0B7FD09E010
:100E60001D4A002802D004281BD11C4A210038004A
:100E700009F0ACFD300009F01BFE154A039B106021
:100E8000002B0CD0019B013BAB4208DD144B984278
:100E900005D8431C1360202232540022F25401353D
:100EA000C6E704280FD90F2302681340042B04D18E
:100EB00001F0F4FE0B4A0300CDE7092B04D143688F
:100EC000094A5B10C7E70123084AC4E78D020020E6
:100ED000B005002068C200000CBA000012BA000081
:100EE0001F0300005FC800007CBC00008BBC00003A
:100EF0000123020010B51A4015D1042801D9026857
:100F000012090B4011D1042901D90B681B090024D7
:100F1000934206D104309B000431C318984206D393
:100F20000124200010BD0022EBE70023EFE7047846
:100F30000A78002C01D1002AF2D00130013194420C
:100F4000ECD00024EDE70000014B18700020704742
:100F50008C02002070B501F0B5FC094C0100251D84
:100F60001F22280009F0ABFD280009F0A1FD042391
:100F700004308008000118432060200070BDC04686
:100F800068020020C368F0B59D00836889B05D19D0
:100F90000300183306930369069A9F00069B02908C
:100FA000DF19436901939B00D3180393CD4B1B7842
:100FB000002B26D17F222B68CB491C1213409B00AB
:100FC0005B58043501929F46029B587804F062F802
:100FD0000023029A137027E0C24B1B78002B10D11C
:100FE0002B68019A1C121340BF4A9B009B58043582
:100FF000E9E7069B3A1DD11ABA4BD82928DD1A22F7
:101000001A70029BB74C9B6821780193EA1A029BE5
:1010100092109B7812021A43029B587804F042F80F
:101020000023029A23701370029B069A9B68019317
:10103000ED1A029BAD10DD60069BFE1A029BB610F6
:101040001E61039B9B1A029A9B10536109B0F0BD6D
:101050001B783C60002B01D01700D2E72B68019968
:101060001C120B40A0499B005B5817000435AAE7EF
:10107000069B3A1DD11A9B4BD82902DD1A221A7001
:10108000BFE728681B78291D3860002B02D01700A5
:101090000D00B6E76B6801991C120B4092499B004A
:1010A0005B58170008358EE7069B3A1DD11A8D4B09
:1010B000D82902DD1A221A70A3E7A4001B782C1984
:1010C0003C60002B01D017009BE72B6801991C1294
:1010D0000B4085499B005B581700043573E7069B5E
:1010E0003A1DD11A7F4BD82902DD1A221A7088E7DF
:1010F0007E49A40061581B783960002B01D017008D
:101100007FE72B6801991C120B4077499B005B58C5
:101110001700043557E7043F744B3A68A400E250C7
:10112000704B1B78002B00D06BE72B68019A1C12C8
:1011300013406D4A9B009B58043544E76B4BA40059
:10114000E058FFF759FE043F06003868FFF754FEE9
:1011500036180120654B76000643E650614B1B783C
:10116000002B00D04DE72B68019A1C1213405E4AF9
:101170009B009B58043526E7069B3A1DD11A594B14
:10118000D82902DD1A221A703BE70698039C012138
:10119000A04202D221000C3909681B783960002B6B
:1011A00001D017002DE72B6801991C120B404E4906
:1011B0009B005B581700043505E7069B3A1DD11AC2
:1011C000484BD82902DD1A221A701AE706990398AB
:1011D00081420FD203000C3B1B6845495B10641829
:1011E000E41AA40023583B603E4B1B78002B05D02B
:1011F000170006E7182119700023F4E72B680199FE
:101200001C120B4038499B005B5817000435DAE686
:10121000069B039A934219D213000C3B1B68344A75
:10122000043FA4185B10E31A039A39689B00995095
:101230002C4B1B78002B00D0E3E62B68019A1C1284
:101240001340294A9B009B580435BCE61822254BC5
:101250001A70EDE7069B039A93422DD2244B3E1F52
:10126000E31814000C3C04932368049A5B10D31A0F
:10127000039A9B009858FFF7BFFD07903068FFF76F
:10128000BBFD2468049B64101C1B079BA4001F1853
:1012900001207F00039B0743E7503700114B1B7869
:1012A000002B00D0ADE62B68019A1C1213400E4AA9
:1012B0009B009B58043586E618220A4B1A70EDE70E
:1012C000069B3A1DD11A074BD82902DD1A221A7043
:1012D00097E60399A40061581B783960002B09D068
:1012E00017008EE68C0200207CBA00004C2D0020F6
:1012F000FDFFFF3F2B6801991C120B40D7499B0053
:101300005B58170004355EE6043F039B3A68A4006F
:10131000E250D34B1B78002B00D072E62B68019A69
:101320001C121340CD4A9B009B5804354BE6039B8F
:10133000A4001C192368043F38685E10FFF75CFDA9
:1013400036180120C64B76001B7806432660002B1A
:1013500000D056E62B68019A1C121340BF4A9B002E
:101360009B5804352FE6069BA4003F1BBC4CBB4298
:101370000CD82378002B00D043E62B68019A1C126E
:101380001340B64A9B009B5804351CE6B54801F053
:1013900075FC2378002B00D033E62B68019A1C12D1
:1013A0001340AE4A9B009B5804350CE6A300ED1891
:1013B000002C00DA38E6AA4B1B78002B00D020E680
:1013C0002B68019A1C121340A44A9B009B580435B9
:1013D000F9E5043F3B68042B04D1A300ED18002C71
:1013E00000DA21E69E4B1B78002B00D009E62B6823
:1013F000019A1C121340994A9B009B580435E2E560
:10140000043F3B68042B06D0A200AD18002C02DA82
:10141000002B00D108E6924B1B78002B00D0F0E5A2
:101420002B68019A1C1213408C4A9B009B58043570
:10143000C9E53A1F13685B10013B002B06DD012153
:101440005B00A4000B432D191360EDE5844B1700DE
:101450001B78002B00D0D4E52B68019A1C12134096
:101460007E4A9B009B580435ADE53A00069B0C3242
:10147000D31AD82B03DD1A22794B1A70C1E5FF234A
:1014800061005B001940FE3BFF3B19433960029944
:1014900006988968241204916D1A0299AD10897812
:1014A0002D020D4303999D40091A891099401D434F
:1014B0000B43BB60029B7D609C70E4B26A4BE4000E
:1014C0000392E358029A9360654A1278002A03D087
:1014D00008331D00039F94E51D00019A9B680C359D
:1014E0001C1213405D4A9B009B58039F6BE53B1FFA
:1014F0001C68039A069B93422DD10A20E3070CD463
:10150000042C13D90F2322681340042B11D120007F
:1015100001F0C4FB09F0CCFA0630643003F076FA2F
:1015200000280FD1043D069B03937DE50720042C82
:10153000F3D02000431E9841FA234042FF33184065
:101540000730EAE7029B2100587803F0BDFD002335
:10155000029A1370E7E7039B039A0C3B1B680299FE
:101560005B109B00D31A0C3B1C601F1D1300083B33
:101570001B685A108A70D2B23B49D2005B005558A2
:101580009B0A029A9B009560ED18039B069A043B08
:101590001B685B109B00D3180393314B1B78002B07
:1015A00000D02EE52B68019A1C1213402B4A9B0099
:1015B0009B58043507E53B1F1868FFF71DFCA40086
:1015C00006003F1B1E2827DC00280DDC244B1B785F
:1015D000002B00D015E52B68019A1C1213401F4AFE
:1015E0009B009B580435EEE401F05AF9033E36188F
:1015F00001F056F91D4B801B9842F9D8184B1B7807
:10160000002B00D0FDE42B68019A1C121340134AF2
:101610009B009B580435D6E40123029A137001F015
:101620003FF9029B0A3886195E60FDE43B1F18688B
:10163000FFF7E2FBA40006003F1B002818DC084B64
:101640001B78002B00D0DCE42B68019A1C1213409D
:10165000024A9B009B580435B5E4C0467CBA0000A2
:101660008C0200209DBC0000542500209F860100B4
:10167000CD4B984203DD1D22CC4B1A70C1E40123EF
:10168000029A137001F00CF9FA239B005E43029B4F
:101690000A3E30185860C7E4A300FF1A0023200058
:1016A0001A003900FFF7B4FBC14EC24C316820006C
:1016B00003F0C2FB3168200003F00DFD316820000B
:1016C00001F08AFDB94B1B78002B00D099E42B6800
:1016D000019A1C121340B84A9B009B58043572E4CF
:1016E000B24BA4001B783F1B002B00D089E42B6871
:1016F000019A1C121340B04A9B009B58043562E4C7
:10170000029803F0E7F9A94B1B78002B00D078E48E
:101710002B68019A1C121340A74A9B009B58043562
:1017200051E43B1F1B68002B3DD13B000C3B1B6869
:10173000DA072BD5390001225B1058000839024323
:101740000A60002B43DD012259001143381F01605C
:101750003900083909681141CB1A39000C39096878
:10176000114223D09B189340A4001343039AA35023
:101770008E4B1B78002B00D043E42B68019A1C127F
:1017800013408D4A9B009B5804351CE4042B06D95A
:101790000F2219680A40092A01D15B68CAE7192299
:1017A000824B1A702DE45B10013BCAE7042909D96A
:1017B0000F2208680240092A04D102339B005B58BB
:1017C000A400D3E71922794B1A70FFF71AFC0435ED
:1017D000CEE7A300069AFB189B1AD82B13DC012234
:1017E000631E002C14DC714B1B78002B01D0FFF71B
:1017F00008FC2B68019A1C1213406F4A9B009B58EF
:101800000435FFF7E0FB1A22684B1A70FFF7F9FB6B
:101810003A601C000437E3E7069A3B1D9B1A634EAF
:10182000D82B03DD1A233370FFF7EBFB069B039ADB
:10183000A40093422AD23B1F1868FFF7DDFA011E6D
:1018400021DD039B0C3B1A68521082421BDB900780
:10185000801A5A4B4018C018039B8000C2583B1B8B
:101860001A60524B3F1B1B780437002B01D0FFF747
:10187000C8FB2B68019A1C1213404F4A9B009B58CF
:101880000435FFF7A0FB20233370EAE71823FBE7BA
:10189000A3009C46FE1A002C17DC1C22434B1A7036
:1018A000002333606346FF1A404B04371B78002B3C
:1018B00001D0FFF7A6FB2B68019A1C1213403E4A89
:1018C0009B009B580435FFF77EFB002033685A10BD
:1018D0008300F15801230B4003D10D21334A1170CD
:1018E000DFE749108A4200DD0A0001308442EFDC64
:1018F000012352001343D4E7A3009C46FE1A002C98
:1019000017DC1C22294B1A70002333606346FF1A30
:10191000264B04371B78002B01D0FFF772FB2B6896
:10192000019A1C121340244A9B009B580435FFF770
:101930004AFB002033685A108300F15801230B4002
:1019400003D10D21194A1170DFE749108A4200DAEC
:101950000A0001308442EFDC012352001343D4E734
:101960003B00083B1868FFF747FA3B1F0600186862
:10197000FFF742FA0023864200DA0433A4003A1B40
:1019800017001360094B04371B78002B01D0FFF7B9
:1019900038FB2B68019A1C121340074A9B009B5886
:1019A0000435FFF710FBC04680EE36008C020020A5
:1019B000B00500208D0200207CBA0000FCFFFF3F34
:1019C0003B00083B1868FFF717FA3B1F0600186832
:1019D000FFF712FAF30FC217B0425341A4003A1BAB
:1019E00017009B001360E14B04371B78002B01D0DC
:1019F000FFF707FB2B68019A1C121340DC4A9B007F
:101A00009B580435FFF7DFFA3B00083B18683B1F83
:101A10001968A600BE1B0423814202D0042802D804
:101A20000023336016E001231842F9D10F23026826
:101A30001A40042AF4D1033A1142F1D10429EFD912
:101A40000A681340042BEBD1FFF752FA431E98416A
:101A500080003060C54BA4001B783F1B0437002B6F
:101A600001D0FFF7CEFA2B68019A1C121340C04A2E
:101A70009B009B580435FFF7A6FA3B00083B18680B
:101A80003B1F1968A600BE1B0023814202D0042818
:101A900002D80423336016E001231842F9D10F2342
:101AA00002681A40042AF4D1033A1142F1D1042900
:101AB000EFD90A681340042BEBD1FFF719FA434220
:101AC000584180003060A94BA4001B783F1B0437AD
:101AD000002B01D0FFF795FA2B68019A1C121340D6
:101AE000A34A9B009B580435FFF76DFA3B00083B67
:101AF0001868FFF781F93B1F06001868FFF77CF9AB
:101B0000F317C20F86425341A4003A1B17009B00F3
:101B10001360964B04371B78002B01D0FFF771FA46
:101B20002B68019A1C121340914A9B009B58043564
:101B3000FFF749FA3B00083B1868FFF75DF93B1FC8
:101B400006001868FFF758F90023864200DD0433C9
:101B5000A4003A1B17001360844B04371B78002B3A
:101B600001D0FFF74EFA2B68019A1C121340804AED
:101B70009B009B580435FFF726FA3B1F1B68A40007
:101B8000043B5A1E93413A1B17009B001360774B8E
:101B900004371B78002B01D0FFF733FA2B68019A2A
:101BA0001C121340724A9B009B580435FFF70BFA36
:101BB0003B00083B1868FFF71FF93B1F0600186839
:101BC000FFF71AF932180120A4003B1B1F00520036
:101BD00002431A60654B04371B78002B01D0FFF7D6
:101BE00010FA2B68019A1C121340614A9B009B5803
:101BF0000435FFF7E8F93B00083B1868FFF7FCF8ED
:101C00003B1F06001868FFF7F7F8321A0120A400FE
:101C10003B1B1F00520002431A60544B04371B78D1
:101C2000002B01D0FFF7EDF92B68019A1C1213402D
:101C30004F4A9B009B580435FFF7C5F93B00083B12
:101C40001868FFF7D9F83B1F06001868FFF7D4F8AB
:101C500002000120A4003B1B1F00724352000243FC
:101C60001A60424B04371B78002B01D0FFF7C9F9EB
:101C70002B68019A1C1213403D4A9B009B58043567
:101C8000FFF7A1F93B1F1868FFF7B6F8061E17D13A
:101C90001F22364B1A70A4003B1B1F001E60334BE3
:101CA00004371B78002B01D0FFF7ABF92B68019AA2
:101CB0001C1213402E4A9B009B580435FFF783F9F2
:101CC0003B00083B1868FFF797F8310006F028FA48
:101CD000012640000643DEE73B1F1868FFF78CF83B
:101CE000061E17D11F22214B1A70A4003B1B1F0098
:101CF0001E601E4B04371B78002B01D0FFF781F9C3
:101D00002B68019A1C121340194A9B009B580435FA
:101D1000FFF759F93B00083B1868FFF76DF83100F1
:101D200006F0E4FA012649000E43DEE73B1F18687F
:101D3000FFF762F8C217801850400122A4003B1B35
:101D40001F00400010431860084B04371B78002B1D
:101D500001D0FFF756F92B68019A1C121340044A70
:101D60009B009B580435FFF72EF9C0468C020020DB
:101D70007CBA0000A300FE1A3068012C24D1FFF7C2
:101D80003BF80494079008F0EFFD0799002900DC68
:101D9000012106F0ABFA049BA400C91801234900F5
:101DA0001943F34B3F1B1B7831600437002B01D0E4
:101DB000FFF727F92B68019A1C121340ED4A9B008C
:101DC0009B580435FFF7FFF8FFF716F8049070688A
:101DD000FFF712F8049B0130C31A0793D3E7A3005F
:101DE000FE1A31002000049301F096F9049B306044
:101DF000FF1ADF4B04371B78002B01D0FFF701F9E6
:101E00002B68019A1C121340DA4A9B009B58043538
:101E1000FFF7D9F83B00083B1868FEF7EDFF3B1FC2
:101E200006001868FEF7E8FF02000120A4003B1B33
:101E30001F003240520002431A60CD4B04371B781A
:101E4000002B01D0FFF7DDF82B68019A1C1213401C
:101E5000C84A9B009B580435FFF7B5F83B00083B88
:101E60001868FEF7C9FF06003B1F1868FEF7C4FF9D
:101E7000320002430120A4003B1B1F00520002431A
:101E80001A60BB4B04371B78002B01D0FFF7B9F861
:101E90002B68019A1C121340B64A9B009B580435CC
:101EA000FFF791F83B00083B1868FEF7A5FF060016
:101EB0003B1F1868FEF7A0FF320042400120A4003B
:101EC0003B1B1F00520002431A60A94B04371B78CA
:101ED000002B01D0FFF795F82B68019A1C121340D4
:101EE000A44A9B009B580435FFF76DF83B1F186808
:101EF000FEF782FFC0430122A4003B1B1F004000ED
:101F0000104318609A4B04371B78002B01D0FFF761
:101F100078F82B68019A1C121340964A9B009B5834
:101F20000435FFF750F83B00083B1868FEF764FFE4
:101F300006003B1F1868FEF75FFF32008240510029
:101F40000122A4003B1B1F000A431A60884B043780
:101F50001B78002B01D0FFF754F82B68019A1C1254
:101F60001340844A9B009B580435FFF72CF83B0034
:101F7000083B1868FEF740FF06003B1F1868FEF795
:101F80003BFF3200024151000122A4003B1B1F0015
:101F90000A431A60764B04371B78002B01D0FFF7F9
:101FA00030F82B68019A1C121340724A9B009B5810
:101FB0000435FFF708F83B000C3B1868FEF71CFFE0
:101FC0003B00083B06001868FEF716FFF1170200F9
:101FD000C317300006F0DCF93B1F04900591186828
:101FE000FEF70AFF02000498059906F085F9430000
:101FF0000120A4003E1B370018435D4B30601B7866
:102000000437002B01D0FEF7FCFF2B68019A1C124D
:102010001340584A9B009B580435FEF7D4FFA30099
:10202000FE1A310020000493FEF76AFD049B306025
:10203000FF1A4F4B04371B78002B01D0FEF7E1FF4E
:102040002B68019A1C1213404A4A9B009B58043586
:10205000FEF7B9FFA300FF1A39002000FEF767FD65
:10206000434B1B78002B01D0FEF7CBFF2B68019A66
:102070001C1213403F4A9B009B580435FEF7A3FFF8
:10208000A300FE1A310020000493FEF78DFD049B8F
:102090003060FF1A364B04371B78002B01D0FEF757
:1020A000B0FF2B68019A1C121340324A9B009B58C8
:1020B0000435FEF788FFA300FF1A39002000FEF761
:1020C00003FE2B4B1B78002B01D0FEF79AFF2B68E9
:1020D000019A1C121340274A9B009B580435FEF7B7
:1020E00072FFA300FE1A310020000493FEF758FE91
:1020F000049B3060FF1A1E4B04371B78002B01D065
:10210000FEF77FFF2B68019A1C121340194A9B00AF
:102110009B580435FEF757FF069B3E1DF31A144CDF
:10212000D82B03DD1A232370FEF76BFF00F0C2FBF0
:1021300043000120184323783860002B02D0370079
:10214000FEF75FFF2B68019A1C121340094A9B009F
:102150009B5837000435FEF736FF069B3E1DF31AE9
:10216000034CD82B08DD1A232370FEF74AFFC04624
:102170008C0200207CBA000000F092FBF54B40007E
:1021800018400123184323783860002B02D0370011
:10219000FEF737FF2B68019A1C121340EE4A9B0092
:1021A0009B5837000435FEF70EFF0123A600BE1B27
:1021B00020001A003100FEF72BFEE84C2068643046
:1021C00002F024FC002802D1043DFEF72DFF029B03
:1021D00021685A78E24802F08CFF0123029A370006
:1021E000137000F05DFBDF4B22681B68063253431F
:1021F0001818029B5860FEF717FFA600BE1B2000B0
:10220000012300223100FEF703FED44C2068643025
:1022100002F0FCFB0028D7D0D14802F065FDDCE7D6
:10222000A4003E1BFEF796FE3700CF4B30601B78B4
:102230000437002B01D0FEF7E4FE2B68019A1C1234
:102240001340C54A9B009B580435FEF7BCFEA40012
:102250003E1B300000F05DFB3700C34B30601B7845
:102260000437002B01D0FEF7CCFE2B68019A1C121C
:102270001340B94A9B009B580435FEF7A4FEA40006
:102280003E1B300000F047FB3700B74B30601B7837
:102290000437002B01D0FEF7B4FE2B68019A1C1204
:1022A0001340AD4A9B009B580435FEF78CFEA300FB
:1022B000FE1A31002000049300F030FB049B3060D4
:1022C000FF1AA94B04371B78002B01D0FEF799FEAB
:1022D0002B68019A1C1213409F4A9B009B5804359F
:1022E000FEF771FEA4003F1B380000F049FB9E4B37
:1022F0001B78002B01D0FEF784FE2B68019A1C127C
:102300001340954A9B009B580435FEF75CFEA300E2
:10231000FE1A31002000049300F05AFB049B306049
:10232000FF1A914B04371B78002B01D0FEF769FE92
:102330002B68019A1C121340874A9B009B58043556
:10234000FEF741FEA4003F1B380000F083FB864BE4
:102350001B78002B01D0FEF754FE2B68019A1C124B
:1023600013407D4A9B009B580435FEF72CFE01214B
:10237000200000F057FB7C4B1B78002B01D0FEF7B0
:1023800040FE2B68019A1C121340734A9B009B5815
:102390000435FEF718FE0021200000F043FB724BCD
:1023A0001B78002B01D0FEF72CFE2B68019A1C1223
:1023B0001340694A9B009B580435FEF704FEA400B5
:1023C0003E1B300000F068FB3700674B30601B7825
:1023D0000437002B01D0FEF714FE2B68019A1C1263
:1023E00013405D4A9B009B580435FEF7ECFDA400AA
:1023F0003E1B300000F064FB37005B4B30601B7805
:102400000437002B01D0FEF7FCFD2B68019A1C124B
:102410001340514A9B009B580435FEF7D4FDA4009D
:102420003F1B380000F026FB4F4B1B78002B01D0E0
:10243000FEF7E7FD2B68019A1C121340464A9B00E9
:102440009B580435FEF7BFFDA4003F1B380003F086
:1024500037F9454B1B78002B01D0FEF7D2FD2B68D6
:10246000019A1C1213403C4A9B009B580435FEF70E
:10247000AAFDA4003E1B300003F0B4F937003A4B2C
:1024800030601B780437002B01D0FEF7BAFD2B68B3
:10249000019A1C121340304A9B009B580435FEF7EA
:1024A00092FDA4003F1B380003F0BAF82E4B1B78B6
:1024B000002B01D0FEF7A5FD2B68019A1C121340DA
:1024C000254A9B009B580435FEF77DFDA4003E1B6A
:1024D000300003F0BBF83700234B30601B78043723
:1024E000002B01D0FEF78DFD2B68019A1C121340C2
:1024F000194A9B009B580435FEF765FDA300FF1A9F
:102500003900200001F010F9174B1B78002B01D087
:10251000FEF777FD2B68019A1C1213400E4A9B00B0
:102520009B580435FEF74FFDA300FF1A3900200029
:1025300000F082FF0C4B1B78002B01D0FEF761FDF1
:102540002B68019A1C121340034A9B009B580435C8
:10255000FEF739FDFEFFFF7F7CBA0000B0050020CA
:102560008D020020040000208C020020A300FF1A2E
:102570003900200000F070FF944B1B78002B01D035
:10258000FEF73FFD2B68019A1C121340904A9B00F6
:102590009B580435FEF717FDA300FF1A39002000F1
:1025A00000F082FF894B1B78002B01D0FEF729FD3C
:1025B0002B68019A1C121340854A9B009B580435D6
:1025C000FEF701FDA300FE1A31002000049303F082
:1025D000AEF9049B3060FF1A7C4B04371B78002B4C
:1025E00001D0FEF70EFD2B68019A1C121340784AA9
:1025F0009B009B580435FEF7E6FCA300FE1A310051
:102600002000049303F09BF9049B3060FF1A6F4B8A
:1026100004371B78002B01D0FEF7F3FC2B68019ADE
:102620001C1213406A4A9B009B580435FEF7CBFCF2
:10263000A300FE1A31002000049303F088F9049BE4
:102640003060FF1A614B04371B78002B01D0FEF776
:10265000D8FC2B68019A1C1213405D4A9B009B58C2
:102660000435FEF7B0FCA300FE1A310020000493ED
:1026700002F08EFF049B3060FF1A544B04371B7826
:10268000002B01D0FEF7BDFC2B68019A1C121340F1
:102690004F4A9B009B580435FEF795FCA300FF1A98
:1026A0003900200000F0C8FF484B1B78002B01D0F8
:1026B000FEF7A7FC2B68019A1C121340444A9B00AA
:1026C0009B580435FEF77FFCA300FF1A3900200059
:1026D00000F012FF3D4B1B78002B01D0FEF791FC60
:1026E0002B68019A1C121340394A9B009B580435F1
:1026F000FEF769FCA300FE1A31002000049300F0ED
:1027000069FE049B3060FF1A304B04371B78002BA6
:1027100001D0FEF776FC2B68019A1C1213402C4A5C
:102720009B009B580435FEF74EFCA300FF1A3900AE
:10273000200000F0DFFF254B1B78002B01D0FEF7B7
:1027400060FC2B68019A1C121340214A9B009B5885
:102750000435FEF738FC069B029AFB1A9B101361A6
:10276000A300FF1A3900200002F0D4F8174B1B78A1
:10277000002B01D0FEF745FC2B68019A1C12134078
:10278000134A9B009B580435FEF71DFC069B029ADA
:10279000FB1A9B101361A300FE1A31002000049362
:1027A00002F0B8F8049B3060FF1A084B04371B781E
:1027B000002B01D0FEF725FC2B68019A1C12134058
:1027C000034A9B009B580435FEF7FDFB8C0200205A
:1027D0007CBA00000023F7B55A1E0192002B07DADD
:1027E00000F0B8FF02F082FB02F0DAFC192301933B
:1027F00000263000194B1968B14212DD184B1A68D7
:1028000001328A420FDAF0241A601D68154F6C43BA
:10281000E35D002B1FD0E419022B06D12000FEF748
:10282000B1FB019BD8E70022EDE7012B0DD1002879
:1028300001D100F035F8F0226A43BB185B680A4901
:10284000C31A8B4201D80223BB54F0235D43054BCE
:10285000EB5C022BE2D00136CCE7C046B405002089
:1028600000000020F41B00209F860100002070471C
:102870000020704700207047002070470122002090
:10288000054B06491A61585004310330585008313D
:10289000801858501A6070470080004004050000FE
:1028A0000122034B1A64A822D20098587047C046F0
:1028B0000080004010B5FFF7F3FFFA21890005F012
:1028C000A5FB10BD00487047F0BC00001D207047FC
:1028D00070B5054E0400335C0D008B4202D003F04E
:1028E00045FF355570BDC046B805002070B50024C1
:1028F000064D635D012B05D10021200003F036FF5A
:102900000023635501341D2CF2D170BDB8050020A1
:1029100070470D2070473B2070470000F8B5012438
:102920000B6806000D00234204D10D20FEF70CFBBE
:102930002000F8BD5B102000052BFAD80E4A9B0042
:102940009C580E4F3B5D002B05D00021200003F06A
:102950000DFF00233B55012E06DD6B68042B03D1D0
:102960000221200003F002FF200003F0ADFD01244E
:1029700040002043DDE7C046D8BC0000B805002079
:10298000F8B501260568354202D04468344203D1C7
:102990000D20FEF7D9FAF8BD6D101C2DFBD80A4F9B
:1029A0007B5D012B04D03100280003F0DFFE7E5553
:1029B000064964108C4202DCE143C917214028001B
:1029C00003F008FEE7E7C046B8050020FF0300005B
:1029D00070B501240D68254204D10D20FEF7B4FA2C
:1029E000200070BD6D101C2D17D80024012804DDB7
:1029F0004C68043C63425C416400094E735DA34231
:102A000004D02100280003F0B1FE7455280003F023
:102A1000E1FE03000420012BE3D00020E1E7C046E3
:102A2000B805002070B504000D001C280ED8084E13
:102A3000335C012B04D0012103F098FE01233355B0
:102A4000290020004D1EA94103F0AEFE70BDC04616
:102A5000B8050020036810B5DA0703D40D20FEF78F
:102A600073FA10BD4168581004394A425141FFF7CA
:102A7000D9FFF6E737B569460A00064B30CB30C2BE
:102A800003680220042B02D100F0E6FC37BD00F001
:102A90000BFDFBE7B0BC000010B5084C6379002BC0
:102AA00005D00021052003F061FE0023637105209D
:102AB00003F090FE43425841800010BDB80500204D
:102AC00010B5084CE37A002B05D000210B2003F051
:102AD0004DFE0023E3720B2003F07CFE434258417D
:102AE000800010BDB80500207047704710B5034A3C
:102AF0000421034801F0FAFE10BDC046B8BC000036
:102B000098C30000E12170B54902144803F0D4FADB
:102B1000FFF7B4FE0A2003F0D1FC0023FF21104A86
:102B2000995401331D2BFBD1012200200D4B0100D4
:102B30001A6004230C4A0D4D1468002CFCD02C683C
:102B40000002013B20431160002BF5D10122084B0C
:102B50001A6003F06DFC00F049FF70BD7C1B002083
:102B6000B805002000D0004000D1004008D500404A
:102B700004D00040F8B50B4E070030000D0003F004
:102B8000E3FA0400A84200DD2C003D00EB1B9C4250
:102B900005DD300003F0E2FA28700135F6E7200089
:102BA000F8BDC0467C1B002010B50100014803F0B1
:102BB0008BFA10BD7C1B002010B5054C200003F0E3
:102BC00091FAE1212000490203F076FA10BDC046D7
:102BD0007C1B0020C3070CD4064B1B68834208D81B
:102BE000054B1B68984204D8031F1B68002B00D0BC
:102BF00018007047E0050020DC05002000230120BC
:102C000010B509499A0001338850642BFAD1074C5A
:102C1000074A0021200007F0C7FB064B064A636005
:102C2000064B1A6010BDC0464C2D0020E405002064
:102C3000D409000030270000E8050020D805002056
:102C400010B5044B044A1A60044B054A1A60FFF79A
:102C5000D5FF10BDE0050020E4050020DC050020C4
:102C6000B80F0020044B1B68186800090238C343E2
:102C7000DB1718407047C046D805002000B59BB050
:102C80000200054901A807F0D3FE01A802F048F8A8
:102C900002F086FAFCE7C04657BD00000A4BC207A7
:102CA00004D4042804D8094B00D0094B18007047FD
:102CB0000F2203681A40031D042AF7D0054B092A86
:102CC000F4D0054BF2E7C0463DBD000012BA00004B
:102CD0000CBA000050BD000047BD00000020064AAD
:102CE0000649131F186013681B0902339B00D21892
:102CF0008A42F6D37047C046E8050020B80F00208E
:102D0000F7B50F2401262E4B2E4A19682E4B2F4D56
:102D1000186813681F002740072F20D813681B0965
:102D200002339B00D218AA42F3D30024284EA500F8
:102D3000AD192868FFF74EFF01342860642CF6D1E6
:102D4000244C2068002802D0FFF744FF20600025B3
:102D5000214B1B680093009B9D4213DBF7BD1B09B1
:102D60009B00D3189A42D9D01F68374208D1B94284
:102D700006D2B84204D3043F3F68002F00D01F6042
:102D8000043BEFE7F0236B43144A9B181A78002AA0
:102D900001D10135DFE71F693C2300266B43DB19B6
:102DA0009B0001930136BB1BF3D4019BB4001C1B99
:102DB0000A4B1C19A069FFF70DFFA061F2E7C0469E
:102DC000E0050020E8050020DC050020B80F002009
:102DD0004C2D0020B80F0020B4050020F41B00206B
:102DE000F7B50124204244D1224B1B689C469842EF
:102DF0003FD3214B1B68019398423AD8031F1B68AD
:102E0000002B36D10200036800941B09002B0FD160
:102E10000099131F196090422BD015682B1F1B6857
:102E2000990069180C68013B14600A602A00EDE7FC
:102E30009D0055192968009C214218D18C4516D84F
:102E4000019C8C4213D30E1F3468002C0FD10F68E5
:102E50000F343C40072C07D92F60151F2B600B68DF
:102E60000A601B090A00D1E700993160CEE7013BF7
:102E7000CCE7F7BDE0050020DC0500200D49F0B5EA
:102E80000B000F260C4D18681C1F27680209023220
:102E9000002F0BD000208B4200D008002060900053
:102EA000091892009B18AB42EDD3F0BDB0431860F7
:102EB000F7E7C046E8050020B80F0020F8B5114C30
:102EC00026000F2233681F0913420DD07D1CAD0070
:102ED000A64204D02A003100200007F052FA002256
:102EE0006319043564191A600237BF00064BF619DE
:102EF0009E42E6D31B1B9B10013B1B012360034B2F
:102F00001C60F8BDE8050020B80F0020D80500209F
:102F1000F0B59BB0FFF7C4FC002407001E4AA300D5
:102F2000D0580134FFF75CFF642CF7D11B4B1868B5
:102F3000002801D0FFF754FF0026194B1B689E4262
:102F400016DBFFF79BFFFFF7DBFEFFF7B7FFFFF78F
:102F5000A7FC144BC21B1B6813491B6801A81B0963
:102F6000023B07F065FD01A801F0DAFE1BB0F0BDE1
:102F7000F02575430D4BED182B78002B01D1013650
:102F8000DBE72B695C1E002CF9DBA300EB189869CA
:102F9000FFF726FF013CF6E74C2D0020B80F00207C
:102FA000B4050020D80500201DBD0000F41B002042
:102FB000F7B5164D4F1C2B6806001B680C000192DC
:102FC0001B099F420ADBFFF7A3FF2B681B681B0945
:102FD0009F4203DB0A20FDF7B7FFFEBD2868A71C50
:102FE000BA00DB1B81181B010B6029600021031F45
:102FF00019600F231E4003002401264340C3083AF2
:103000009A189A42E9D9019902C3FAE7D805002033
:10301000F7B503000122134004000D000193002BBB
:103020002AD1164B1B68834226D8154B1B68834256
:1030300022D90F23134F386000681840FFF7B8FFFC
:10304000019B3C68061E3B6016D0236804301B09B8
:103050009D4200DD1D00AA00211D251F07F088F9F3
:10306000FFF73CFE2E60FFF74BFE00232B6022682B
:103070000F339A43226034002000FEBDE00500209B
:10308000DC050020B80F00200323043010B5C11761
:1030900019400918891000220420FFF789FF10BD8C
:1030A00070B5050008000C00FFF7EEFF00230028B4
:1030B00004D170BDE95CC21811710133A342F9DB80
:1030C000E343DB171C40002304192371F1E70000E0
:1030D00010B501240B681C4016D05C10200005F0D0
:1030E000B3FA0B4905F07EF907F064F803F0B6FC7B
:1030F0000022084B06F018FA03F058FC06F0EAFF2D
:1031000043000120184310BD0D20FDF71DFFE5E72A
:10311000D30237390000D040086870B5012405009B
:10312000254006D1042804D90F2302681340042B3C
:1031300003D00E20FDF708FF70BDFFF7AFFD037849
:103140002900233B5A4253411022C01807F066FD64
:1031500080239B05C218044B9A4201D91420E9E749
:1031600040002043E8E7C046FFFFFF3F10B5034A99
:103170000221034801F0BAFB10BDC04670BD00003B
:1031800068BD00000020704710B51E20FDF7DCFE72
:1031900010BD10B51E20FDF7D7FE10BD10B51E20C6
:1031A000FDF7D2FE10BD10B51E20FDF7CDFE10BDFF
:1031B00010B51E20FDF7C8FE10BD10B51E20FDF78E
:1031C000C3FE10BD10B51E20FDF7BEFE10BD10B52C
:1031D0001E20FDF7B9FE10BD7047000010B5034A70
:1031E0000921034801F082FB10BDC04690BD0000DC
:1031F000D8BD00000120034B1860034B1B688340BF
:1032000018437047DC0F0020BC0F0020F0B5EFF32F
:1032100010810123194083F31088134C134AA446EC
:103220001268134E013A9340124F134A002B17D0E5
:10323000146803420FD03D682C60C046C046C046AB
:10324000C046C046C046C046C0460C4C15682468FF
:1032500025605B08EAE765462C6014683460F8E78F
:1032600081F31088F0BDC04608050050080000201A
:103270000C050050C80F0020D00F0020C40F002004
:1032800030B585B001AD0C220649280007F070F872
:103290000024285D01210134FFF71AFB0C2CF8D122
:1032A00005B030BD64BE0000F0B585B06A463C4B49
:1032B0003C4913801C2301AF93700C310922380064
:1032C00007F056F8FFF7F6FA374B384DC0182B6861
:1032D000984201D200232B602C68002C44D13E5D23
:1032E00001213000FFF7F4FA01340121300003F02E
:1032F0005BFA092CF3D100246B461E5D01213000DE
:10330000FFF7E6FA01340021300003F04DFA032CF8
:10331000F2D1C82080000138C046C046C046C04631
:10332000C046C046C046C046C046C046C046C0466D
:10333000F1D100210420FFF7CBFA6B460021187869
:10334000FFF7C6FA6B4600215878FFF7C1FA6B46C3
:1033500000219878FFF7BCFAFFF7ACFA002413308D
:103360002860200005B0F0BDFFF7A4FA2B68002408
:103370009842F6D3042003F0A7F80D4B0D4EC01869
:103380000BD430603068032104F0CAFE00230A4ADF
:1033900030602B6013600124E3E73460F2E7C0463D
:1033A0001A1B000064BE000010270000D40F00208C
:1033B000C8FEFFFFBC0F0020DC0F002010B5012469
:1033C000044002D04410200010BD0D20FDF7BCFDCC
:1033D000F9E700000868F8B5C3071AD5FFF7EEFF54
:1033E0000300203B5E2B23D80520012258430023F5
:1033F000104E451DA84217D005211024375C3C42D1
:1034000000D09B180139520064100029F7D1013017
:10341000F0E704280CD90F2203681A40042A07D1C8
:103420001B0905D00079DBE701205B001843F8BDDC
:103430000120FCE779BE00000022054B10B51A60A0
:10344000044B1B68934201D002F0E6FA002010BD45
:10345000D80F0020A01A002070B508680D00FFF7F3
:10346000ADFF04006868FFF7A9FF621E0100042A8F
:1034700014D8451E042D11D805236B439B18012237
:1034800015009D402B00064805682B430360054B43
:103490001B68002B02D0200002F0BFFA002070BD94
:1034A000D80F0020A01A002070B508680D00FFF7A3
:1034B00085FF04006868FFF781FF621E0100042A8F
:1034C00013D8451E042D10D805236B439B180122E9
:1034D0009A400748036893430360064B1B68002B20
:1034E00003D00022200002F098FA002070BDC046F0
:1034F000D80F0020A01A0020F0B5050089B0086898
:103500000C00FFF75BFF0690022D36DD6068FFF7C9
:1035100055FF0190A068FFF751FF04000127231D0C
:10352000661E0793731C0293079B9E4235D00523AA
:1035300073430593019B019D05330493049BAB42A8
:103540001ED0042E16D86B1E042B13D80122059B07
:103550002349013B5B199A409446224A0B68106844
:10356000069A3A4003920DD062461A430A6001223D
:1035700000280DD17F000135E0E701240194CDE75B
:10358000029ECFE7624693430B600028F2D0039A75
:103590000299280002F041FAECE7019B1E1D042E5F
:1035A0001AD8012C18D1002505273B0021006B43B8
:1035B0009B1999400B000A4A013511689943094B40
:1035C00011601B68002B05D0019B0022581D2900AB
:1035D00002F023FA052DE8D1002009B0F0BDC04665
:1035E000D80F0020A01A002010B5041E10DA002405
:1035F0000A4BA400E25801239340094A0949136089
:10360000094A1160094A0A4911600A4A136010BD4B
:10361000FFF75CF9A042EADDEAE7C046ECCA000029
:10362000D00F002008050050C80F0020C40F002054
:103630000C050050180500502B4BF7B51B680C000B
:10364000002B03D101204042FFF7CEFF2468012662
:10365000250035401AD0FF2263101202601210407C
:10366000DAB21043FF221B021204134018431F4B0F
:103670001B68202B06D1B4401D4BA40EA400E358B8
:1036800000021843FFF7C2FD0020FEBD042CFBD949
:103690000F2322681340092BF6D1FF2763683F02EE
:1036A0005B100193019B9D42EEDAAB00E3189B682F
:1036B000334216D05A105812D1B238400843FF2175
:1036C000120209040A401043084A1268202A06D14F
:1036D0005B009B0E06499B00020258581043FFF7FF
:1036E00095FD0135DEE7C046D00F00200800002020
:1036F00054C000000200086810B5C3070FD5401081
:103700001823012A03DD4A68042A00D10833054A38
:103710001360FFF7FDF8FFF767FF002010BD0120E1
:103720004042EDE708000020086810B5C30703D544
:10373000FFF744FE054B1860054B1B68002B03D0B8
:10374000024B186802F06AF9002010BDD80F002063
:10375000A01A00207FB5A04C2368002B0AD19F4AF5
:103760001268002A06D19E4B1B68002B01D0FFF780
:103770009BFD7FBD9B4D2A68002A26D1984A12687E
:10378000002A1BD0FFF790FD0028F2D0FFF778FD4C
:10379000924B24681A681C60002A16D0002C14D1A1
:1037A00001AD0C229049280006F0E2FD285D0021C1
:1037B0000134FFF78DF80C2CF8D1DAE7874A12684C
:1037C000002AE5D1002BE3D0E0E700211A2002F027
:1037D000EBFF00211B2002F0E7FF00211C2002F07C
:1037E000E3FF2E68012E5CD0022E00D1A2E0002E55
:1037F00050D101363100794C03202368994302F0FF
:10380000D3FF0420216801404B42594102F0CCFF14
:10381000102123680A2019404B42594102F0C4FF8D
:1038200080212368090119404B425941062002F0CA
:10383000BBFF80212368090219404B4259410720F0
:1038400002F0B2FF80212368490219404B425941DE
:10385000092002F0A9FF80212368890219404B4208
:103860005941192002F0A0FF80212368C9021940A4
:103870004B425941182002F097FF802321681B0317
:1038800019404B425941172002F08EFF31001A2097
:1038900002F08AFF2B680321581C04F027FD2960E1
:1038A00067E702214D4C1720236819404B425941CC
:1038B00002F07AFF08212368182019404B42594131
:1038C00002F072FF80212368C90019404B42594120
:1038D000042002F069FF80212368490119404B420E
:1038E00059410A2002F060FF80212368C901194074
:1038F0004B425941032002F057FF8021236889037E
:1039000019404B425941092002F04EFF80232168A3
:103910001B0419404B425941192002F045FF310068
:10392000062002F041FF3100072002F03DFF310088
:103930001B20ADE72021294C1720236819404B425A
:10394000594102F031FF40212368182019404B42B1
:10395000594102F029FF80212368192019404B4268
:10396000594102F021FF80212368490019404B4250
:103970005941092002F018FF80212368890019406D
:103980004B425941072002F00FFF80212368890133
:1039900019404B425941062002F006FF802123685E
:1039A000490319404B4259410A2002F0FDFE802193
:1039B0002368C90319404B425941032002F0F4FE29
:1039C000802321685B0419404B425941042002F0D6
:1039D000EBFE01211C205BE7D80F0020CC0F00205C
:1039E000DC0F0020C00F002064BE0000012010B5D5
:1039F0004042FFF7F9FD10BD10B5034A0921034805
:103A000000F074FF10BDC04654C100009CC100000E
:103A100030B502248025094B094AED009C505C59C1
:103A2000002CFCD0A124E400884202D3002199504C
:103A300030BD8025ED0018514019F5E700E0014048
:103A40000405000010B5002806D1C020B0214002B6
:103A50008902FFF7DDFF10BDB02080218002C9027E
:103A6000F7E7000043425841064B40421840B0235C
:103A70009B02C018036800201A0E532A01D11B02B2
:103A8000180A704700C0FEFF30B501248025054BA1
:103A9000054AED009C505C59002CFCD001600021CF
:103AA000995030BD00E001400405000043425841F8
:103AB000074B40421840B0239B02C018A62310B504
:103AC0000902DB05090A1943FFF7DEFF10BDC046F6
:103AD00000C0FEFF70B5012480250D4B0D4EED009A
:103AE0009C515C59002CFCD0002902DC00229A5128
:103AF00070BD557814782D0225439478013924043B
:103B00002543D478043224062C4310C0ECE7C04689
:103B100000E001400405000070B505004B680A0094
:103B20009C1C2100A400FFF7D5FF281970BD0000E0
:103B3000134B1B68002B0CD08022B023D2029B02B7
:103B400000280BD11A1D5B681B0E522B00D11000F0
:103B50007047B022C02392025B02F1E782420DD986
:103B600003681B0E522B09D1436802339B00C01817
:103B7000824203D903681B0E522BE9D00020E7E7ED
:103B8000E010002070B50020FFF7D2FFFF260500EF
:103B9000002801D1280070BD03681C143440FFF7D1
:103BA000C7FFDA2CF4D10500F2E700008022F0B55F
:103BB0005200A1B00021674806F0F6FB80220021E8
:103BC0005200654806F0F0FB644BFF271B681A00A3
:103BD000049353425A4110000592FFF733FF049CAF
:103BE0000020631E9C415E4B64421C405D4BE41808
:103BF000FFF7C8FF0600002E2DD10498FFF732FF13
:103C0000411C0598FFF752FF059A574D534B2C6006
:103C10001A60FEF7D1FF514B64201B68A0215A4265
:103C200053414F4A5B421340B0222C6892029B18CA
:103C3000E41A6043490204F073FAA022520203001E
:103C400000924A49220007A806F0F2FE07A801F0F8
:103C500067F821B0F0BD3268131412123A403B40AD
:103C600003921A000A3A092A49D83A4B039A995CF6
:103C7000002931D110223E4806F096FB35002B6812
:103C800003991A123A40914209D11A143A400B2A68
:103C900027D0132A2DD00A2A01D1354B1D602800C8
:103CA000FFF746FF051EEAD1314B196800290FD0F6
:103CB0002000FFF731FF04002D4B5B1959680029E4
:103CC00003D02000FFF728FF040004350C2DF3D1AA
:103CD000204B0121039A99543000FFF729FF060079
:103CE00089E73B40022BDADC214A9B00D3185D6058
:103CF000D5E7102200211E4806F056FBCFE71A0038
:103D0000153A082AE8D8144A0399525C002AE3D1EC
:103D10003500152B00D01500300003681A143A4006
:103D2000152A0FD01D2A00D10025FFF701FF00281A
:103D3000F3D1002D04D020002900FFF7EDFE040090
:103D4000054BC6E7039A1B123B409A42EDD1050092
:103D5000EBE7C046E00F0020E8100020E010002054
:103D600000C0FEFF04C00200E410002035C20000C5
:103D7000DC2E0020F0B50020B7B00024FFF7D8FEFD
:103D8000270005002600002D2ED1284D2868FFF7BA
:103D900069FE32003B0001900094254904A806F01A
:103DA00047FE04A800F0BCFF224B64201C682B686F
:103DB000A0215A425341204A5B421340B022920252
:103DC0009B18E41A6043490204F0AAF9A0225202A7
:103DD000030000921949220004A806F029FE04A855
:103DE00000F09EFF37B0F0BDFF226B6829689C464B
:103DF0000233FF180B12013613409C4200DA1C00FC
:103E0000FF200A1402400392624601400192009191
:103E1000039A0B4904A806F00BFE04A800F080FFEB
:103E20002800FFF785FE0500ADE7C046E010002042
:103E3000A6C20000E410002000C0FEFF50C2000037
:103E400092C2000070B50020FFF70CFE04000120B4
:103E5000FFF708FE844200DA04000A4B1D686A423C
:103E6000554128001D60FFF7EDFDA0226B42520274
:103E70001340054A28009B18044A611C1360FFF791
:103E800015FE70BDE010002004800100E410002049
:103E9000F8B50020FFF7E6FD07000120FFF7E2FD7F
:103EA0003E00204D0643204C0DD18021C020C90288
:103EB0004002FFF7ADFD01213000FFF7F7FD1B4B7E
:103EC0002E6023601DE0874209DD0023B0212B60B6
:103ED000164B8902236023680020012517E0012387
:103EE00080212B60124BC9022360F4E7120E522A84
:103EF00008D0002800D023600E4800F011FFFFF723
:103F0000A1FFF8BD28005A68023292009B188B422C
:103F100005D21A68561CE9D10028F2D0D1E72160F9
:103F2000EFE7C046E0100020E4100020048001000C
:103F300004C002006BC20000F0B585B003920322FA
:103F40000333DC17294D1440E4182B68284F5A42DC
:103F5000534180225B42D202A4103B409B18A21C1A
:103F60000291244E910000910190316800980A1846
:103F7000934215D2FFF71AFE2B685A425341802212
:103F80005B421F40D202BF183368009A9B189F42C1
:103F900006D2194800F0C4FE0025280005B0F0BD87
:103FA000029B356819066B461A7BA423DB05134375
:103FB000FF222F00090C1943019B12041B0413401C
:103FC00019432800FFF760FD0837281D21003760DE
:103FD000FFF75AFD002C04D00A9A21003800FFF7A1
:103FE00079FD009B083BFF183760D6E7E010002002
:103FF00000C0FEFFE41000200FC2000010B5FFF764
:10400000D5FD10BD70B59AB0FFF742FFFF221E4CE0
:10401000D2000021200006F0C7F9FF25FFF7B2FD0E
:104020000026002814D10200C300E3580130591EB5
:104030008B41D218FF28F7D1144901A806F0F8FCEB
:1040400001A800F06DFE124800F06AFE1AB070BDC3
:1040500003681A142A400A2A0AD11A122A40FF2A8F
:1040600003D0D200A1180B71A050FFF761FDD8E773
:10407000132AFAD11B122B40FF2BF6D0DB00E218DB
:104080001671E650F1E7C04654250020DBC200005F
:10409000EFC200000021094B094A5960013151600B
:1040A00059680029FCD00021196101239360022284
:1040B000044B8131FF315A501A607047FC100040A8
:1040C0000010004000E100E00222064B0121DA6707
:1040D0000022054B5A61054A11615A69002AFCD039
:1040E0007047C04604E100E0FC10004000100040B2
:1040F00010B5044C2378002B01D0FFF7E5FF00201A
:10410000207010BDE91100200120024B1B685B00EC
:10411000184370476C12002003480368002B02D13B
:104120001422037102607047042F00200120024B0B
:104130001B685B00184370470C00002070B504003A
:104140000D001600FEF7B6FB8023012200215B055F
:104150005B6E6270E270020AA271020CE2711A0ACE
:1041600060716372000EA2721A0C1B0E267025710C
:10417000A1702072E272237370BD0000124B10B563
:104180001B68124C5A1C0FD0114C002B0CD0114C38
:10419000012B09D0104C022B06D00D4C042B03D060
:1041A0000E4C052B00D10B4C21000D4806F078FC7D
:1041B000200006F07DFC0300042204339B0809481C
:1041C0001B011343036010BD1000002077C30000E3
:1041D00070C3000082C3000087C300007CC30000DE
:1041E000F02E0020EC2E002070B5214C2278002A01
:1041F0003DD1204B01215A608022D20511605A68BE
:10420000002AFCD0002207201B4B1C4901255A50D4
:104210000439585008315A5019481A4958501A4907
:104220001A485A501A495A50A622D2009D500822C4
:1042300018495A500431585002201749585017490C
:1042400017485850174804395850182016495850E4
:10425000C12189005A500539FF3958589218024334
:104260005A501249124A9950FFF714FF257070BD39
:10427000E9110020FC000040001000400C05000087
:10428000746962751C05000024050000200004020A
:104290002C05000014050000340500003C0500005A
:1042A000FFFF00002110010054050000EA1100206A
:1042B0000405000070B50E4B06001B78002B01D1E1
:1042C000FFF792FF00200B4D2C7884420ED00A4B52
:1042D000202219780323091B1940084B4901C918EA
:1042E000300006F045F80120013C2C7070BDC0463E
:1042F000E911002070120020E8110020EA110020CE
:10430000002370B588B0984227DD0D6801262C0087
:1043100034409C4221D12300042D1ED90F222B684A
:104320001A402300092A18D16A681F2A15D968463D
:10433000FFF7C0FF230000280FD06B461978330029
:10434000A14203DB6B461B5D5B003343A200AA184E
:1043500001349360202CF2D10423180008B070BD02
:1043600070B5414B8AB01B78002B01D1FFF73CFFA1
:1043700002AD2800FFF79EFF002802D100200AB0FE
:1043800070BD2B780B2BF9D96B78012BF6D1EB781C
:10439000012BF3D10023354E354C336023712B793B
:1043A000344A1360002B0ED1152169444A780B78EA
:1043B00012021A438B781B041A43CB781B06134353
:1043C0003360002318E0012B20D1152169444A787D
:1043D0000B7812021A438B781B041A43CB781A21EC
:1043E0001B06134333600E236A7C6944934200DD4D
:1043F000130000229A4232D104200021E218043333
:104400009B101B01034311712360B8E7022B03D1FA
:104410006A7B10331621E8E7042B0DD11521082201
:104420006944684605F0A4FF0098019902F02EFA4D
:1044300005F050FE3060C4E7052BC2D115210822DB
:104440006944684605F094FF0098019902F01EFA4D
:1044500005F040FE30606A7D0A231E21C5E78D5CB1
:10446000A01805710132C5E7E91100206C12002087
:10447000042F00201000002010B5134B04001B78FF
:10448000002B01D1FFF7B0FEFFF71EFE00200F4A00
:104490000F49104B54505860013010605868002884
:1044A000FCD0002018610130906018690028FCD011
:1044B000094B0A481B785B011B185350FFF704FE99
:1044C000FFF7E8FD10BDC046E911002000100040D4
:1044D00004050000FC100040E8110020EA11002053
:1044E00010B588B000281DDD0A68012113000B40BB
:1044F00018D1042A16D90F2014682040092811D198
:1045000050681F280ED998001018806800240842AF
:1045100001D04010C4B26846C4540133202BF2D1FC
:10452000FFF7AAFF002008B010BD000010B500285A
:1045300013DD0C68E30710D56410532C0DD8084B1D
:104540001B78002B01D1FFF74FFEFFF7BDFDA12324
:10455000044ADB00D450FFF79DFD002010BDC0468B
:10456000E91100200010004010B500280EDD0C6895
:10457000E3070BD56410FF2C08D8054B1B78002BE4
:1045800001D1FFF731FE034A034BD450002010BD88
:10459000E9110020001000402405000013B5002898
:1045A00014DD0C68E30711D5094B64100093094B27
:1045B0000193072C0AD8084B1B78002B01D1FFF779
:1045C00013FE6B46054A1957054BD150002016BD06
:1045D000E2ECF0F4F8FC0004E911002000100040C7
:1045E0000C05000070B588B0002820DD01240868A3
:1045F00004401CD104281AD90F2302681340042B4D
:1046000015D1FEF74BFB060006F052FA0500122802
:1046100000D912252A0002210D326846FFF78EFDCF
:104620006B465D73A54205DC6846FFF725FF002059
:1046300008B070BD2300325D6B449A730134F1E71A
:10464000F0B50D008BB0012832DD086801220400AE
:1046500014402DD104282BD90F2301680B40042BC3
:1046600026D16B68134223D0FEF718FB6E68070053
:104670007310019306F01CFA05000E2800D90E25D0
:104680002A000121113202A8FFF758FD6A4612796B
:1046900002AB5A7302AA73129373019B76141B0E1A
:1046A000D67313745574A54205DC02A8FFF7E4FE27
:1046B00000200BB0F0BD3A5D02A963189A74013472
:1046C000F1E730B589B0002814DD0C68E30711D597
:1046D000102268460021FFF731FD6B466A466510DF
:1046E0005D73684663122D0E64149373D47315744E
:1046F000FFF7C2FE002009B030BD0000174B184A7A
:104700005968002903D0002159600131916019696D
:1047100000291FD0002018618023DB00D3581149E5
:10472000012B18D1A923DB00D3585B420B600E4943
:104730000B78032B01D801330B7003200B490B7846
:10474000013303400B700A495B015B180949535060
:104750000123936070470860FAE7C046FC100040F0
:10476000001000400C00002070120020E811002012
:10477000EA1100200405000010B5034A0E21034889
:1047800000F0B4F810BDC04600C30000F7C200003E
:10479000044A05491368C85401339B059B0D1360F7
:1047A0007047C0468C1600208C12002070B5114C4A
:1047B000114A2368834202DC0023236016E0155C63
:1047C000411C2E00FA3E012E05D899420FDA555CA5
:1047D000013D1F2D01D90800ECE70100151A565CB8
:1047E0006E5401318B42FADC181A206070BD1570CE
:1047F000FAE7C046981A00209816002010B5FEF778
:104800004FF8064B1A68824201D900221A601B68D1
:10481000C31A034898428041404210BD88120020CC
:10482000204E000010B5094C094A236812689342D3
:1048300000D110BD074AD05CFEF7B6F90028F8D0C9
:10484000236801339B059B0D2360ECE79016002045
:104850008C1600208C12002010B50400064B074A6D
:104860001B6812689B1ADB439B059B0DA34200DB70
:1048700010BDFFF7D7FFF1E78C160020901600203F
:10488000F7B5050056680191B000441C06301700CA
:10489000FFF7E2FFFB20FFF77BFF1C20FFF778FF0D
:1048A000E8B2FFF775FFE0B22412FFF771FFE0B244
:1048B000FFF76EFF6B461879FFF76AFF0025AE42DF
:1048C00000DCF7BDAB00FB189C680135E0B2FFF7D8
:1048D0005FFF2012C0B2FFF75BFF2014C0B2FFF7EA
:1048E00057FF200EFFF754FFE9E7000070B5074EB1
:1048F0003368092B08DC0C255D43054C0133285136
:1049000064196160A260336070BDC04694160020D7
:10491000282F0020F0B587B002900C00012803DC9E
:104920001B20FCF711FB45E0244B08680093C307EC
:1049300009D4042807D90F2302681340042B02D19D
:10494000FEF7ACF900901D4B60680193C30709D4D2
:10495000042807D90F2302681340042B02D1FEF765
:104960009DF901900027164B1B680493049BBB42E2
:10497000D6DD0C267E43134B0099F618306806F0FE
:1049800085F8051E05D17368B6680593059B9D42A1
:1049900001DB0137EAE730680199039606F076F803
:1049A0000836002808D121000298039B08310238FC
:1049B0005B68984707B0F0BD0135E7E767BD0000C9
:1049C00094160020282F002010B5FCF709FAFFF7F5
:1049D00013F8FEF78BF8FEF7C9FBFEF7FFFBFFF7B6
:1049E000CBFE00F041FE01F01BF810BD962210B581
:1049F00012010021034805F0D7FC0022024B1A6087
:104A000010BDC046F41B0020B4050020064B074A29
:104A10001B6812689B1ADB439B059B0D0122834296
:104A200000DC0022100070478C1600209016002039
:104A3000F8B505000C0016001F1E0ED10320FFF76D
:104A4000E5FF002808D0FA20FFF7A2FEE8B2FFF742
:104A50009FFEE0B2FFF79CFEF8BD501DFFF7D6FFAA
:104A60000028F9D0FB20FFF793FEE8B2FFF790FE95
:104A7000E0B2FFF78DFEF0B2FFF78AFE3012C0B24F
:104A8000FFF786FE3C00E31B9E42E5DD2078FFF742
:104A90007FFE0134F7E7000070B50024F0250B4BD2
:104AA0001B68A34202DCFFF7A1FF70BD2B0063432C
:104AB000074A9B181A78002A05D05978002311203C
:104AC0001A00FFF7B5FF0134E9E7C046B40500203E
:104AD000F41B0020F8B507000024F0252B006343E9
:104AE0000C4A01349E18B74211D0317800290BD0FE
:104AF0000133D15C002311201A00FFF799FF2A002F
:104B00000021300005F050FC0A2CE7D1F8BD024B23
:104B10001C60F9E7F41B0020B4050020FFB5012359
:104B20001700FFB00190029115001F4011D004AA98
:104B300013706B1004A953706A128A7005221B0E41
:104B40006D140B71CD700B000299FFF771FF7FB0F0
:104B5000FFBD042A1FD90F2312681340042B26D14E
:104B6000023B04AA28001370FEF798F8040005F031
:104B70009FFFF823FF33984200D91800B84204DCA5
:104B8000421C04AB02990198DFE701377B1EE35C0E
:104B900004AAD355F2E7042A7ED1032304AA043DD4
:104BA00013706B425D41130055700222EAE7092B36
:104BB000CDD16946053B04AA13706B685A10009268
:104BC0005B1204AA09789370009B5170132B01DDCE
:104BD000142300936A46127804ABDA7005AC009B8C
:104BE000BB4202DC04ABE21ACCE70126BB00EB18A7
:104BF0009868064006D1042837D90F23026813406D
:104C0000022B0CD1012323704310637042121B0E40
:104C10004014A270E070237105340137DFE7042BE4
:104C200021D1023B2370FEF739F8039005F040FFD5
:104C3000A31C0C2809D86070864201D19C19ECE7AE
:104C4000039A925D9A550136F6E70C226270039A38
:104C5000925D9A550136092EF9D12E23E372237302
:104C600063730E34D9E7012B07D103230438237073
:104C70004342584160700234CFE7092B09D1053B0C
:104C800023704368E6705A105B126270A37004349C
:104C9000C3E726700134C0E7002A00D057E77CE75D
:104CA00070B502000024F0210D4E08006043801909
:104CB0004578954203D001340A2CF6D170BDF0221C
:104CC000002105F071FB074A1368013BA34200D1A4
:104CD0001460002329001A001120FFF7A9FEEDE758
:104CE000F41B0020B405002010B5B2B002236A46C0
:104CF0000400137005F0DCFEC72800D9C72000238C
:104D0000984207DC421C6B46FE211420FFF790FE00
:104D100032B010BD694601335A1EA25CCA54EFE797
:104D200030B5B3B002236A460500137005F0C0FE2B
:104D30000400C72800D9C72400239C420BDC2000B4
:104D40003230FFF789FD621C6B46FF211420FFF70C
:104D50006FFE33B030BD694601335A1EAA5CCA5497
:104D6000EBE70000F7B5234B06001B68F02100932A
:104D70000023009A9A4211DC0024F0231A006243B7
:104D8000019201991C4A55182F78002F12D0013436
:104D90000A2CF3D11948FFF7C3FF29E00A005A4350
:104DA000154882185078B04202D11278002A1FD1DB
:104DB0000133DEE7F0223900280005F0F5FA02237E
:104DC0000D4A0199EB6053540D4AF1008A58009B3B
:104DD0006E70AE70AA602F616F61A34202DC054B5A
:104DE00001341C60002331001A001020FFF720FE60
:104DF000F7BDC046B4050020F41B002071C80000B8
:104E00005425002010B5FFF747FEFF24084AE300B1
:104E10005B429B18074AD35C043B012B03D8E04359
:104E2000C0B2FFF79FFF013C002CEFD110BDC04680
:104E3000FC07000054250020F7B50E00FF247F2555
:104E400001901C4AE300D31A1B4A9A181278062ACA
:104E500001D0032A1DD1FF22D2009B181868836855
:104E60002B401C2B15D1C3681A002A40042A10D1EC
:104E700002692A40192A0CD11B0A01339B000C300D
:104E8000C018FDF70BFF070005F012FE0023B0422B
:104E900009D0013C002CD4D1F7BD019AF95CD25C59
:104EA0009142F6D101339E42F7DCE043C0B2FFF7F6
:104EB00059FFEEE754250020FC07000070B50500FF
:104EC000FF24084AE3005B429B18074AD35CAB42CD
:104ED00003D1E043C0B2FFF745FF013C002CF0D105
:104EE00070BDC046FC07000054250020F7B5FDF753
:104EF000D7FC514B1A68824201D900221A601A6805
:104F00004E49821A8A4200D883E01860FDF7D2FC2D
:104F1000071E00D101370020FDF7BEFD01900020E3
:104F2000FDF7CEFD019B0090454C464D002B14D063
:104F30002368002B00D07AE02B682760002B00D17B
:104F400071E0414B01261B78002B63D10920FFF74C
:104F5000B5FF3E4B1E703C4B1E70009B002B12D0C9
:104F60002B68002B0FD123682F60002B1ED0374BEE
:104F700001261B78002B52D10920FFF79FFF334BEE
:104F80001E70314B1E702368002B0FD02F4E3278CD
:104F9000002A0BD19F4200D227602368FB1A312BD5
:104FA00004D90720FFF78AFF012333702B68002BF9
:104FB0000FD0254E3278002A0BD1BB4200D92F608A
:104FC0002B68FF1A312F04D90820FFF777FF012340
:104FD00033702368002B0CD0019B002B09D11B4E92
:104FE0003378002B02D10720FFF768FF00232360EE
:104FF00033702B68002B0CD0009B002B09D1124C76
:105000002378002B02D10820FFF758FF00232B60E4
:105010002370F7BD0720FFF751FF0C4B9CE70820DA
:10502000FFF74CFFADE7009B002B9CD1ABE7009A4C
:10503000002A95D1AAE7C046841200200F2700005D
:10504000741200207C1200208012002078120020B0
:1050500037B500240500FFF71FFD01A80194FDF7F7
:1050600009FD21002000FEF7E7F9FEF773FBFDF7CD
:105070003BFDFDF73AFDFEF7B9FCFDF737FCA54215
:1050800004D0FDF7BBFD0248FFF74AFE37BDC0461E
:1050900062C80000002310B501001A001120FFF7BC
:1050A000C7FC10BD07B56B46197069465A701312DC
:1050B0008B701314120ECB700A716B46010005221F
:1050C0001320FFF7B5FC07BD10B50A000100122040
:1050D000FFF724FD10BD70B5050008000C0032304C
:1050E000FFF7BAFB2B00220000211B20FFF7A0FCDA
:1050F00070BD10B50C000300110014202200FFF752
:1051000097FC10BD012370B5FF24084A41185B428B
:10511000884201D3D84370BD06781D0A23407340EE
:105120009B009B5801306B40F2E7C04644C400002E
:10513000002313B501930B4BC2000400D058002884
:1051400005D0436808309900FFF7DCFF0190092083
:10515000FFF782FB01AB042221001720FFF768FC58
:1051600013BDC0465425002070B506000020FEF790
:10517000DFFC0024FF25002801D1200070BD03685A
:105180001A142A40152A07D11B122B40B34200D112
:105190000400FEF7CDFCEEE71D2AFAD10024F8E763
:1051A000F0B580279DB0FFF73DFBAD4CAD4D2068BD
:1051B000FF00391A4019FDF7DDFC23680600C3180B
:1051C0002360002B0ED11DB0F0BD2068391A2818BD
:1051D000FDF7D0FC236806001B182360FDF760FB79
:1051E000A14B1860002EF0DC2B78FA2B00D013E1D5
:1051F0002368022B07DCFFF701FB0028E3D0012026
:10520000FFF7D4FADFE76878AC78023818281FD89F
:1052100002F0F2FE0D2024282B341E3E6872768C9C
:10522000DEEF1E1E1E1E1E1E1E1E1E1EFD00FF2C5D
:105230000ED02000FFF734FD00228C4BE100CA5055
:105240005B181A712100009213001320FEF774FE00
:105250000320D5E72000FFF785FDF9E72000FFF7E1
:105260001FFDF5E7FFF7CEFDF2E7FFF715FC002085
:10527000FFF7EEFE7E48FFF753FDE9E7632CE7D822
:105280007C4BA200D25821001520FFF747FCDFE736
:1052900000242000FFF768FF061E03D10134642CB0
:1052A000F7D1D5E7083005F003FC05000530FFF71E
:1052B000D3FAFB20FFF76CFA1D20FFF769FAE0B282
:1052C000FFF766FAE8B2FFF763FA2812C0B2FFF7F9
:1052D0005FFA3700BB1B9D42E0DD387AFFF758FAD2
:1052E0000137F7E700211D2000910B000A00FEF7AF
:1052F00023FEFDF783FCABE72000FFF719FFA7E7CC
:10530000FDF7E0FA03AC5C4A642100905B4B20009F
:1053100005F05CFB02232000237005F0C9FB23008D
:10532000020000211620FFF783FB91E700244F4A7B
:10533000E300D558002D28D06B689E00701DFFF744
:105340008BFA2B0000253200083321000120FFF7E3
:105350006FFB0020FEF7ECFB2F002E00002818D179
:10536000002F04D03A0001212000FFF789FA002D18
:1053700004D02A0002212000FFF782FA002E04D078
:10538000320000212000FFF77BFA0134FF2CCED140
:105390005EE7FF2103681A120A40A24209D11A14DB
:1053A0000A400B2A08D10B400CD0012B0CD0022B49
:1053B0000CD0FEF7BDFBD1E7132AFAD100252F0050
:1053C0002E00F6E70600F4E70700F2E70500F0E735
:1053D0000024FFF761FB2200210000942300DA2063
:1053E000FEF7AAFDFF222100D200204804F0DCFFD6
:1053F0007FE7012C02D1FEF7BDFC29E7022C02D188
:10540000FEF7FCFD24E70120FFF722FE20E7002342
:1054100021001A001A2086E7FB2B00D0EFE6226855
:10542000042A00DCE7E62E79E878154B36020643BD
:105430009E4200DDE3E6331D9A4200DCDBE6EB5CD6
:10544000FE2B00D0DBE66B78AC78711E1B2B6BD08B
:1054500018D8012B2BD0082B3DD0701DD0E6C046AC
:10546000981A002098160020881200205425002049
:1054700044C800004C2D00205BC8000056C8000046
:10548000F60300001D2B60D052D31E2BE5D1012C5A
:10549000E3D10029E1DD6B79002B03D01C00322B16
:1054A00000DD322464235C43344B1C60D5E7FF2CC1
:1054B000D3D02000FFF7F4FB6D79314AB31E009280
:1054C00021002A000A20FEF737FD2E4BE400E050B1
:1054D0001B191D71C1E7632CBFD86A79022A13D04A
:1054E000032A1BD0012AB8D1E979AB790902194303
:1054F0002B7AA4001B0419436B7A1B060B435B0039
:105500001343214AA350A8E70029A6DDB11E1C4879
:10551000FDF7C6FD1C4BA400E0509EE7AB79A4004C
:105520005A1E93419B00ECE71848FFF785FC94E76F
:10553000FF2C92D06A79022A8FD811490B20009152
:105540002100B31EFEF7F8FC87E70B00632900DD9E
:105550006323002203A893420ADCD9430022C9171F
:10556000194041180A700133009021001520E9E725
:10557000A918497981540132EDE7C04604000020A2
:105580009E160020542500204C2D00209D16002042
:105590000122094B1A60094A1368002BFCD0032230
:1055A000074B1B68D8171040C0180123801006381D
:1055B000400018437047C04600C0004000C1004092
:1055C00008C500400120704710B5064C200000F0CF
:1055D0005DFB0549200000F081FB0122034B1A60AE
:1055E00010BDC046C41A0020801A06009C1A002074
:1055F00010B501210D20FDF76BF901210E20FDF7FB
:1056000067F900210F20FDF763F9044C200000F03A
:1056100079FA1021200000F091FA10BDA41A0020A0
:1056200010B504680D20E30703D56410FF2C03D9DF
:105630001720FBF789FC10BDFFF7DAFFE1B2024843
:1056400000F09EFA0020F6E7A41A002010B5FFF73C
:10565000CFFF0021034800F093FA430001201843D4
:1056600010BDC046A41A002010B5034A0821034803
:10567000FFF73CF910BDC04688C80000C8C800004C
:105680000D4B70B51B6804000E001500002B01D1F6
:10569000FFF79AFFE1B2094C200000F0B6FBF1B22F
:1056A000200000F0B9FAE9B2200000F0B5FA2000BD
:1056B00000F016FC70BDC0469C1A0020C41A0020E1
:1056C00010B501240368234205D04168214202D06D
:1056D0008268224203D10D20FBF736FC10BD581022
:1056E000802801D91520F7E74910FF2901D9162094
:1056F000F2E75210FF2A01D91720EDE7FFF7C0FFAC
:105700000020EBE7F7B501242300A0421DDD0D6862
:105710002C421AD01A4B25411B684C68002B01D132
:10572000FFF752FFE9B201272500164E3D40300039
:1057300000F06BFB002D0AD03C413000E1B200F0DC
:105740006BFA300000F0CCFB00231800FEBD042CE7
:10575000F7D90F2322681340092BF2D163685B103D
:105760000193019BAB42ECDDAB00E3189968394231
:1057700004D04910C9B2300000F04EFA0135F0E70C
:105780009C1A0020C41A0020144B70B51B68050039
:105790000E00002B01D1FFF717FF114CEDB22900CD
:1057A000200000F032FBF1B2200000F035FA0021B9
:1057B000200000F035FB002801D0404270BD0122DE
:1057C0002900200000F01CFB200000F016FA002841
:1057D000FAD0200000F016FAF0E7C0469C1A00202C
:1057E000C41A002010B501240368234202D0416886
:1057F000214203D10D20FBF7A7FB10BD58108028D4
:1058000001D91520F7E74910FF2901D91620F2E741
:10581000FFF7BAFF40002043EFE70000002370B518
:10582000344D0400EB5601330BD10D211D20FFF741
:10583000ABFF5A2814D101222A212A703D38FFF7E4
:105840001FFF0023EB56022B2AD0032B49D0012B3C
:105850004CD121001D200124FFF796FF644225E072
:105860000F211920FFF790FF332805D102235F2273
:105870002B7020211A38E2E70D211E20FFF784FF4C
:10588000C7280AD1032300222A21A9382B70FFF749
:10589000F7FE1B222A211E20D1E700232B70D0E720
:1058A000012C13D129211920FFF76EFF7F2801DD7C
:1058B0000138FF3803007F3301DA7F204042642340
:1058C0007F21584302F02CFC604370BD032C0BD1A8
:1058D0002B211920FFF758FF043CE7E72D21192061
:1058E000B9E721001E20B6E7052CF7D001240020DF
:1058F0006442E4E71400002070B50120FFF78EFF3A
:1059000004000320FFF78AFF05000520FFF786FF4C
:105910006D43644340436419201804F011FC01F006
:10592000E5F804F0D7FB43000120184370BD10B523
:105930000120FFF773FF43000120184310BD10B58D
:105940000320FFF76BFF43000120184310BD10B583
:105950000520FFF763FF43000120184310BD00003E
:10596000F8B501231C00984234DD0F683B4231D06A
:105970004E6835001D402DD1042E2BD90F223168E1
:105980000A40092A26D173685C10202C00DD2024EF
:10599000114B1B68002B01D1FFF716FE7F10F9B2E7
:1059A0000E4F2200380000F02BFAA5420FDA380023
:1059B00000F023F90028FAD0380000F023F9012282
:1059C000AB004000F31810439860AD18EDE70120DC
:1059D000640004432000F8BD9C1A0020C41A002073
:1059E000002070470120704700207047002070475A
:1059F000012070470020704700207047002070474A
:105A0000002070470020704700207047002070473A
:105A100000207047002070477047704770470000B3
:105A200010B5034A0E210348FEF760FF10BDC046C3
:105A300018C9000088C9000010B5FDF763F8FDF72C
:105A4000FFF8FEF7C1FF0448FFF76AF9FEF7DAFA3C
:105A5000FFF7D8F910BDC04611CA000010B5FCF719
:105A6000B9FE10BD70B5002504AC24780573A942B9
:105A700005D10A4B0A4A23210A4804F00BFC0160B5
:105A80000949920052589B0002715B58A40083712F
:105A90006358856043710223C37170BD29CA000039
:105AA0008ECA000037CA0000ECCA0000037B002B3E
:105AB00004D14373837303610133037370470000A0
:105AC0001FB50191A02100240068C900D2B2445042
:105AD000012A10D0A24209D0032A0AD0074A8350D3
:105AE000074B019AC250012343501FBD02221343AA
:105AF000F4E70422FBE70622F9E7C046540500005C
:105B00002405000010B50400FFF7D0FFA122236890
:105B1000A179D20099506179064A200099502179E3
:105B200004329950044B19685A689B68FFF7C8FF04
:105B300010BDC0460C050000B81A00204BB2002B67
:105B40000FDB80233F290FD81F290FD80F290FD82B
:105B500007290FD803290FD81B060168074A8B5065
:105B6000704780239B04F8E7DB04F6E71B05F4E7A6
:105B70005B05F2E79B05F0E7DB05EEE72405000097
:105B80000368074A99501A00FC32D1680029FCD0FA
:105B9000A321C90058580023C0B2D3607047C04643
:105BA0001C05000007B58022074BD2051A600022B1
:105BB0009A6002321A710F230C3200930349023BA0
:105BC0000348FFF74FFF07BDB81A00200030004020
:105BD000A41A0020F8B505000E0017000024BC42EE
:105BE00008D02B68315D1B6828009847002801D039
:105BF0000134F4E72000F8BD704710B51C3000F008
:105C0000A9F910BD10B51C3000F096F910BD10B503
:105C10001C3000F0A5F910BD70B5437E0D00002BBF
:105C200001D1002070BD6430040000F0A2F900280A
:105C3000F7D12000290000F070F90120F2E7000000
:105C4000F7B50193FA23002504009B0083600D4BF8
:105C50004560083303601C300F00160000F052F955
:105C60002000643000F04EF9074A2761B600B358AF
:105C700020006375019B9B009B586576A576A375F4
:105C8000FEBDC046CCCA0000ECCA00000123A02221
:105C9000C375837D0E49C133FF33D2059B009950F4
:105CA000437DC133FF339B009950CC220169094BDE
:105CB0005204CA5005220169243BCA50827D016901
:105CC0000833CA500269417D034BD1507047C0462A
:105CD0000C060000240500000C050000A022002393
:105CE00010B50469D200A3500A4CA1420FD90A4C46
:105CF0008C425B4109495B420B40CD21C9045B18D2
:105D000004690749635005210369995010BDCC23EC
:105D10005B04F5E7A086010090D00300000098FD29
:105D200024050000F7B5040000200D000193824215
:105D300065D01600402A00D9402627001C373800BD
:105D400000F0F6F8B1232269DB00D5508022012350
:105D5000216992008B50A27E002A03D1226913622E
:105D6000226913600025731EAB4207D1019B002BF3
:105D700004D08022022123699200995001222369D4
:105D80001A622369FC33DA68002A02D19A6A002A6F
:105D9000F9D09A6A002A0BD1DA60A3232269DB00CA
:105DA000D1583800C9B2013500F0B7F8B542DAD39E
:105DB000019B2269002B0FD11300FC339B6A002B3F
:105DC0000AD10133A376D3612369FC33DA6C002A4C
:105DD000FCD00022DA640AE000230121A37651619D
:105DE0001A002369FC3399680029FCD09A60236962
:105DF000FC339A6A002A01D000229A62E8B2FEBD02
:105E000010B50123FFF78EFF10BD0300AC3310B5B2
:105E100004001970643000F08BF80123637610BD24
:105E20000023020070B5AC3243760D001178B12228
:105E300004000069D20081508022216992008B50B9
:105E400022690133136222699360260064363000B0
:105E500000F080F8002812D0300000F06DF81E4BE2
:105E60002269D0502369FC331A6A002A02D19A6A47
:105E7000002AF9D09A6A002A01D11A62E5E723695B
:105E80000122002D0DD11900FC31896A002908D1A9
:105E9000DA612369FC33DA6C002AFCD00022DA6470
:105EA00007E05A612369FC339A68002AFCD000227B
:105EB0009A6000202369FC339A6A82420BD0986270
:105EC0002169064A8B588B501800022B03D0181FEB
:105ED000431E9841033070BD1C050000C40400003F
:105EE00010B50121FFF79CFF10BD000010B5132372
:105EF000142202490248FFF7A3FE10BD00400040F3
:105F0000C41A002010B540220021040004F04CFA0D
:105F1000002320002364636410BD10B53F24026C8D
:105F2000531C2340446C9C4201D08154036410BD37
:105F30000023036443647047436C026C934206D0B1
:105F40003F21C25C01330B404364100070470120C5
:105F50004042FBE7036C406C181A00D54030704794
:105F6000436C026C934201D0C05C704701204042F8
:105F7000FBE73F22036C406C01331340181A434285
:105F80005841C0B27047000003210A4802680A4322
:105F90000260094802680A4302600849084A094B3E
:105FA0009B1A03DD043BC858D050FBDC00F012F80C
:105FB000FAF7AAF824050040540500403CD0000040
:105FC000000000204C020020FEE7FEE7FEE7FEE7AF
:105FD000FEE7FEE72D4B10B51A68D2B2012A0FD1A9
:105FE0002B4A126812070BD12A4AE0241168F022CA
:105FF0000800104021422DD12749096811422CD0B8
:106000001A68D2B2012A12D12149096809070ED1B2
:10601000F020204909680140402908D11E4909683B
:10602000014204D18020C121C005C90042501B6833
:10603000DBB2012B0DD1164B1B681B0709D1154B89
:106040001A68F0231A40A02A0FD1134A12681A4284
:106050000ED010BD3028CFD0D2E7104A10491160C1
:106060008021104A09021160CAE7D02AF1D1ECE779
:106070000D4B1A68012A04D00C4A1A601A68012ACA
:10608000FCD1C0220A4B1A60E3E7C046E00F00F0E3
:10609000E40F00F0E80F00F0EC0F00F00405004002
:1060A000DFFF07C0186C004000EC0640759300004D
:1060B00014EC06400120704710B503681322DB6919
:1060C000984710BD70470000054B0269D150036925
:1060D000FC331A6A002AFCD0002201201A627047A1
:1060E0001C050000030010B55C331A781F231A400A
:1060F0001E3B19009140114AD167C2220421046954
:106100009200A150026953600269D360A02300226B
:106110000169DB00CA5001230169094A5B428B50C7
:106120000169084A8B5001690C3A8B5001690832A9
:106130008B501430FFF7FCFE10BDC04604E100E0B8
:106140000C0500001405000010B51430FFF702FF25
:1061500010BD10B51430FFF703FF10BD10B514309B
:10616000FFF7EAFE10BD0000030070B55E331A7839
:106170000469724BE25003005D331A780469704B76
:10618000E250030061331C7802696E4B012C00D091
:106190009EE005005F352E78A225ED0056510200E5
:1061A00060321578A1220669D200B5500269D45038
:1061B0009623DB00994200D88CE096231B0199427C
:1061C00000D88AE096235B01994200D888E09623A4
:1061D0009B01994200D885E0E1239B01994200D8B8
:1061E00082E09623DB01994200D880E0E123DB01C5
:1061F000994200D87DE096231B02994200D87AE0AC
:10620000E1231B02994200D877E096235B02994272
:1062100000D874E0E1235B02994200D871E0E123E9
:106220009B02994200D86EE0474B994200D86CE03F
:10623000E123DB02994200D86AE0E1220023120345
:106240008A425B41414A5B421340802252059B18BF
:1062500001693F4A8B50A02304220169DB00CA5028
:1062600000210369FC33D9600369FC3319620123FF
:1062700001690B6001698B60C1210469890062506A
:106280001F215C3002780A4093406231314AFF316D
:1062900053500021415600293CDA0F230B40083BA4
:1062A0002D4C9B089B001B1903242140A140FC346A
:1062B0008C40DD69A5432C00C0258D402900214379
:1062C000D9611F23017819401E3B8B40136070BDBC
:1062D00000246CE79E23DB02BAE79D231B03B7E78C
:1062E0001E4BB5E71E4BB3E7EC239B03B0E71D4BFA
:1062F000AEE71D4BACE71D4BAAE71D4BA8E71D4BB6
:10630000A6E71D4BA4E71D4BA2E78023DB049FE714
:106310001B4B9DE78C080F4BA400E41803230B4094
:10632000FF21C025DB009940AD0066598E43310046
:10633000C0269E4033000B436351C2E70C050000AA
:10634000140500006C05000090D0030000D0BEFED4
:106350002405000000E100E000ED00E000B01300C3
:106360000050270000A04E0000F0750000509D0076
:1063700000F0EB0000903A0100E0D70100B0AF035D
:1063800000705F07F7B5009308AB1B7800250193F9
:10639000FA2304009B0083600E4B456008330360C2
:1063A00014300F001600FFF7ADFD23005C332761AA
:1063B0001E70009B084A9B00995823005D3319709A
:1063C000019B20009B009A5823005E33DD701A70F9
:1063D000FEBDC04670CB0000ECCA0000036910B5DA
:1063E0001A00FC32D2680400002A0AD0A322D2008C
:1063F00099581430C9B2FFF790FD00222369FC338D
:10640000DA6010BD10B50248FFF7E8FF10BDC046C6
:106410007C1B0020162307B5022200930249013B92
:106420000248FFF7AFFF07BD002000407C1B0020A3
:1064300010B5002801D004F073FA10BD70470000B9
:1064400010B500F011F8FFF7F9FF012000F000FA95
:10645000FFF7F2FAFFF702FB024B002BFAD000E045
:1064600000BFF7E700000000C420114B80001A585D
:1064700010491140C02212020A431A50C021802242
:10648000490092025A501A608023A3220021DB05A2
:10649000D20099500122F9309A60074BFF30195011
:1064A000C120023180001950403019501A607047E5
:1064B00000E100E0FF00FFFF00100140014B186009
:1064C0007047C04660000020F7B5002320285AD846
:1064D000384B8000C258042A5BD007D8022A54D017
:1064E00055D80423012A09D000234CE0062A54D0B1
:1064F00051D31A2A53D002231B2AF5D12E4A1168F0
:1065000008294ED909294FD00A240226A0200125A6
:106510002A4AC00015502A482A4D07681C20BF008F
:1065200007402948019700685759009027481B02E7
:1065300007401F43C02300989B020340FF20575190
:106540005759000207401F43019B1F43009B5801FE
:106550006023184007433E43565101251C4B1560EC
:1065600058680028FCD000205860A1230125DB00DA
:10657000D3585560A025ED0050511BB2A14202D066
:1065800015D2611ACB401800FEBD0823B6E71023D0
:10659000B4E72023B2E74023B0E78023AEE701232E
:1065A000ACE708240026B1E70C000126AEE7091B82
:1065B0008B40E8E7ECCA00005C000020007000405F
:1065C00018000020040500001C000020FF00FFFF51
:1065D000FC700040F0B520285BD8364B8000C258D4
:1065E000354B1E68002E30D1C227344BBF00D8591E
:1065F000334C03250440C02000022043D851C0245E
:1066000080206400800018512E4F18602E4B803C73
:10661000D859FF3CA043D8510437D859A843204348
:10662000D8510837D8590C35A84384460720654609
:106630002843D851A820C0001E50C12080268000C9
:1066400076021E501C601C4B1C60142500202B0081
:106650001E4C2E0046433659771C1BD14343E25053
:10666000A0230325C132FF329200DB05D550184B21
:106670001A68082A14D114234343E3189A6812486D
:106680005132FF32920059601150DA68C1239B00E9
:10669000C250F0BD9642E1D001300328D9D1F8E7CD
:1066A000082A02D9083AD140E5E708239A1A91400E
:1066B000E1E7C046ECCA0000E01B002000E100E07A
:1066C000FF00FFFF040500000090004020000020B4
:1066D000600000202149F0B54A6C2148002A14D0FE
:1066E000A025A12600230124ED05F600C258571C61
:1066F00006D0C7187F68002F02D027009740AF51FF
:1067000014333C2BF2D100234B64A0230121DB0581
:1067100000260F009C4614234B43C3181A1F12680F
:10672000104C0E4D920014195219526C002A10D0C0
:106730001A00143A1268551C09D0103B1B68FF2B35
:1067400005D03B00934065461A00074BEA50FC34E5
:10675000666401310429DED1F0BDC046FC900040E2
:1067600020000020009000400C05000000B520280B
:1067700010D80C4A8000835803290BD8A0220800A7
:10678000C133FF33D2059B0001F036FC0209050737
:106790000021D15000BD0C21FBE70421F9E70321C2
:1067A000F7E7C046ECCA000020280AD8074B800053
:1067B000C25801239340A022D205002902D10449E6
:1067C00053507047A121C900FAE7C046ECCA000047
:1067D0000C05000003000020202B0AD8A021A222D3
:1067E000C905D2008858034A9B009B58D840012312
:1067F00018407047ECCA0000F7B506000D000C0009
:106800008B180193019B671B9C4207D0336821784A
:106810001B683000984701340028F3D13800FEBDD2
:106820000849094A094B10B51B688858FA22190A09
:106830001B0618439200002301F0AAFD4904C00B77
:10684000084310BD0010014004050000E41B0020B7
:1068500070B5041E09D0FFF7E3FF050000F014F83F
:10686000FFF7DEFF401BA042F8D370BD0022044BAF
:106870009A60044A13680133DBB213607047C04664
:10688000FC100140E41B002070470000F0B5C64634
:1068900000B5CB0F9846404A4B005B0D9A1882B06A
:1068A0000D000400132A2FDC002A49DB3B4F17415F
:1068B0003E000E40064323D07F08390029400C4398
:1068C0000AD03749BD438C4663445C425C41802317
:1068D000DB021341E4071D434146CE0031492B0042
:1068E0008E192200346875682000290001F0F6FE38
:1068F000009001910098019922002B0003F086F886
:1069000002B004BC9046F0BD332A08DD8023DB00D2
:106910009A42F5D102000B0001F0E0FEF0E7224AB6
:106920009446012263445242DA400242E8D05208BF
:106930000242D1D094438022D2051A411443CBE7BE
:106940004B005B080343DBD00B031B0B1C43634270
:10695000234380244D0C24031B0B23406D042B4345
:1069600019004346DA000F4B9B181C685D68020053
:106970000B002000290001F0B1FE00900191009869
:10698000019922002B0003F041F842464B005B08BE
:10699000D60733431900B3E701FCFFFFFFFF0F00E9
:1069A000EEFBFFFFA0CB0000EDFBFFFFF8B5274A91
:1069B0004B005B0D9A180C000700132A10DC002A0C
:1069C00036DB234B13410B423AD08024240314417D
:1069D000002064189C430600250030002900F8BD03
:1069E000332A0EDD80230600DB000D009A42F4D12D
:1069F00002000B003800210001F070FE06000D00BF
:106A0000EBE7144D0600AC46012563446D42DD40C2
:106A1000AC4663460D000342DFD033239A1A323B63
:106A200093401818874200D94C1C63469843D2E71C
:106A3000C90FCC070020531CCDD1074B1C43CAE71C
:106A400006000D000028C0D1C7E7C04601FCFFFFCB
:106A5000FFFF0F00EDFBFFFF0000F03F30B5214AC4
:106A60004B0087B05B0893421EDD1F4A934205DD51
:106A700002000B0002F0CAFF07B030BD02AA00F00E
:106A800095F803231840049A059B012813D0022887
:106A90001DD0002814D00298039900F06FFB8023CA
:106AA0001B069C466144E7E7002300220093002375
:106AB00001F0DEF8E0E70298039900F05FFBDBE706
:106AC000012402980399009401F0D2F8D4E701243C
:106AD00002980399009401F0CBF880231B069C4692
:106AE0006144C9E7FB21E93FFFFFEF7FF0B547466F
:106AF000CE4680B58DB004000D0000F067FA294B3A
:106B000006001B780F005BB29846013310D02200BC
:106B10002B002000290003F0C1FA8146002807D18C
:106B2000002200232000290001F00AFC002806D1E1
:106B3000300039000DB00CBC90469946F0BD0123E1
:106B40000293194B0694079503934B460A934346C9
:106B500004940595002B15D0002300221900100085
:106B600002F0D8F8434608900991022B0ED103F0A9
:106B7000AFFB212303600A9B0193002B0CD1089EDD
:106B8000099FD5E7002300240893099402A801F087
:106B9000C1F90028EFD1EAE703F09AFB0A9B0193C1
:106BA0000360ECE764000020B0CB0000F0B54E4677
:106BB0004546DE465746E0B5E14B4C008FB0904667
:106BC000894664089C4200DC87E0DE4B9C4222DC64
:106BD000DD4A002900DC92E0DC4B02F017FFDB4BC2
:106BE00006000F009C4200D17EE1D94AD94B02F049
:106BF0000DFF02000B00414630000A604B60390077
:106C000002F004FFD34BD24A02F000FF43460125B5
:106C10009860D9606BE0D04B9C4200DC8FE0CF4B9A
:106C20009C4200DD55E1CE4A231592469A445146D6
:106C30000905631A19001D00040003F04BFA03F064
:106C40007FFA02000B00200029000892099302F04D
:106C5000DDFE0022C34B02F067FC0F00060003F0CC
:106C600039FA03F06DFA04000D0002000B00300049
:106C700039000A940B9502F0C9FE0022B94B02F0CC
:106C800053FC002200230C900D9101F053FB0028CF
:106C900000D192E1002300222000290001F04AFBEC
:106CA000434243410133B04A41460192022208A8BF
:106CB0000092524600F07CFB4B460500002B16DA92
:106CC000802243461206944642465B68454263442E
:106CD0005360D3686344D36009E00B00020041466F
:106CE0000A604B600022002300258A60CB602800E8
:106CF0000FB03CBC90469946A246AB46F0BD934BC4
:106D000001F0ECFC914B06000F009C4200D13DE1EC
:106D10008F4A904B01F0E2FC02000B00414630002C
:106D20000A604B60390002F071FE894A894B01F01C
:106D3000D5FC012543466D429860D960D7E701F044
:106D400049F88A4A8A4B06000F0002F0EDFB002248
:106D5000884B01F0C3FC03F0BDF9050003F0F0F926
:106D6000794A7A4B0490059102F0DEFB02000B0099
:106D70003000390002F04AFE754A06000F00049800
:106D80000599744B02F0D0FB029003911F2D00DC9B
:106D9000C7E0029A039B3000390002F037FE8346B9
:106DA0008A4653465B0024155B0DE31A102B6CDDFD
:106DB00004980599D322674B520502F0B5FB0200F7
:106DC0000B00300039000292039302F01FFE0A000C
:106DD000010013000691079202003900300002F012
:106DE00015FE029A039B02F011FE06000F000498A4
:106DF0000599614A614B02F097FB32003B0002F0BB
:106E000005FE069E079F0B0002003900300002922B
:106E1000039302F0FBFD4B005B0D83468A46E41AA8
:106E2000312C32DD04980599B822544B920502F0BA
:106E30007BFB03000C000200029303940B000698F6
:106E4000079902F0E3FD02000B0006000F00069810
:106E5000079902F0DBFD029A039B02F0D7FD484A36
:106E60000290039104980599464B02F05DFB029A4B
:106E7000039B02F0CBFD02000B00300039000292B0
:106E8000039302F0C3FD83468A465A465346414661
:106E900030000A604B60390002F0B8FD029A039B93
:106EA00002F0B4FD44460B000200A260E3604B46D2
:106EB000002B00DB1BE75B46236080231B0653444B
:106EC000636080231B069C466144A060E1606D42C4
:106ED0000DE70B00020002F099FD43460025986083
:106EE000D9601860596002E7D3221A4B520502F0AC
:106EF0008DFD214A214B0D00040002F087FD0200A8
:106F00000B00414620000A604B60290002F07EFD24
:106F10001A4B194A02F07AFD434601259860D96060
:106F2000E5E602000B003000390002F06FFD6B1E39
:106F3000154A9B009B5883468A46A342A5D130E759
:106F4000FB21E93F7BD9024000004054FB21F93F7F
:106F50003163621A61B4D03DFB213941FFFFEF7FFD
:106F6000EAFBFFFF0000704138CC000083C8C96D08
:106F7000305FE43F0000E03F7370032E8A19A33BAB
:106F8000C14920259A837B39B8CB0000D3220C4B12
:106F9000520501F0A3FB0B4A0B4B04000D0001F05E
:106FA0009DFB02000B00414620000A604B60290057
:106FB00002F02CFD034A044BB9E6032373E6C046F6
:106FC00061B4D03D7370032E8A19A33BF8B54746D0
:106FD000CE46674B80B50A000F0019000500394006
:106FE000994200D19BE004000100002F69DD3F15AC
:106FF00000D1B4E05F4B12039C468023120B5B036D
:1070000013435B00CA0F67449B184A00F80703D577
:10701000D20F5B009B188A0079108C4600218020DB
:107020001624894680030D189D4202DC29185B1B3B
:107030008144D50F5B00013C5B1952004008002CD5
:10704000F1D100208046802020250027000609E09D
:107050008B425CD0D40F5B00013DE3185200400826
:10706000002D16D0C4198B42F2DD27180E00002C1B
:1070700049DB5B1AA242894149425B1A121BD40FB9
:107080005B00013D80443100E31852004008002DB0
:10709000E8D113434ED143465B0837494A468846F8
:1070A000494652104244C90702D5802109060B43C4
:1070B00061460F05BD18180029000CBC9046994682
:1070C000F8BD7B005B0803433900002BF5D0002F8F
:1070D0003CD1E30A153A6405002BFAD08020400326
:1070E00003423FD1002700E00F005B00791C034200
:1070F000FAD0250020208D40401A2900D71B2200FD
:10710000C2401A4376E7FE43F60F8E19B1E7944268
:10711000A0D82718002CF6DB1E000023AEE70200E3
:107120003B002800390002F0FFF92A003B0001F083
:10713000D5FAC2E74346013303D0434601335B0827
:10714000ABE7012398460023C144A6E73B000200B9
:1071500002F05CFC02000B0001F0DCFDADE7130067
:107160000022BBE70127210020207F42C6E7C0465E
:107170000000F07F01FCFFFF0000E03FF0B5474654
:10718000CE4680B587B000920193754B4F00814683
:1071900088467F089F4263DC02F09CFF002800D1F4
:1071A000D4E04A4643464846414602F0BDF9040051
:1071B0000D006C4A6C4B02F0B7F96C4A6C4B01F055
:1071C0008DFA22002B0002F0AFF96A4A6A4B02F0F6
:1071D0001DFC22002B0002F0A7F9684A684B01F061
:1071E0007DFA22002B0002F09FF9664A664B02F0FE
:1071F0000DFC22002B0002F097F9644A644B01F069
:107200006DFA22002B0002F08FF902900391002208
:10721000604B2000290002F087F9029A039B0600C8
:107220000F002000290002F07FF9009A019B040062
:107230000D004846414602F077F902000B0020009D
:10724000290002F0E3FB02000B003000390002F0DD
:10725000DDFB02000B0000204F4902F0D7FB70E07D
:1072600002000B0002F060F904000D003D4A3E4BA5
:1072700002F05AF93D4A3E4B01F030FA22002B0051
:1072800002F052F93B4A3C4B02F0C0FB22002B00BB
:1072900002F04AF9394A3A4B01F020FA22002B0059
:1072A00002F042F9374A384B02F0B0FB22002B00C3
:1072B00002F03AF9354A364B01F010FA2B00220061
:1072C00002F032F9354B029003919F429FDD344B1F
:1072D00000229F423DDC334900207B182E491600D6
:1072E0001F0002F093FB049005910022294B20001F
:1072F000290002F019F932003B0002F087FB029AE4
:10730000039B06000F002000290002F00DF9009AEF
:10731000019B04000D004846414602F005F90200B9
:107320000B002000290002F071FB02000B0030006E
:10733000390002F06BFB02000B000498059902F083
:1073400065FB07B00CBC90469946F0BD0020124981
:10735000F7E7154B002604920593144FC5E7C04686
:10736000FFFF3F3ED43888BEE9FAA8BDC4B1B4BD22
:107370009EEE213EAD529C804F7E923E9015CB19E1
:10738000A001FA3E7751C1166CC1563F4C55555578
:107390005555A53F0000E03F0000F03F3233D33F9A
:1073A0000000E93F0000E0FF0000E73F0000D23F9F
:1073B000F0B5DE464E4645465746E0B5DC4CA544A2
:1073C0000D9114001900A49A0993DA4B9200D65833
:1073D0004D1E03901821E01E0696029500F0A0FEB7
:1073E000C3430100DB1719404B1C9A009B1ADB00BA
:1073F0001B190B9105934C1B771918D4A59BA5005D
:107400009C463F1922AE6544013707E0286802F028
:1074100097FE013403C60435BC4208D0002CF5DACF
:1074200000200021013403C60435BC42F6D1069B7E
:10743000002B01DA00F0FDFB069B03990133DB0012
:107440009A46099BDA00944600920022914672AA5D
:107450000492B94A6144934688469AAB63449B447C
:10746000029B002B00DABCE15D4600260027039C4E
:107470004D442A686B6803CC02F056F802000B00FA
:107480003000390001F02AF9083D06000F0044459C
:10749000EFD1049B4B441E605F6008239C46E1448F
:1074A000D145DDD10EA804218446494261448C4671
:1074B000069A93009C44614684460A910399083BCE
:1074C00063448C460C93009B009263449B46009A55
:1074D0000498D10003008C46634408911E685F68DD
:1074E000002A33DD954980468C466244D300984497
:1074F00070AB9A460EAB99460022914B3000390092
:1075000002F012F802F0E6FD02F01AFE00228D4BA6
:1075100004000D0002F008F802000B0030003900F2
:1075200002F074FA02F0D6FD4B4601C39946434679
:1075300020001A685B68290001F0D0F808235B423C
:107540009C46E04406000F00D045D5D1059B300095
:107550001A003900984600F0DFFCFF2300229B054B
:1075600004000D0001F0E0FF00F038FC0022764B33
:1075700001F0DAFF02000B002000290002F046FAB9
:107580000D00040002F0A6FD814602F0D9FD0200C4
:107590000B002000290002F039FA060040460F00D7
:1075A000002800DCEEE0009B18215A1E92000EAB72
:1075B0009B58091A1D000D41A9448D405D1B0EAB5F
:1075C0009D5017231B1A1D41002D2DDD01239C46C4
:1075D000009BE144002B00DC1CE20E9C0123002CEC
:1075E00000D0B5E0009A012A09D099000EAA54589B
:1075F0000133002C00D0ACE0009A9A42F5D1059BF3
:10760000002B0EDD012B00D1A8E1022B09D1009B3C
:107610000EA95A1E92000EAB9B5807939B029B0A21
:107620008B50022D00D1C1E0002300223000390030
:1076300000F080FE009B002800D194E2069A591EBB
:107640008A4210DC414A0A9894460EAA6344944642
:1076500000229B0063441C68043B22438342FAD10E
:10766000002A00D0C0E0069B0EAA013B9B00D35825
:10767000002B00D0B3E001220C9B043B596801327F
:107680000029FAD0009B9C466244110007921A0020
:1076900001338B4246DC0B9863468046A59C4344ED
:1076A000A046099C9B00A1464A449844D30022AAC4
:1076B0009146049A99449446089BA59A634484464B
:1076C000614494469A468B0063440093434658684D
:1076D00002F036FD4B4618605960029B002B24DBFC
:1076E0004D46039C0026002701E0286869680CCC01
:1076F00001F01AFF02000B003000390000F0EEFF2D
:10770000083D06000F005C45EFD153469E60DF60E8
:1077100004239C460433E0449C46009BE144E2443D
:107720009845D3D1079B0093D1E600260027ECE7CC
:1077300094FDFFFF80CD000018FEFFFFFFFFFF1F3D
:107740000000703E0000704100002040FFFFFF3F3E
:10775000002180225204141B0EAA54500099994211
:107760000EDD0EA884469B000EAA8900D258614403
:107770006344CF4800E01A68821A04C38B42FAD1EE
:1077800001243CE7059B002B06D1009B0EAA013B80
:107790009B00D558ED1517E70022C64B300000F0CE
:1077A000EDFD002800D024E100253DE732003B003C
:1077B0000020C14902F02AF906000F00002C00D178
:1077C00032E7059A0020BC4900F0A6FB02000B003E
:1077D0003000390002F01AF906000F0024E70122F8
:1077E00050E70026002754E64B46059A0793884643
:1077F0008B000EA9CB58183A08950592002B0DD195
:107800008C464146AD4B43449B006344043B58685F
:107810000139183A0028F9D088460592059A0020C7
:10782000A54900F079FB434604000D00002B00DA67
:1078300005E29E000EAB9C464346DB0066449C4638
:10784000059370AB9946049F67440097306802F037
:1078500077FC22002B0001F067FE0022386079607F
:10786000974B2000290001F05FFE083F04000D0047
:10787000043EB945EAD14AAB03939B4600239A469E
:10788000069B4246994643460132029204934B4678
:10789000002B00DAAAE080208A4B009D9846C005A4
:1078A000894900260027002408E008239C46083563
:1078B000E044544511DC4346186859682A686B68EF
:1078C00001F032FE02000B003000390000F006FF2C
:1078D000013406000F00A145E7DA5B46C0C39B46B2
:1078E00001239C46009BE244083B0093029B9A457F
:1078F000CDD1049B9846A49B022B00DD8EE0002B8B
:1079000037DC1FD1059B00271D00039B00249C46EC
:107910001E006544083E2A686B683800210000F0AC
:10792000DDFE083D07000C00AE42F4D1089B002BA1
:1079300003D080231B069C4664443A0023000D9923
:107940000A604B600720079B18409B239B009D44C7
:107950003CBC90469946A246AB46F0BD009B0EA9A2
:107960005A1E92000EAB9B5807935B025B0A8B502A
:1079700057E64346002B00DA70E100200021DB00CF
:107980004AAAD61848AF32687368083E00F0A6FECF
:10799000B742F8D1089B002B00D025E10B00020074
:1079A0004A984B990D9C2260636002F02FF8434681
:1079B00007000C00002B13DD01254CAEB14638004A
:1079C0002E0021004C4601360CCC00F087FEA1466B
:1079D000B045F7DA089B07000C00002B00D015E13A
:1079E0003A0023000D998A60CB60ABE700260027A0
:1079F00073E701239C46009BE1440225002B00DD38
:107A0000EBE532003B0000202B4901F0FFFF0600B0
:107A10000F0009E60024F2E54AAB0393A49B032B75
:107A200000D08FE74346002B00DC14E1039ADB0013
:107A30009B46130091465B441E685F68234B43449A
:107A40000293DB00994448AB9A464B465C681B683E
:107A50001800210032003B000090019100F03EFE32
:107A600004000D0002000B000098019901F0CEFF08
:107A70003B00320000F032FE4B469860D9601C603B
:107A80005D6008235B429C46E14426002F00CA4506
:107A9000DBD14346012B00DCE3E0039A13005B4497
:107AA0001E685F68029BDB0099464A44904610E0DE
:107AB000FFFFFF000000E03F0000F03FFFFFFF3F3F
:107AC0000000703E40CD0000FB21F93FFFFFFF1F8B
:107AD000984643465C681B681800210032003B0052
:107AE0000090019100F0FAFD04000D0002000B006F
:107AF0000098019901F08AFF32003B0000F0EEFD92
:107B00004346039A9860D9601C605D60083B26007C
:107B10002F009A42DCD14D46944600260024474669
:107B2000083565442A686B683000210000F0D6FDF6
:107B3000083D06000C00AF42F4D1039B4A9F5D68EC
:107B40009968D868089B002B65D08022120694465D
:107B50000D9B6544604464441F605D609960D8601B
:107B60001E615C61EEE69A464B460793059B30002A
:107B70005A423900089500F0CFF900223A4B06002E
:107B80000F0000F0FBFB002824D0384B002230000F
:107B9000390001F0C9FC02F09DFA5246040095003C
:107BA00002F0CEFA0022304B01F0BEFC02000B00C6
:107BB0003000390001F02AFF02F08CFA0EAA505171
:107BC0000122059B524418339046059393000EAA58
:107BD000D45023E65346300039009C0002F07AFA74
:107BE0000EAB1851D04619E680230D9A1B06CB1810
:107BF000106053600B0002004A984B9901F006FF99
:107C0000434607000C00002B00DDD5E680231B0651
:107C10009C466444E4E62B003A000D9D2A606B60AC
:107C20000A000300AA60EB60320023002A616B6146
:107C300088E6099BDB00009372AB049332E4A49BBB
:107C4000022B00DDE8E6002B00DD92E600D079E6AD
:107C5000002700246AE6002600246EE700200021A9
:107C600098E60026340068E7000070410000703E8E
:107C7000F0B5CE46474680B587B000920193474A9B
:107C80004B00814688465B08934207DC41464846E4
:107C900002F020FA4146031E484666D04A46434653
:107CA0004846414601F040FC04000D0002000B0074
:107CB0004846414601F038FC394A3A4B06000F006D
:107CC0002000290001F030FC374A384B01F09EFEBD
:107CD00022002B0001F028FC354A364B00F0FEFC58
:107CE00022002B0001F020FC334A344B01F08EFEC1
:107CF00022002B0001F018FC314B324A00F0EEFC60
:107D00000E9B02900391002B34D000980199002221
:107D10002D4B01F009FC029A039B04900591300061
:107D2000390001F001FC02000B000498059901F0F4
:107D30006DFE22002B0001F0F7FB009A019B01F081
:107D400065FE224A04000D00214B3000390001F08D
:107D5000EBFB02000B002000290000F0BFFC02003A
:107D60000B004846414601F051FE07B00CBC90465E
:107D70009946F0BD02000B002000290001F0D4FB61
:107D8000124A134B01F042FE32003B0001F0CCFBE3
:107D90004A46434600F0A2FCE7E7C046FFFF3F3EED
:107DA0007CD5CF5A3AD9E53DEB9C2B8AE6E55A3E85
:107DB0007DFEB157E31DC73ED561C119A0012A3F21
:107DC0001111813FA6F810110000E03F49555555AB
:107DD0005555C53F49004B0819007047474AF0B553
:107DE0004F4691464B005B0D99444646D6464A465F
:107DF000C0B505000C000E0088460700132A27DCDA
:107E0000002A4BDB3E4B13419A460B00524613406F
:107E1000034318D03B4A3C4B2800210000F05EFC95
:107E20000022002300F0A0FA002847D0002C04DA3A
:107E300080234A465B031341984446465346002735
:107E40009E43380031001CBC90469946A246F0BDC6
:107E5000332A08DD8023DB009945F4D102000B00B2
:107E600000F03CFCEFE7294A944601226344524269
:107E7000DA4092460242E6D0224A234B28002100F3
:107E800000F02CFC0022002300F06EFA002815D030
:107E9000002C1EDB534646469F430FE0194A1A4BFF
:107EA0002800210000F01AFC0022002300F05CFAF8
:107EB000002803D0002C04DB002700263800310006
:107EC000C1E76400640825430027002DF6D0104E5A
:107ED000F4E74B46142B0BD03422D21A01239340E3
:107EE0005D19BD4208D201239C462F00E044D1E732
:107EF000133B9C46E044CDE72F00CBE701FCFFFF9E
:107F0000FFFF0F009C7500883CE4377EEDFBFFFF10
:107F10000000F0BF002070474B0070B55B0D1400EF
:107F20000A00002B1AD14B005B08034315D0234BEA
:107F3000002201F0F9FA224B9C422DDB0A004B0093
:107F40005B0D363B1F4DE318AB422ADC002B0DDDE9
:107F50001D4C1B0522401A43110070BD1B4DAB4246
:107F6000F0D102000B0000F0B9FBF6E71D0035353B
:107F700019DA174B02009C4209DD0B00154816491F
:107F800000F032F8134A144B01F0CEFAE5E70B008B
:107F90001248134900F028F8104A114B01F0C4FAB6
:107FA000DBE70200E9E7084C363322401B051343A8
:107FB000190000220B4B01F0B7FACEE70000504346
:107FC000B03CFFFFFE070000FFFF0F80FF0700002F
:107FD00050C300009C7500883CE4377E59F3F8C21A
:107FE0001F6EA5010000903C30B54A00DB0FDB0797
:107FF00052081A43110030BD02B4714649084900C5
:10800000095C49008E4402BC7047C0460022430808
:108010008B4274D303098B425FD3030A8B4244D350
:10802000030B8B4228D3030C8B420DD3FF22090292
:1080300012BA030C8B4202D31212090265D0030B51
:108040008B4219D300E0090AC30B8B4201D3CB0347
:10805000C01A5241830B8B4201D38B03C01A524189
:10806000430B8B4201D34B03C01A5241030B8B428B
:1080700001D30B03C01A5241C30A8B4201D3CB0276
:10808000C01A5241830A8B4201D38B02C01A52415B
:10809000430A8B4201D34B02C01A5241030A8B425E
:1080A00001D30B02C01A5241CDD2C3098B4201D376
:1080B000CB01C01A524183098B4201D38B01C01AF4
:1080C000524143098B4201D34B01C01A524103096B
:1080D0008B4201D30B01C01A5241C3088B4201D31A
:1080E000CB00C01A524183088B4201D38B00C01AC7
:1080F000524143088B4201D34B00C01A5241411AEE
:1081000000D20146524110467047FFE701B50020FA
:1081100000F0F0F802BDC0460029F7D076E77047BE
:1081200003460B437FD4002243088B4274D30309D8
:108130008B425FD3030A8B4244D3030B8B4228D379
:10814000030C8B420DD3FF22090212BA030C8B429F
:1081500002D31212090265D0030B8B4219D300E03F
:10816000090AC30B8B4201D3CB03C01A5241830BC4
:108170008B4201D38B03C01A5241430B8B4201D374
:108180004B03C01A5241030B8B4201D30B03C01A9D
:108190005241C30A8B4201D3CB02C01A5241830A17
:1081A0008B4201D38B02C01A5241430A8B4201D346
:1081B0004B02C01A5241030A8B4201D30B02C01A70
:1081C0005241CDD2C3098B4201D3CB01C01A5241D7
:1081D00083098B4201D38B01C01A524143098B4260
:1081E00001D34B01C01A524103098B4201D30B0149
:1081F000C01A5241C3088B4201D3CB00C01A52416E
:1082000083088B4201D38B00C01A524143088B4232
:1082100001D34B00C01A5241411A00D201465241CB
:10822000104670475DE0CA0F00D04942031000D3EA
:108230004042534000229C4603098B422DD3030A3F
:108240008B4212D3FC22890112BA030A8B420CD34F
:10825000890192118B4208D3890192118B4204D378
:1082600089013AD0921100E08909C3098B4201D3F8
:10827000CB01C01A524183098B4201D38B01C01A32
:10828000524143098B4201D34B01C01A52410309A9
:108290008B4201D30B01C01A5241C3088B4201D358
:1082A000CB00C01A524183088B4201D38B00C01A05
:1082B0005241D9D243088B4201D34B00C01A5241DC
:1082C000411A00D20146634652415B10104601D369
:1082D0004042002B00D54942704763465B1000D3F3
:1082E000404201B5002000F005F802BD0029F8D099
:1082F00016E770477047C046D0400B1C1141203A2A
:1083000003D49C461341184363465242934018439A
:108310007047C0468446101C62468C46191C634652
:1083200000E0C0461FB501F097F8002801D40021F5
:10833000C8421FBD10B500F0EFFF4042013010BD34
:1083400010B501F089F8002801DB002010BD0120E4
:1083500010BDC04610B501F07FF8002801DD0020F7
:1083600010BD012010BDC04610B501F011F8002865
:1083700001DC002010BD012010BDC04610B501F089
:1083800007F8002801DA002010BD012010BDC0460A
:10839000F0B5CE46474615042D0C2E0080B50704D7
:1083A000140C3F0C9946030C7E435D4367436343C3
:1083B0007F19340CE4199C46A54203D980235B0243
:1083C0009846C4444B4643435143250C3604654408
:1083D000360C2404A4195B19591820000CBC9046D3
:1083E0009946F0BDF0B54E4657464546DE46E0B5E7
:1083F00043025B0A450083B00F1C99462D0EC60F41
:10840000002D57D0FF2D24D08020DB00C00418435E
:10841000002381469A469B467F3D7C027A00FB0FF3
:10842000640A120E984623D0FF2A4BD0E300802422
:108430000020E4047F3A1C43AD186B1C47460193AF
:10844000534677403A000F2B48D87D499B00CB58C4
:108450009F46002B00D085E008339A46063B9B469A
:108460007C027A00FB0FFF25640A120E9846DBD1CE
:10847000002C00D090E0524601231A43924601207E
:10848000DBE74C4658461700022824D0032800D1C9
:10849000CFE00022002301284DD15802D205400A26
:1084A000FF071043384303B03CBC90469946A246B0
:1084B000AB46F0BD002B5BD104239A46033B00255D
:1084C0009B46AAE7FF35002C60D1524602231A438F
:1084D00092460220B1E7FF220023DEE74B461B0C49
:1084E0009C464B462604360C180461463300220C89
:1084F0006446000C43434E435043544380191A0CC6
:108500001218964203D9802149028C4664441B0408
:108510001B0C1004C01883015E1EB341800E18436B
:10852000130C1B199B0103431C00230179D5012364
:1085300062081C401443019A7F32002A4DDD630714
:1085400004D00F232340042B00D00434230103D58F
:108550003C4B019A1C408032FE2ABCDCA3015B0A22
:10856000D2B29AE70C239A46093BFF259B4654E773
:10857000180001F071FE4A46431F76259A400023F9
:108580006D4291462D1A9A469B4646E75246032372
:108590001A439246032050E7200001F05DFE431F7E
:1085A0002D1A9C40763D002047E780230027DB03FF
:1085B000FF2272E7424666E74C463200584662E7C1
:1085C00080234A46DB031A4222D01C4220D1234397
:1085D0005B025B0A4746FF225FE701239A1A1B2AC8
:1085E00021DC23000199D3409E318C401A002300E6
:1085F0005C1EA34113435A0704D00F221A40042AD9
:1086000000D004335A0111D49B015B0A002244E7D5
:1086100080234A46DB0313435B025B0A3700FF22D9
:108620003BE7019587E70022002336E7012200237C
:1086300033E78023DB0323435B025B0AFF222CE743
:1086400090CD0000FFFFFFF770B500283DD0C317A5
:10865000C5185D40C40F280001F0FEFD9E22121ACD
:10866000962A07DCD2B2082833DD08388540680234
:10867000400A23E0992A0BDD052329001B1AD94063
:1086800003001B339D402B005D1EAB4119430D00C1
:10869000052801DD431F9D402B000F490B406E074D
:1086A00009D00F263540042D05D004335D0102D5D5
:1086B0009F220B40121A9B01580AD2B24002D205E7
:1086C000400AE4071043204370BD0024002200202C
:1086D000F4E76802400AF1E7FFFFFFFBF0B54F4601
:1086E0004646D6460C000903C0B5490A470F5E004E
:1086F00039431F03DB0F9C4665007B0A570F1F435E
:108700006D0DE40F760DA146C000B846D200AB1B3C
:1087100064457BD0002B5FDD002E00D0A4E03E003E
:10872000164300D112E15E1E002E00D09EE1871A92
:108730004346B84280410125C91A4042091A0B023A
:1087400000D431E149024E0A002E00D16EE1300022
:1087500001F082FD0300083B1F2B00DD61E12022B8
:108760003900D21A9E40D1409F400E439D4200DD09
:1087700051E15D1B6B1C1F2B00DD7CE12021C91A20
:108780003D0030008F408840DD40791E8F41310030
:1087900007222843D940002507433A40002A09D040
:1087A0000F233B40042B05D03B1DBB42BF417F4202
:1087B000C9191F000B0200D426E26A1CC64B5505DE
:1087C0006D0D9A4200D106E1C44AFF080A405307E2
:1087D00052023B43120B8EE0002B00D0B8E06B1C22
:1087E0005B055B0D012B00DC30E1871A4346B84284
:1087F000B641CB1A76429E1B330200D54CE13B00BA
:108800003343A1D100220024002570E0002B00DCBE
:10881000E5E0002E00D183E0AF4EB54260D0802667
:1088200036043743B846382B00DC3EE14346134359
:108830001F007A1E97413F18874280414042091825
:108840000B0200D4B0E0A44B01359D4200D1C3E03F
:10885000A24A7B080A4001210F401F435108D30759
:1088600007221F433A4099E79B4EB54238D08026F5
:1088700036043743B846382B00DDDCE01F2B00DC24
:1088800030E11E004746203EF740BC46202B04D076
:108890004026F31A46469E403243170063467A1E2E
:1088A00097411F43CCE0002B00D104E24346134321
:1088B00000D159E14B07C00818438023C9081B03A6
:1088C000194208D04546ED081D4204D14346D00860
:1088D000590708432900420FC9007F4D1143C000CA
:1088E0004B07CA087C49C00803438D4268D0120375
:1088F0006D05120B6D0D002112031800130B0A0DEC
:1089000012051A43764B2D0513402B435B00E407F9
:108910005B08234319001CBC90469946A246F0BD53
:108920003E00164312D05E1E002E00D000E18718D4
:108930008742804141444042091801250B0233D54A
:10894000022585E764463300414610001D00C7E755
:10895000002D00D0DAE00C000443F3D05C1C00D101
:108960009FE15D4CA64200D12FE1DB43382B00DDB7
:1089700066E11F2B00DD83E120240500E41A0F00CF
:10898000DD40D940A0404346A7405B1A441EA041A9
:1089900098462F433843171ABA42924143465242EF
:1089A000991A64463500CAE607223A40002A00D0E8
:1089B000F6E64B07CA084849FF083B438D4296D16B
:1089C0001900114300D19EE1802109030A431203DB
:1089D000120B414D8FE71500002200238BE7002B7F
:1089E00000D0C7E06B1C5F057F0D012F00DCF1E0BC
:1089F000394DAB4200D1B9E085180A008542894162
:108A00004244494251180722CF076D082F434908B5
:108A10003A401D00C2E607223049ED1A31403A4083
:108A2000BCE63E002838864000279FE6380001F06B
:108A300013FC20308EE6434613431F007A1E9741F5
:108A4000C71BB84280414042091A78E60E003B003D
:108A500006431343002D61D1002E00D0F4E0002B1B
:108A600000D11BE164463900100039E71A4FBB42C0
:108A70007AD03300FFE630001F3DE840202B03D0C2
:108A80004021CB1A9E4037437B1E9F41072207435C
:108A90003A400021002589E7171A4346BA42B641F9
:108AA000591A76428E1B64464EE61F2B00DDADE060
:108AB00020264746F61AB740B9461700B246DF40AF
:108AC0004E463E4337005646B240561EB24117430B
:108AD0004246DA408918AEE6FF070000FFFF7FFF3D
:108AE000FFFF0F8020264746F61AB740B946170009
:108AF000B246DF404E463E4337005646B240561E11
:108B0000B24117434246DA40891A99E77F4CA642A0
:108B10005BD0802424045B42214327E7002E0CD144
:108B2000002B00D1CBE0644639001000774DD7E62A
:108B3000764FBB4218D0330075E6002B14D04B079C
:108B4000C00818438023C9081B03194207D0FC083A
:108B50001C4204D17907D0080843E14621004C4665
:108B6000420FC9001143C000684DB9E61D00002244
:108B70000023C0E6002D5BD10D00054300D1E2E6E5
:108B80005D1C00D1B0E0614DAE421FD0DB43382BFD
:108B900071DC1F2B00DD96E020250F00ED1AAF40A1
:108BA000B9460700AA46DF404D463D432F005546D3
:108BB000A840D940451EA84188440743BF189742A2
:108BC00092415142414435003AE6644635004146FF
:108BD000100085E60B000343002D00D063E6002B58
:108BE000F5D04346134300D17AE687188742804187
:108BF00007224144404209183A400B0200D4D5E60E
:108C0000434B01351940C9E5380069E61E00474667
:108C1000203EF740BC46202B04D04026F31A46469F
:108C20009E403243170063467A1E97411F4302E677
:108C3000364DAE42CAD080252D045B422943A6E7BB
:108C40000843411E8841A6E6002B00D148E6871A5A
:108C50004346B842B641CB1A76429E1B33024BD5EF
:108C6000171A4346BA429241591A5242891A0722A8
:108C700064463A4092E501430F00791E8F419DE71B
:108C80001C000F00203CE740202B03D04024E31AB7
:108C900099400843411E884138437CE60022002465
:108CA00025E6171A4346BA429241591A5242891A86
:108CB0006446350043E541461000144D10E680221D
:108CC0000024120380E61D000F00203DEF40BC464B
:108CD000202B03D04025EB1A994008430700634638
:108CE000781E87411F4369E7871897429B4141449B
:108CF0005B42C9183500A3E53B003343CED00722C1
:108D000031003A4052E600231A00F4E5FF07000064
:108D1000FFFF7FFFF0B55746DE464E464546E0B5BD
:108D2000834607000E03480085B092461C00360BB0
:108D3000400DCD0F002800D19DE0954B984239D0D1
:108D40008023F6001B041E43924A7B0F334399464F
:108D5000944603006344009300230026FF0002931F
:108D600023031B0B98466300E40F52465B0D0194EE
:108D700000D1B3E086498B4200D19EE04246D1004B
:108D8000802212040A435146490F11438B46814900
:108D900052468C4600996344CB1A0021D2000093BE
:108DA0002B0063409A460F2E00D905E17A4BB6009E
:108DB0009B599F465B463343994600D0B8E0022357
:108DC0000826002700900293CAE7CB463A00029992
:108DD0000195019B9A46022927D0032900D180E200
:108DE000012944D06D49009B8C4663441C00002C33
:108DF00038DD530700D013E2D2085B46DB0109D50A
:108E00005946674B19408B468021C9008C46009B10
:108E100063441C00634B9C4207DC5B4664055F07B0
:108E20005B0217431B0B620D02E000230027584A28
:108E300000211B031C0B0B0D1B05234314055A4A71
:108E4000380013401C4353466400DB0764081C438E
:108E5000210005B03CBC90469946A246AB46F0BD09
:108E60000122524201231B1B382B00DCADE1002202
:108E700000230027DCE75B46334399465ED0002E93
:108E800000D18AE1300001F0E7F903000B3B1C2B15
:108E900000DD7BE11D22D31A5A460100DA40083971
:108EA0008E4013005F46334399468F403F4B002668
:108EB0001B1A00930023029352E7414653460B438B
:108EC0003B499B468C46009B634400935B46002BCA
:108ED0003BD1022300221E43022161E74346134394
:108EE0009B4637D04346002B00D162E1404601F05B
:108EF000B3F903000B3B1C2B00DD53E1020041469C
:108F0000083A914088461D21CB1A5146D9400B00A2
:108F100041460B439B46534693401A00009B25490C
:108F20009C46604403008C4663440093002137E76D
:108F30000323B14600900C26029311E7002300930F
:108F400001330426002702930AE70323C3461E4386
:108F5000032125E701331E430022012120E70023DE
:108F60009A46802300271B03094A61E7802349466C
:108F70001B03194200D1E2E05946194200D0DEE05D
:108F80000B431B0317001B0BA246014A50E7C046C8
:108F9000FF07000001FCFFFFD0CD0000FF03000031
:108FA000FFFFFFFEFE070000FFFF0F800DFCFFFF2D
:108FB00001F8FFFFF3030000D94500D9CBE000D151
:108FC000C6E03C0048460027009B013B00935B46FF
:108FD000160E1B021E431302984633041B0C9946BF
:108FE000310C0191FFF798F84A4642430B04210CDB
:108FF000050019438A4207D98919013D8E4203D8D9
:109000008A4201D9851E8919881A0199FFF784F8C7
:1090100009048C464A46210464464243090C030075
:1090200021438A4204D98919013B8E4200D8F1E0DC
:109030002D041D43AB464346891A4246280C1204B0
:109040001D0C5B46140C22001B041B0C5A4303949A
:109050006B434443029568431B19150CEB189C4263
:1090600003D980246402A44660441C0C15041B042C
:109070002D0C20185D19814277D373D00C1AA24AA7
:109080007D1BAF42BF419446009B7F426344E01B7F
:109090001C00864200D1DBE00199FFF73DF84A460B
:1090A00042430B04290C070019438A4207D9891946
:1090B000013F8E4203D88A4201D9871E8919881A36
:1090C0000199FFF729F809044A46894629044D46C3
:1090D0004243090C030029438A4207D98919013BFD
:1090E0008E4203D88A4201D9831E89193F04891A06
:1090F0003A00039F1A43380013041B0C584381465F
:109100000298150C6F43434345434846000C844680
:10911000DB1963449F4203D98020400284466544A2
:1091200048461F0C00041B04000C7D191818A942A6
:1091300000D284E000D17FE001231A4357E6802368
:109140004A461B0313431B031B0BAA466F4A6FE6D9
:10915000BA4200D935E74B46DC0758087B081C4368
:10916000FF0734E70024AF4289D247444745A44172
:109170005B466442A4196418013BA6421ED2A04279
:109180006DD800D1B6E0241A9B4678E703005A4612
:10919000283B9A400027914688E6584601F05CF843
:1091A000203072E603005246283B9A409346002244
:1091B000B4E6504601F050F820309AE6A642E2D1DB
:1091C000B845DCD9341A9B4659E71F2B65DC504C57
:1091D0000099A4465C46614408008C40110082401E
:1091E000D940501E82410C4314435A46DA401300C2
:1091F000620709D00F222240042A05D02200141D44
:109200009442894149425B181A0262D50122002327
:1092100000270DE68A4200D80AE7831E891907E76E
:109220000F231340042B00D1E6E5171D974292410E
:1092300053429B44FA08E0E5002800D1D7E57118B5
:10924000531EB14227D3A94215D358D01A0073E751
:10925000002B00DC04E6012300229B44CDE5022321
:109260004744474589415B429C46494289190C194C
:10927000E344241A03E743465F0047459B41B84651
:109280005B429E19023A8919A94200D054E7404531
:1092900000D051E7ABE51A00F6E71F215F464942CF
:1092A0000C1BE740202B07D01A49009B8C466344D7
:1092B00018005B4683401A43501E82413A430727F9
:1092C0000023174009D00F21002311401400042966
:1092D00095D122005F075B021B0BD20817430022C7
:1092E000A6E5802359461B030B431B0317001B0BEA
:1092F000064A9DE5BD42B2D89B460024BFE68045A4
:10930000B9D31A00C3E7C046FF030000FF070000FF
:109310001E0400003E040000F0B54F464646D64607
:109320008446C0B58046194E18030F034D00000B4C
:109330005C0082463F0B6D0DC90F9146640DDB0F3B
:109340000120B5420AD0B44203D0A54201D157450D
:109350000CD01CBC90469946A246F0BD66463E43E2
:10936000F7D1AC42F5D154461443F2D10120C8459F
:10937000EFD1994207D0002DEBD163461F4338004F
:10938000471EB841E5E70020E3E7C046FF070000BD
:10939000F0B54F464646D6464D00C0B50E03C90F40
:1093A0008A462C491F035C008046360B6D0D9146A2
:1093B0003F0B640DDB0F8D421ED08C4216D0002D6A
:1093C0001ED130438446002C01D13A4323D062465B
:1093D000002A1AD09A4529D0514602200139084066
:1093E00001381CBC90469946A246F0BD3900114395
:1093F000E5D002204042F4E73043FAD1AC420FD02E
:10940000002C0FD13A43E7D00CE00122013B9343FB
:1094100018000130E5E763460020002BE1D0DBE7D0
:109420003A43E6D19A45D7D1A542D5DCA54205DB22
:10943000BE42D1D808D00020BE42D2D2504601232D
:10944000013898430130CCE7C845C5D80020C8454D
:10945000F4D3C6E7FF070000F0B54F464646D646B0
:109460004D00C0B50E03C90F8A462E491F035C008C
:109470008046360B6D0D91463F0B640DDB0F8D4220
:1094800018D08C4211D0002D18D130438446002CC6
:109490001ED13A431CD163460020002B30D05146E8
:1094A00002200139084001382AE039001143EAD08E
:1094B000022025E03043FBD1AC4226D0002C26D13F
:1094C0003A4324D15146022001390840013817E0BF
:1094D0006246002A0FD09A45E1D1A54205DBBE4283
:1094E000DDD819D00020BE420AD2504601230138EF
:1094F0009843013004E00122013B934318000130FE
:109500001CBC90469946A246F0BD3A43D0D19A453C
:10951000C5D1A542C3DCE0E7C845C0D80020C84596
:10952000E3D3EDE7FF070000F0B55746DE464E46B1
:109530004546E0B5834606000F03480087B09246D3
:109540001D003F0B400DCC0F002800D16FE0DE4B1B
:10955000984238D08023FF001B041F43730F3B4306
:109560000193DA4B0027994600239B46F60081447D
:109570002B0369001B0B52469846490DED0F00293D
:1095800000D185E0D04B994200D173E04346DA0028
:1095900080231B0413435246CC48520F8446134386
:1095A000524600206144D200894421006940009164
:1095B0008C46012149448A460F2F00D990E0C449C6
:1095C000BF00CF59BF465B463B43019300D06AE1E1
:1095D00002230827002681469B46C9E732005846E9
:1095E000019B61460091022800D175E0032800D15B
:1095F000FEE1012800D02CE10023002700260025F1
:109600003F032A0D3F0BB34812053A4302401B05A6
:109610001343009A5B00D1075B080B43300019002D
:1096200007B03CBC90469946A246AB46F0BD5B46AF
:109630003B43019300D12FE1002F00D1A5E1380079
:1096400000F00AFE03000B3B1C2B00DD96E11D22FF
:10965000D31A5A460100DA405E4608398F4013009B
:109660008E403B4301939C4B00271B1A99460023D5
:109670009B467DE7414653460B4393498C46E14464
:10968000002B00D01AE102220220174300228CE7AF
:10969000134300D10DE14346002B00D181E1404648
:1096A00000F0DAFD02000B3A1C2A00DD72E1010035
:1096B000434608398B4098461D239A1A5346D34097
:1096C0001A004346134352468A404946081A8249C3
:1096D00089468144002068E77B4B002700268EE7FF
:1096E000140C1204120C1100370C3604350C79439B
:1096F00028008C462E006043604483465643210078
:10970000300C80465846794340440291844506D93E
:109710008846802149028C46E04441460291360445
:10972000010C360C00048B4681191E0C1B041B0C0B
:109730000391190079438C46280075436544A84677
:109740005843050C45447743A94203D98021490277
:109750008C466744290C8C4639000004000C2D040B
:109760002D186144AB4405915946049101990F04A9
:109770003F0C080C390051434243904602008C468E
:10978000090C8B4662437C4344445C44A04503D9A6
:109790008021490288464244210C884661460904DA
:1097A000090C8C4639005943434370437E430F0CE8
:1097B000F6182404BE19644442448C46B34203D9CB
:1097C00080235B0298464044029B61469846049B76
:1097D000370443449B46AB45AD416B420D040599AC
:1097E0002D0C8C467F196744FD18A8465D462D193F
:1097F000A542A44193466442A446C344DC448F423C
:10980000BF4198459B4193459241A445A4415B4289
:109810007F421F43360C52426442BF192243BF1895
:10982000624638184302D20D039913436A020A4371
:10983000501E82416146ED0D2A434E023243D9014A
:1098400000D4B3E00126500832400243DE07324321
:109850005B08224C5444002C62DD510709D00F20D4
:109860001040042805D0101D9042924152429B188E
:109870000200D90104D580241948E400034054446F
:109880001848844200DD27E75E075B02D2081F0B01
:10989000630516435B0DB2E60023994601330427A6
:1098A00000269B4664E60323019781460C279B46CE
:1098B0005EE6012201201743002276E603230320FF
:1098C0001F43434671E6C046FF07000001FCFFFF4F
:1098D00010CE0000FFFF0F800DFCFFFFFF03000014
:1098E000FFFFFFFEFE0700000023802700933F03D9
:1098F0000026434B83E6019B3200A446584670E69F
:10990000AC466EE6802701993F0339422DD03B4299
:109910002BD11F433F033F0B00951600384B6EE6DB
:1099200001252D1B382D00DD66E61F2D40DC354856
:109930001C005044160082408440EE40501E82417C
:1099400034431443EB40620709D00F222240042A1B
:1099500005D02200141D9442804140421B181A0277
:109960003ED501230027002649E68027019B3F03BF
:109970001F433F033F0B0094214B40E603005A4630
:10998000283B9A40002601926DE6584600F064FCA0
:10999000203057E603005246283B9A40130000222D
:1099A00093E6504600F058FC20307BE6CA4650E76C
:1099B0001F201E004042041BE640202D03D0124C05
:1099C0005444A3401A43501E8241324307260027C5
:1099D000164009D00F200023104014000428B9D1EC
:1099E00022005E075B021F0BD2081643002306E627
:1099F00080273F031F433F033F0B1600004BFEE54C
:109A0000FF0700001E0400003E040000F8B55746A2
:109A10004E464546DE460C000903E0B5490A460FAE
:109A20005F0031431E03DB0F760A9B46530F33431F
:109A3000C84E6500C000E40FD2006D0DA2468146FD
:109A40007F0D9C469046B74200D1B9E05B460126A7
:109A500073409B46EE1BA34500D183E0002E63DDDF
:109A6000002F00D0B1E06346134300D123E1731E01
:109A7000002B00D0BAE1861A6346B042804101252E
:109A8000C91A4042091A0B0200D447E149024B0AA5
:109A900098464346002B00D189E1404600F0DCFBAC
:109AA0000300083B1F2B00DD7CE120223000D21A8E
:109AB0004146D040994002009E400A439D4200DD4D
:109AC0006AE15D1B6B1C1F2B00DD94E1202110005F
:109AD0003500C91A8E40DA408840DD40711E8E4143
:109AE000110007222843002506433240002A09D0EE
:109AF0000F233340042B05D0331DB342B6417642C9
:109B000089191E000B0200D43DE26A1C914B5505D9
:109B10006D0D9A4200D119E18F4AF6080A405707A5
:109B200052023743120B9BE0002E00D0C5E06E1CA2
:109B30007605760D012E00DC48E16746861ACB1BC0
:109B4000B042BF417F42B8461F004346FF1A3B0068
:109B5000B8461B0200D55FE137439AD100220024AA
:109B6000002579E0002E00DCFAE0002F00D18DE026
:109B7000784B9D4267D0802367461B041F43BC4639
:109B8000382E00DC52E1634613435A1E93411E18DF
:109B900086428041404209180B0200D4BEE06D4B62
:109BA00001359D4200D1D2E06B4A73080A40012181
:109BB0000E401E435108D30707221E43324095E74B
:109BC0001E00164300D045E740E7624B9D423AD065
:109BD000802367461B041F43BC46382E00DDEBE0A4
:109BE0001F2E00DC3AE133006746203BDF403B009C
:109BF000202E05D04027BF1B6646BE40324390460C
:109C00004646721E96413343DAE0002B00D114E23F
:109C10006346134300D168E180234E07C008C9089A
:109C20001B030643194208D06046C008184204D1FD
:109C300063460100D2085E071643F3009946C90047
:109C4000720F444D11434B46DE08424B4F073743DA
:109C5000CA089D4200D16EE012036D05120B6D0D16
:109C600000211203130B0A0D12051A433B4B2D055D
:109C700013402B435B00E4075B08234338001900C3
:109C80003CBC90469946A246AB46F8BD634613439A
:109C900011D0731E002B00D007E186188642804148
:109CA00061444042091801250B0237D502257BE7A4
:109CB0003E00614691463500C5E75C46002D00D068
:109CC000E1E00B000343F3D0731C00D1ACE1214B66
:109CD0009F4200D13AE1F343382B00DD6FE11F2BA7
:109CE00000DD8CE120250E00ED1AAE40B0460600E6
:109CF000AA46DE40454635432E005546D940A84089
:109D00006346451EA8415B1A9C463043161AB24270
:109D1000924163465242991A3D00B4E6072232400E
:109D2000002A00D0E4E60B4BF6084F073743CA0879
:109D30009D4200D090E73B00134300D1A6E1802371
:109D40001B031A431203120B024D89E71500002270
:109D5000002785E7FF070000FFFF7FFFFFFF0F8061
:109D6000002E00D0C7E06B1C5E05760D012E00DCD6
:109D7000F0E0C84DAB4200D1B9E085180A00854239
:109D800089416244494251180722CE076D082E438B
:109D9000490832401D00A9E6BF49ED1A11400722CB
:109DA0003240A3E6320028388240002686E63000A2
:109DB00000F052FA203073E6634613435A1E934173
:109DC000C61AB04280414042091A5CE60E0067465E
:109DD00006431743002D5ED1002E00D0F3E0002F84
:109DE00000D11EE15C46614691462CE7A94FBE4278
:109DF0007BD01E00F1E610001F3DE840202B03D071
:109E00004021CB1A9A401643731E9E4107220643F7
:109E100032400021002583E7161A6346B242804192
:109E2000591A40420B1A98465C4632E61F2E00DD56
:109E3000ABE02027BB1B9A4663465746BB4099467A
:109E400013004F46F3401F433B005746BA40571E8E
:109E5000BA4113436246F240891898E62027BB1B9B
:109E60009A4663465746BB40994613004F46F34017
:109E70001F433B005746BA40571EBA411343624640
:109E8000F240891A9CE7834B9F425FD080252D04C6
:109E90007342294320E7002E0CD1002F00D1D0E0DF
:109EA0005C46614691467B4DCDE67A4FBE421CD062
:109EB0001E0065E6002F18D0C0084E07064380201C
:109EC000C9080003014208D06346DC08044204D1FB
:109ED0002100DA46D2085E071643F30099460124B2
:109EE0005346C900720F11431C406A4DABE61D007A
:109EF00000220027B4E6002D59D10B00034300D106
:109F0000D6E6731C00D1B2E0624B9F421ED0F343F1
:109F1000382B6FDC1F2B00DD97E020250E00ED1A9B
:109F2000AE40B0460600AA46DE40454635432E0008
:109F30005546A840D940451EA8418C440643B61852
:109F400096429241514261443D0025E63D00614602
:109F5000914678E60B000343002D00D055E6002B18
:109F6000F5D06346134300D16DE6861886428041E2
:109F700061444042091800220B0200D4D0E6464B4F
:109F800001351940B2E5B1465DE633006746203B36
:109F9000DF403B00202E05D04027BF1B6646BE4059
:109FA000324390464646721E96413343EFE5394BA5
:109FB0009F42CBD080252D0473422943A8E7084354
:109FC000411E8841A2E6002F00D13CE66346861A76
:109FD000CF1AB0429B415B42FB1A98461B024ED5FA
:109FE000161A6346B2429241591A5242891A5C4685
:109FF00000227BE501430E00711E8E419FE71D008C
:10A000000E00203DEE40B046202B04D04025EB1A38
:10A0100099400843814648464346411E88411843BB
:10A0200074E60022002417E6161A6346B2429241F3
:10A03000591A5242891A3D0025E561469146154D4F
:10A0400001E680220024120379E61D000E00203D67
:10A05000EE40B046202B04D04025EB1A994008432F
:10A0600081464E464346711E8E411E4367E7861861
:10A0700096429B4161445B42C9183D008CE54746CE
:10A080003743CED007224146324049E600273A0006
:10A09000E6E5C046FF070000FFFF7FFF70B50C4EEE
:10A0A0000D031C0349005B002D0B490D240B5B0DB8
:10A0B000B14208D0064900208B4203D1144320004E
:10A0C000441EA04170BD05430120002DFAD1F1E7E7
:10A0D000FF07000030B5144D0A034B00120B5B0D57
:10A0E000C90F0024AB4211DD104CA34210DC8024C8
:10A0F000640322430E4CE41A1F2C0CDD0D48C31AD6
:10A10000DA4013005C42002900D11C00200030BD61
:10A11000094BCC18FAE7094DE040AC4663449A403D
:10A1200013000343EEE7C046FE0300001D040000D9
:10A130003304000013040000FFFFFF7FEDFBFFFF6F
:10A1400070B500282DD0C317C5185D40C40F280076
:10A1500000F082F8154B1B1A5B055B0D0A2815DD14
:10A160000B38854000222D032D0B002110002D03FC
:10A170000A0D2D0B12052A430D4D1B052A401343D2
:10A180005B00E4075B082343190070BD020029004F
:10A19000153291400A000B21081AC5402D032D0BE2
:10A1A000E3E70024002300250022DEE71E04000070
:10A1B000FFFF0F804100090E4B1C70B5DBB2460259
:10A1C000750AC40F012B14DDE0239B006D07360BCD
:10A1D000CB1800210A0D280012051C4D32435B05E7
:10A1E0002A405B0813435B00E4075B082343190024
:10A1F00070BD002914D1002D1ED0280000F02CF8CD
:10A200000A281CDC0B232A001B1ADA400300153332
:10A210009D400F4B12031B1A5B05160B5B0DD8E715
:10A22000002D06D0320B802636036D071643094BEE
:10A23000CFE7084B0026CCE700230026C9E7030040
:10A240002A000B3B9A400025E3E7C046FFFF0F8042
:10A2500089030000FF0700001C2101231B04984212
:10A2600001D3000C10391B0A984201D3000A0839A7
:10A270001B09984201D30009043902A2105C40185E
:10A280007047C04604030202010101010000000002
:10A290000000000030B51C00094B05001B6885B0AC
:10A2A000D868084B002A01D1074B1A00029201938B
:10A2B00000912B002200054900F026F800F08EFDE9
:10A2C0006800002050CE000067BD00005DCE000099
:10A2D000014B18687047C04668000020084B10B555
:10A2E0000400002B02D0002100E000BF054B1868DD
:10A2F000836A002B00D09847200001F045FBC04640
:10A30000000000008CCE00000EB403B5010003ABCA
:10A31000044804CB0068019300F076F802B008BC52
:10A3200003B018476800002070B500260C4D0D4C96
:10A33000641BA410A64209D1002601F027FB0A4D98
:10A340000A4C641BA410A64205D170BDB300EB58A3
:10A3500098470136EEE7B300EB5898470136F2E72D
:10A360003802002038020020380200204802002075
:10A37000002310B59A4200D110BDCC5CC454013307
:10A38000F8E710B5884202D98B18984203D300230E
:10A3900007E08B5C8354013AFBD210BDCC5CC45403
:10A3A00001339A42FAD1F8E703001218934200D120
:10A3B000704719700133F9E7936810B5013B93605A
:10A3C000002B04DA9469A34207DB0A2905D013683D
:10A3D000581C10601970080010BD00F033FC01001B
:10A3E000F9E7F8B506000F001400D518AC4201D10A
:10A3F000002007E021783A003000FFF7DDFF01344C
:10A40000431CF3D1F8BD0000F0B59FB002900F00DF
:10A4100016000593002805D083690493002B01D111
:10A4200000F0DCFD7B4B9F425BD1029B5F68BB89E8
:10A430001B0762D53B69002B5FD0002306AC63612C
:10A44000203363761033A37635002B78002B01D0B0
:10A45000252B5CD1AB1B04930CD032003900029841
:10A46000FFF7BFFF431C00D1C4E06269049B944620
:10A47000634463612B78002B00D1BBE001220023F1
:10A480005242626002A9543252186E1C2360E3608B
:10A49000A3601370A365317805225F4800F0BCFE0D
:10A4A000751C002835D12268D30604D5532302A990
:10A4B0005B1820211970130704D5532302A95B18D8
:10A4C0002B21197033782A2B2CD0350000210A203B
:10A4D000E3682A786E1C303A092A64D900292ED004
:10A4E00026E04E4B9F4202D1029B9F689FE74C4B58
:10A4F0009F429CD1029BDF6899E73900029800F0E7
:10A50000F7FB002899D0012040421FB0F0BD013573
:10A510009BE7414B2268C01A012383401343236009
:10A520002E00B8E7059B191D1B680591002B01DB68
:10A53000099304E05B42E3600223134323602B781A
:10A540002E2B0AD16B782A2B35D1059B02351A1D8B
:10A550001B680592002B2BDB0793324E29780322D0
:10A56000300000F059FE002806D04023801B8340B5
:10A570002268013513432360297806222A486E1C7D
:10A58000217600F049FE00283AD0284B002B25D137
:10A590000722059B07339343083305936369039AA6
:10A5A0009B18636150E7434301219B18350090E7F6
:10A5B00001235B42D0E700230A201A0001356360C3
:10A5C00029786E1C3039092903D9002BC5D0079290
:10A5D000C3E74243012352183500F1E705AB00936E
:10A5E0003A00134B2100029800E000BF0390039B48
:10A5F0000133D3D1BB895B0600D584E70B9884E790
:10A6000005AB00933A000A4B2100029800F080F855
:10A61000ECE7C046E4CE000090CE000004CF00007E
:10A62000C4CE000096CE00009ACE000000000000CC
:10A63000E3A30000F7B5150001938A680B69009049
:10A640000C00934200DA130022002B604332127890
:10A65000002A01D001332B6023689B0602D52B68AA
:10A6600002332B60062723681F4027D02300433383
:10A670001B785A1E93412268920630D42200019919
:10A6800043320098089EB047431C25D0062320681B
:10A690002A68E16803400025042B03D18D1AEB439F
:10A6A000DB171D40A3682269934201DD9B1AED1858
:10A6B0000027BD4220D1002010E00137E3682A685E
:10A6C0009B1ABB42D2DD2200012319320199009866
:10A6D000089EB047431CF0D101204042FEBD30200F
:10A6E000E1184331087021005A1C45310978A2183D
:10A6F000433202331170C1E7220001231A3201995B
:10A700000098089EB047431CE6D00137D1E700000F
:10A71000F0B589B004920A00433205930390029287
:10A720000A7E0C000E9B6E2A00D186E01FD8632A99
:10A7300033D008D8002A00D18CE0582A4DD025000B
:10A7400042352A7030E0642A01D0692AF7D11968AD
:10A7500025680A1D280629D508681A60002803DA2A
:10A760002D23029A404213706B4E0A274FE0732A42
:10A7700074D008D86F2A1FD0702AE0D1202209682F
:10A780000A43226003E0752A16D0782AD7D1220026
:10A79000782145321170614E22E025001A68423559
:10A7A000111D196013682B70012365E008681A6099
:10A7B0006906D3D500B2D1E719682568081D18606D
:10A7C00008682E0605D5544E08276F2A1BD00A2785
:10A7D00019E06D06F7D580B2F5E745314E4E0A70A7
:10A7E00018682268011D00681960150621D5D30775
:10A7F00002D520231A4322601027002803D12023EA
:10A8000022689A4322602300002243331A7063684F
:10A81000A360002B58DB04222168914321600028AB
:10A8200054D1029D002B5AD02500337842352B702D
:10A8300055E05506DBD580B2D9E71A680D68101DC2
:10A840004969186013682E0601D5196002E06D068B
:10A85000FBD519800023029D23614FE01A68111D6A
:10A860001960156800216268280000F0D5FC0028F6
:10A8700001D0401B6060636823610023029A13705B
:10A880003CE023692A0004990398059DA847431CCE
:10A890003ED023689B0715D4079BE068984239DABD
:10A8A000180037E022000123193204990398059E0D
:10A8B000B047431C2CD00135E368079A9B1AAB4282
:10A8C000F0DCE9E70025F7E70028ADD0029D39006C
:10A8D000FDF722FC735C013D2B700028F7D1082F97
:10A8E00009D12368DB0706D563682269934202DC3D
:10A8F0003023013D2B70029B5B1B2361059B07AA44
:10A9000000932100049B0398FFF794FE431CB8D1E9
:10A910000120404209B0F0BDA1CE0000B2CE00003F
:10A920000D4B70B51C680500A36B002B0FD11820D0
:10A9300000F056FC094BA0630360094B0122436001
:10A94000084B83600B238381002302614361002253
:10A95000A36B1D615A6170BD680000200E33CDAB42
:10A9600034126DE6ECDE0500124B10B51C68A36BCB
:10A97000002B0FD1182000F033FC0F4BA0630360B5
:10A980000E4B012243600E4B83600B238381002317
:10A9900002614361A46B0B4A206961690A4BFDF7B0
:10A9A000F7FC0122002380185941206161614800B1
:10A9B000400810BD680000200E33CDAB34126DE6A8
:10A9C000ECDE05002D7F954C2DF451580CB430B5BC
:10A9D000164B9DB00C1E1D6808DA8B2301202B60DE
:10A9E00040421DB030BC08BC02B01847822302A907
:10A9F0009B008B810023029008619C4200D0631E63
:10AA00008B604B6101235B42CB81209A21AB2800F4
:10AA1000019300F03DFD431C01DA8B232B60002CD9
:10AA2000DFD00023029A1370DBE7C04668000020E5
:10AA30000EB400B50B499CB01DAB02900690079177
:10AA400004910948094904CB0591006802A90193C2
:10AA500000F01EFD0023029A13701CB008BC03B066
:10AA60001847C046FFFFFF7F680000200802FFFF75
:10AA7000020010B51378541C002B05D1CC5CD454C3
:10AA80000133002CFAD110BD2200F3E702780B78D5
:10AA9000002A03D0013001319A42F7D0D01A704712
:10AAA00003000A7801311A700133002AF9D1704786
:10AAB0000023C25C0133002AFBD1581E704730B519
:10AAC0000500002A00D130BD0C78013A6B1C2C70B7
:10AAD0000131002C05D19A189A42F4D01C70013330
:10AAE000FAE71D00EDE710B50378002B0FD10B78C6
:10AAF0005A4253415B42184010BD0023CA5C002AF1
:10AB0000FAD0C45C944201D10133F7E701300378F5
:10AB1000002BF2D11800EFE7F0B51F000E0087B050
:10AB20000590019102920C98347800F0EAFA08221C
:10AB300000194378751C134036D12D2C36D1B51C25
:10AB400074780126002F62D0102F09D1302C07D144
:10AB500020222B789343582B54D110276C78023540
:10AB60002D4B3900F31818000393FDF7D5FA049123
:10AB700001210023494202008C461800210030398F
:10AB800009291AD80C00A74223DD591C09D06346B5
:10AB9000824206D302D10499A14202DB0123784309
:10ABA00020182C780135E9E72E00BCE72B2C01D0CA
:10ABB0001E00C7E7B51C7478FAE72100413919294E
:10ABC00001D8373CDFE721006139192901D8573C0A
:10ABD000D9E75A1C08D1059A23331360029B0398C6
:10ABE000002B09D107B0F0BD002E00D04042029AE0
:10ABF000002AF7D0002B01D06B1E0193029B019A13
:10AC00001A60EFE73024002FAAD10827A8E7302CDC
:10AC10009ED00A27A4E7C046FFFFFF7F37B5130089
:10AC2000064A05001068046A002C00D1044C0A0092
:10AC300000942900FFF770FF3EBDC0466800002069
:10AC4000CC000020F8B505000E001400002804D048
:10AC50008369002B01D100F0C1F9224B9C422DD118
:10AC60006C68A369A360A3891B0731D52369002BF6
:10AC70002ED023682269F7B2981A6369F6B283422C
:10AC800005DC2100280000F03BF9002826D1A3684C
:10AC90000130013BA36023685A1C22601F70636966
:10ACA000834204D0A389DB071AD50A2E18D12100CC
:10ACB000280000F025F9002812D00FE00A4B9C4232
:10ACC00001D1AC68CDE7094B9C42CAD1EC68C8E71A
:10ACD0002100280000F00CF80028CAD00126764296
:10ACE0003000F8BDE4CE000004CF0000C4CE000068
:10ACF000364B70B51D6806000C00002D05D0AB6901
:10AD0000002B02D1280000F069F9314B9C420FD191
:10AD10006C680C23E25E93B219072DD4D90611D4C6
:10AD200009230120336037331343A381404270BDB0
:10AD3000284B9C4201D1AC68EBE7274B9C42E8D101
:10AD4000EC68E6E75B0713D5616B002908D02300A8
:10AD50004433994202D0300000F06AFA0023636362
:10AD60002422A3899343A381002363602369236082
:10AD70000823A2891343A3812369002B0BD1A021AF
:10AD80008022A389890092000B40934203D02100C6
:10AD9000300000F0E1F90123A289134011D0002313
:10ADA000A36063695B42A361002023698342BED133
:10ADB0000C23E25E1306BAD540231343A381013866
:10ADC000B5E7920700D46369A360EDE7680000204F
:10ADD000E4CE000004CF0000C4CE000010B5062071
:10ADE00000F090FC012000F0CFFD0000F7B58A894B
:10ADF00005000C00130760D44B68002B04DC0B6CBF
:10AE0000002B01DC0020FEBDE76A002FFAD00023F2
:10AE10002E682B6080235B01216A1A4034D0606D5C
:10AE2000A3895B0706D56368C01A636B002B01D04A
:10AE3000236CC01A0200216A00232800E76AB84781
:10AE4000A189431C06D12B681D2B30D82B4ADA4030
:10AE5000D3072CD50023636023692360CB0405D579
:10AE6000431C02D12B68002B00D16065616B2E6002
:10AE70000029C7D023004433994202D0280000F0B3
:10AE8000D7F900206063BEE701232800B847431CC0
:10AE9000C6D12B68002BC3D01D2B01D0162B01D19E
:10AEA0002E60AFE74023A2891343A381ABE7402381
:10AEB0000B430120A3814042A5E70F69002FA1D0D9
:10AEC0000B680F60DB1B01930023920700D14B69D5
:10AED000A360019B002B00DC94E7019B3A00216AF0
:10AEE0002800A66AB047002803DC4023A289134348
:10AEF000DFE7019B3F181B1A0193EAE7010040209E
:10AF00000B6970B505000C00002B01D1002070BD4D
:10AF1000002804D08369002B01D100F05FF80B4BAF
:10AF20009C4209D16C680C22A35E002BEED021005C
:10AF30002800FFF75BFFEAE7054B9C4201D1AC68B4
:10AF4000F1E7044B9C42EED1EC68ECE7E4CE000064
:10AF500004CF0000C4CE0000002310B5040003603D
:10AF60004360836081814366C28103614361836181
:10AF7000190008225C30FFF717FA054B2462636260
:10AF8000044BA362044BE362044B236310BDC04631
:10AF900045B700006DB70000A5B70000D1B70000AD
:10AFA00010B5024900F08CF810BDC04601AF00009A
:10AFB00070B568254A1E55430E002900743100F013
:10AFC00081F9041E08D000212A00016046600C307F
:10AFD000A0606832FFF7E8F9200070BD836913B5FF
:10AFE0000400002B28D18364C3640365134B144A07
:10AFF0001B6882620193984201D101238361200082
:10B0000000F020F86060200000F01CF8A060200034
:10B0100000F018F80022E06004216068FFF79CFF50
:10B0200001220921A068FFF797FF02221221E068A0
:10B03000FFF792FF0123A36113BDC0468CCE000031
:10B04000A1AF0000F8B51C4B07001E68B369002BC8
:10B0500002D13000FFF7C2FF4836B4687368013B85
:10B0600004D53368002B07D03668F6E70C22A55EBE
:10B07000002D0DD06834F2E704213800FFF798FF67
:10B0800030600028F0D10C2304003B602000F8BDA4
:10B0900020000A4B656625606560A560E360256158
:10B0A0006561A561082229005C30FFF77DF96563C1
:10B0B000A563A564E564E9E78CCE00000100FFFF0D
:10B0C000F7B504000700002601914834002C01D197
:10B0D0003000FEBD6368A5680093009B013B0093B0
:10B0E00001D52468F2E7AB89012B08D90E22AB5EAB
:10B0F000013304D029003800019B98470643683586
:10B10000EBE7EC300068704770B50E001D000E23B1
:10B11000C95E96B01400002907DA00232B60B389BA
:10B120001B0611D48023DB000FE06A4600F088FB89
:10B130000028F2DBF022019B12021340054A9B1803
:10B140005A4253412B60EDE740230020236016B0A4
:10B1500070BDC04600E0FFFFF7B502268B890500F1
:10B160000C00334206D023004733236023610123C0
:10B170006361F7BD01AB6A46FFF7C6FF00990700A0
:10B18000280000F09FF8002808D10C22A35E9A0541
:10B19000EFD4032293431E43A681E4E70F4BAB6237
:10B1A0008023A28920601343A381009B20616361F7
:10B1B000019B002B0DD00E23E15E280000F052FB16
:10B1C000002806D00322A38993431A0001231343C6
:10B1D000A381A0893843A081CBE7C046A1AF00007E
:10B1E00010B5034B0100186800F06CF810BDC046A4
:10B1F0006800002082B0002900D101A9101E06D0ED
:10B20000002B06D013780B601078431E984102B0D3
:10B21000704702204042FAE7C9B28218904201D139
:10B220000020704703788B42FBD00130F6E7000026
:10B2300070B50500002910D00C1F2368002B00DA20
:10B24000E418280000F034FB1D4A1368002B05D1D8
:10B2500063601460280000F02CFB70BDA34209D984
:10B26000216860188342F3D118685B684118216037
:10B27000EEE713005A68002A01D0A242F9D91968F2
:10B280005818A0420BD1206809185818196082423A
:10B29000E0D110685268411819605A60DAE7A0429C
:10B2A00002D90C232B60D5E721686018824203D1B4
:10B2B000106852684118216062605C60CAE7C0464D
:10B2C000E81B0020032370B5CD1C9D430835060004
:10B2D0000C2D1ED20C25A9421DD8300000F0E8FA32
:10B2E000254A14682100002919D1244C2368002B19
:10B2F00003D1300000F0CAF920602900300000F0CE
:10B30000C5F9431C2BD10C233000336000F0D1FA77
:10B3100003E0002DDFDA0C233360002070BD0B68E2
:10B320005B1B19D40B2B03D90B60CC18256003E0F1
:10B330004B688C420DD11360300000F0BAFA200047
:10B3400007220B30231D9043C31AE7D05A42E25024
:10B35000E4E763600C00EFE70C004968C3E70323F0
:10B36000C41C9C43A042E1D0211A300000F08EF9A9
:10B37000431CDBD1C7E7C046E81B0020EC1B0020C4
:10B38000F8B507000D001600002905D11100FFF7E0
:10B3900099FF04002000F8BD002A03D1FFF748FF01
:10B3A0003400F7E700F086FA2C00B042F2D2310008
:10B3B0003800FFF787FF041EECD029003200FEF7AB
:10B3C000D7FF29003800FFF733FFE3E7F0B58E68B9
:10B3D00085B007000C00039201939E423CD8902355
:10B3E0008A89DB001A4234D00325096923685B1A75
:10B3F0000293636902985D43EB0F5D19019B6D1029
:10B4000001331B18AB4200D91D00530532D529006A
:10B410003800FFF757FF061E09D10C233B6040237D
:10B420000120A28940421343A38105B0F0BD029AD6
:10B430002169FEF79DFFA389144A1A408023134314
:10B44000A381029B2661F61826606561019EED1AB4
:10B45000A560019B9E4200D9019E3200039920689D
:10B46000FEF78FFFA36800209B1BA36023689E1933
:10B470002660DAE72A003800FFF782FF061EE0D1D7
:10B4800021693800FFF7D4FEC7E7C0467FFBFFFF06
:10B49000F0B59FB0029005938B890F0016001B0634
:10B4A00011D50B69002B0ED14021FFF70BFF38603F
:10B4B0003861002805D10C23029A013813601FB0AF
:10B4C000F0BD40237B61002306AC636120336376CB
:10B4D0001033A37635002B78002B01D0252B46D1D5
:10B4E000AB1B04930CD0320039000298FFF76EFFBB
:10B4F000431C00D1AEE06269049B944663446361DF
:10B500002B78002B00D1A5E001220023524262607B
:10B5100002A9543252186E1C2360E360A3601370BA
:10B52000A365317805225448FFF776FE751C002884
:10B530001FD12268D30604D5532302A95B1820210A
:10B540001970130704D5532302A95B182B21197016
:10B5500033782A2B16D0350000210A20E3682A7898
:10B560006E1C303A092A4ED9002918D010E0013556
:10B57000B1E7414B2268C01A012383401343236083
:10B580002E00CEE7059B191D1B680591002B01DBE2
:10B59000099304E05B42E3600223134323602B78AA
:10B5A0002E2B0AD16B782A2B35D1059B02351A1D1B
:10B5B0001B680592002B2BDB0793304E2978032262
:10B5C0003000FFF729FE002806D04023801B83406F
:10B5D00022680135134323602978062228486E1C0F
:10B5E0002176FFF719FE00283CD0264B002B25D1F1
:10B5F0000722059B07339343083305936369039A36
:10B600009B18636166E7434301219B183500A6E759
:10B6100001235B42D0E700230A201A000135636052
:10B6200029786E1C3039092903D9002BC5D007921F
:10B63000C3E74243012352183500F1E705AB0093FD
:10B640003A00114B2100029800E000BF0390039BD9
:10B650000133D3D1BB890B985B0600D42FE70120BF
:10B6600040422CE705AB00933A00074B21000298BB
:10B67000FFF74EF8EAE7C04690CE000096CE0000F5
:10B680009ACE000000000000CDB30000002370B58A
:10B69000064C05000800236000F060F9431C03D14C
:10B6A0002368002B00D02B6070BDC046A02F002067
:10B6B00070B504000D001F2904D916230360012072
:10B6C000404270BD436C002B04D08A009B181A685E
:10B6D000002A08D1200000F031F82A0001002000E3
:10B6E00000F01AF8EDE70020012AEAD0511C03D13E
:10B6F000162301302360E4E7002428001C609047F3
:10B700002000DEE710B5034B01001868FFF7D0FFFB
:10B7100010BDC04668000020002370B5064C05002F
:10B7200008001100236000F001F9431C03D12368D5
:10B73000002B00D02B6070BDA02F002010B500F0B2
:10B74000E5F810BD70B50C000E25495F00F0BAF8A1
:10B75000002803DB636D1B18636570BDA389024A73
:10B760001340A381F9E7C046FFEFFFFFF8B51F00C4
:10B770008B8905000C001600DB0505D50E23C95E7C
:10B780000022022300F080F8A389054A2800134014
:10B79000A38132000E23E15E3B0000F02BF8F8BDE0
:10B7A000FFEFFFFF70B50C000E25495F00F06CF84D
:10B7B000A389421C03D1054A1340A38170BD802296
:10B7C00052011343A3816065F8E7C046FFEFFFFF16
:10B7D00010B50E23C95E00F021F810BD0B1E04D079
:10B7E000FF2A04D98A2303608B3B180070470A7034
:10B7F0000123FAE770B50500080011000022064C8D
:10B8000022601A0000F0B8F8431C03D12368002B13
:10B8100000D02B6070BDC046A02F0020002370B563
:10B82000064C05000800236000F060F8431C03D1BB
:10B830002368002B00D02B6070BDC046A02F0020D5
:10B84000002370B5064C050008001100236000F0CD
:10B8500055F8431C03D12368002B00D02B6070BD2A
:10B86000A02F0020002370B5064C050008002360BF
:10B8700000F054F8431C03D12368002B00D02B6048
:10B8800070BDC046A02F002070B505000800110053
:10B890000022064C22601A0000F050F8431C03D12D
:10B8A0002368002B00D02B6070BDC046A02F002065
:10B8B000704770470B1F1B68181F002B01DA0B58CD
:10B8C000C018704770B50500080011000022064C32
:10B8D00022601A0000F03AF8431C03D12368002BC1
:10B8E00000D02B6070BDC046A02F00205822012040
:10B8F000014B40421A607047A02F002058220120BF
:10B90000014B40421A607047A02F002058220120AE
:10B91000014B40421A607047A02F00205822024B72
:10B9200000201A607047C046A02F00205822012036
:10B93000014B40421A607047A02F0020582201207E
:10B94000014B40421A607047A02F0020582201206E
:10B95000014B40421A607047A02F0020044A136830
:10B96000002B00D1034B1818106018007047C04618
:10B97000F01B0020A82F002058220120014B40423C
:10B980001A607047A02F0020FEE7C046F8B5C046F9
:10B99000F8BC08BC9E467047F8B5C046F8BC08BC69
:10B9A0009E467047646174610000000020BA000088
:10B9B000EB01000029BA00001704000031BA0000B2
:10B9C0002D07000038BA00003D0800003DBA000015
:10B9D000DF02000048BA0000830400004DBA0000F6
:10B9E000B509000059BA00001B02000063BA00004C
:10B9F0003506000071BA0000A105000072616E6496
:10BA00006F6D00616C6C006C6173740066616C73C7
:10BA100065007472756500252E3135732E2E2E004B
:10BA20006D616B654C697374006164644C6173741F
:10BA30000064656C657465006A6F696E00636F70A1
:10BA40007946726F6D546F0066696E64006A6F6943
:10BA50006E537472696E677300756E69636F6465A7
:10BA6000417400756E69636F6465537472696E67C3
:10BA700000667265654D656D6F727900C80F0000D4
:10BA8000D80F0000F20F000070100000A810000096
:10BA9000DE100000161100003C11000078110000BB
:10BAA000BA1100001012000054120000C012000071
:10BAB000081300002E13000066130000AC130000F2
:10BAC000D213000000140000321400006A140000B9
:10BAD000EE140000B61500002C16000098160000A9
:10BAE000E01600000017000022170000D217000027
:10BAF00018180000C80F0000C80F0000C80F000091
:10BB000090180000F818000060190000C01900002B
:10BB1000081A00007A1A0000EC1A0000341B00001A
:10BB20007A1B0000B01B0000F61B00003C1C00004C
:10BB3000841C0000D81C00002C1D0000741D000097
:10BB4000DE1D0000141E00005C1E0000A41E00008C
:10BB5000EC1E0000261F00006E1F0000B61F000034
:10BB6000C80F0000C80F0000C80F00001E20000012
:10BB7000C80F00005420000080200000B620000004
:10BB8000E2200000C80F0000C80F0000C80F00002E
:10BB9000C80F0000182100005A210000C80F000043
:10BBA000C80F0000AA210000FA2100002022000096
:10BBB000C80F0000C80F0000C80F00004E22000090
:10BBC0007E220000AE220000E42200000E230000CE
:10BBD000442300006E23000096230000BE230000D3
:10BBE000EE2300001E240000482400007224000000
:10BBF000A2240000CC240000C80F0000C80F0000E1
:10BC0000C80F0000C80F0000C80F0000FC2400008F
:10BC1000282500006C25000098250000C4250000A0
:10BC2000FA25000030260000662600009C26000051
:10BC3000C8260000F42600002A270000C80F0000D4
:10BC4000C80F0000C80F0000C80F0000C80F000098
:10BC5000C80F0000C80F0000C80F0000C80F000088
:10BC6000C80F0000C80F0000C80F0000C80F000078
:10BC7000C80F0000562700008C27000028256420EC
:10BC80006974656D206C6973742900286F626A6538
:10BC9000637420747970653A2025642900537461B7
:10BCA000636B20756E646572666C6F7700000000D0
:10BCB0000700000003000000FABC0000712800002B
:10BCC00002BD0000752800000BBD00006D280000BB
:10BCD00014BD0000792800000000000001000000F1
:10BCE0000200000003000000040000000A00000041
:10BCF0006D6963726F3A62697400686173546F6E44
:10BD00006500706C6179546F6E650068617353658E
:10BD100072766F00736574536572766F00474320C7
:10BD2000746F6F6B2025642075736563733B2066A9
:10BD300072656520256420776F726473003C496EDC
:10BD400074656765723E003C4F626A6563743E00CD
:10BD50003C4C6973743E000D0A564D2050616E696B
:10BD6000633A2025730D0A006D69736300000000BB
:10BD700080BD00001931000089BD0000D1300000F5
:10BD8000686578546F496E740073696E0000000036
:10BD9000DCBD000085310000E4BD000089310000F9
:10BDA000EEBD0000A7310000F7BD0000B13100007A
:10BDB00002BE0000BB3100000EBE0000C531000015
:10BDC0001FBE0000CF31000035BE000093310000DF
:10BDD0004EBE00009D3100006E65740068617357AF
:10BDE00069466900737461727457694669007374B7
:10BDF0006F70576946690077696669537461747535
:10BE000073006D794950416464726573730074689E
:10BE1000696E674465736372697074696F6E0063FD
:10BE20006C6561725468696E6744657363726970AA
:10BE300074696F6E00617070656E64546F546869E8
:10BE40006E674465736372697074696F6E006170C8
:10BE500070656E64546F5468696E6750726F706578
:10BE6000727479001A1B1C03040607090A171819B3
:10BE700003040607090A1718190000000000080843
:10BE80000800080A4A4000000A5FEA5FEA0ED92E5D
:10BE9000D36E19324489330C924C924D080800003D
:10BEA0000004880808040804848488000A448A403E
:10BEB00000048EC480000000048800000EC0000052
:10BEC0000000080001224488100C9252524C048C4D
:10BED00084848E1C824C901E1EC244924C06CA5210
:10BEE0005FE21FF01EC13E02448ED12E1FE2448845
:10BEF000100ED12ED12E0ED12EC4880008000800BD
:10BF000000048004880244880482000EC00EC00829
:10BF1000048244880ED126C0040ED135B36C0C9235
:10BF20005ED2521C925C925C0ED010100E1C92528B
:10BF3000525C1ED01C901E1ED01C90100ED013718F
:10BF40002E12525ED2521C8808081C1FE242524C2C
:10BF50001254981492101010101E113B75B131112B
:10BF60003935B3710C9252524C1C925C90100C9269
:10BF7000524C861C925C92510ED00C825C1FE48461
:10BF80008484125252524C1131312A44113135BB42
:10BF90007112524C9252112A4484841EC488101E7D
:10BFA0000EC808080E10080482410EC242424E0418
:10BFB0008A400000000000001F0804800000000EFE
:10BFC000D2524F10101C925C000ED0100E02424E46
:10BFD000D24E0C925C900E06C81C88080ED24EC23F
:10BFE0004C10101C92520800080808024002424CF3
:10BFF00010149814920808080806001B75B1310047
:10C000001C925252000C92524C001C925C90000EFA
:10C01000D24EC2000ED010100006C8049808080EB8
:10C02000C807001252524F0011312A440011313515
:10C03000BB00124C8C9200112A4498001EC4881E2A
:10C0400006C48C8486080808080818080C8818009C
:10C05000000C8360000000000100000002000000EE
:10C0600003000000040000000500000006000000BE
:10C070000700000008000000090000000A0000009E
:10C080000B0000000C0000000D0000000E0000007E
:10C090000F0000001000000012000000140000005B
:10C0A00016000000180000001A0000001C0000002C
:10C0B0001E000000200000002300000026000000F9
:10C0C000290000002C0000002F00000032000000BA
:10C0D000360000003A0000003E0000004200000070
:10C0E000460000004B00000050000000550000001A
:10C0F0005A00000061000000680000006F000000AE
:10C10000760000007D000000840000008B0000002D
:10C110009200000099000000A0000000A7000000AD
:10C12000AE000000B5000000BC000000C30000002D
:10C13000CA000000D1000000D8000000DF000000AD
:10C14000E6000000ED000000F4000000FB0000002D
:10C15000FF000000A4C10000F5310000AFC10000E5
:10C1600029370000B9C1000039340000C6C1000001
:10C1700059340000CDC10000A9340000D6C1000030
:10C18000F9340000E2C10000D5330000F3C1000023
:10C190003936000000C20000F53600006469737093
:10C1A0006C6179006C696768744C6576656C006DCC
:10C1B00062446973706C6179006D62446973706C7C
:10C1C00061794F6666006D62506C6F74006D6255E8
:10C1D0006E706C6F74006D62447261775368617049
:10C1E00065006D625368617065466F724C6574746A
:10C1F0006572006E656F506978656C53656E64009A
:10C200006E656F506978656C53657450696E004E49
:10C210006F7420656E6F75676820726F6F6D206533
:10C2200076656E20616674657220636F6D70616300
:10C2300074696F6E00436F6D70616374656420464E
:10C240006C61736820636F64652073746F72650A34
:10C2500025642062797465732075736564202825D0
:10C2600064252529206F66202564004261642072C0
:10C2700065636F726420666F756E642064757269A1
:10C280006E6720696E697469616C697A6174696F3F
:10C290006E002564202564202564202825642077ED
:10C2A0006F72647329002564207265636F72647312
:10C2B0002C20256420776F7264732C206D6178497F
:10C2C000442025642C20636F6D70616374696F6E08
:10C2D000206379636C657320256400526573746F05
:10C2E00072656420256420736372697074730053EF
:10C2F00074617274656400726164696F00000000AB
:10C300008EC30000F14000009BC3000061430000A9
:10C31000ABC3000001430000B9C30000E1440000CA
:10C32000C4C3000009410000D4C300007D410000E7
:10C33000E8C3000019410000F7C30000C346000035
:10C3400003C40000414600000CC40000E5450000A5
:10C3500017C400002D45000022C4000069450000FC
:10C360002BC400009D45000034C400002D41000096
:10C370006E756D626572006E6F6E65006F746865D4
:10C3800072007061697200737472696E670064692B
:10C390007361626C65526164696F006D657373618E
:10C3A00067655265636569766564007061636B6596
:10C3B0007452656365697665007061636B6574537B
:10C3C000656E64007265636569766564496E74655F
:10C3D0006765720072656365697665644D65737340
:10C3E0006167655479706500726563656976656437
:10C3F000537472696E670073656E64496E74656725
:10C4000065720073656E64506169720073656E6475
:10C41000537472696E67007365744368616E6E650C
:10C420006C0073657447726F757000736574506F3C
:10C43000776572007369676E616C537472656E67BD
:10C440007468000000000000963007772C610EEE43
:10C45000BA51099919C46D078FF46A7035A563E95B
:10C46000A395649E3288DB0EA4B8DC791EE9D5E082
:10C4700088D9D2972B4CB609BD7CB17E072DB8E781
:10C48000911DBF906410B71DF220B06A4871B9F3D6
:10C49000DE41BE847DD4DA1AEBE4DD6D51B5D4F40F
:10C4A000C785D38356986C13C0A86B647AF962FD74
:10C4B000ECC9658A4F5C0114D96C0663633D0FFAC1
:10C4C000F50D088DC8206E3B5E10694CE44160D5C7
:10C4D000727167A2D1E4033C47D4044BFD850DD2B1
:10C4E0006BB50AA5FAA8B5356C98B242D6C9BBDBC4
:10C4F00040F9BCACE36CD832755CDF45CF0DD6DCBF
:10C50000593DD1ABAC30D9263A00DE518051D7C865
:10C510001661D0BFB5F4B42123C4B3569995BACFF0
:10C520000FA5BDB89EB802280888055FB2D90CC611
:10C5300024E90BB1877C6F2F114C6858AB1D61C18A
:10C540003D2D66B69041DC760671DB01BC20D298A9
:10C550002A10D5EF8985B1711FB5B606A5E4BF9F36
:10C5600033D4B8E8A2C9077834F9000F8EA8099629
:10C5700018980EE1BB0D6A7F2D3D6D08976C649194
:10C58000015C63E6F4516B6B62616C1CD8306585AD
:10C590004E0062F2ED95066C7BA5011BC1F408828A
:10C5A00057C40FF5C6D9B06550E9B712EAB8BE8BCB
:10C5B0007C88B9FCDF1DDD62492DDA15F37CD38C54
:10C5C000654CD4FB5861B24DCE51B53A7400BCA352
:10C5D000E230BBD441A5DF4AD795D83D6DC4D1A484
:10C5E000FBF4D6D36AE96943FCD96E34468867AD5B
:10C5F000D0B860DA732D0444E51D03335F4C0AAAFA
:10C60000C97C0DDD3C710550AA41022710100BBEFC
:10C6100086200CC925B56857B3856F2009D466B943
:10C620009FE461CE0EF9DE5E98C9D9292298D0B078
:10C63000B4A8D7C7173DB359810DB42E3B5CBDB725
:10C64000AD6CBAC02083B8EDB6B3BF9A0CE2B603A6
:10C650009AD2B1743947D5EAAF77D29D1526DB045B
:10C660008316DC73120B63E3843B64943E6A6D0DA6
:10C67000A85A6A7A0BCF0EE49DFF099327AE000AF1
:10C68000B19E077D44930FF0D2A3088768F2011E84
:10C69000FEC206695D5762F7CB67658071366C191B
:10C6A000E7066B6E761BD4FEE02BD3895A7ADA103C
:10C6B000CC4ADD676FDFB9F9F9EFBE8E43BEB7171D
:10C6C000D58EB060E8A3D6D67E93D1A1C4C2D838A7
:10C6D00052F2DF4FF167BBD16757BCA6DD06B53F0D
:10C6E0004B36B248DA2B0DD84C1B0AAFF64A03364C
:10C6F000607A0441C3EF60DF55DF67A8EF8E6E31CB
:10C7000079BE69468CB361CB1A8366BCA0D26F2513
:10C7100036E2685295770CCC03470BBBB916022260
:10C720002F260555BE3BBAC5280BBDB2925AB42B75
:10C73000046AB35CA7FFD7C231CFD0B58B9ED92C8A
:10C740001DAEDE5BB0C2649B26F263EC9CA36A75EF
:10C750000A936D02A906099C3F360EEB85670772A6
:10C7600013570005824ABF95147AB8E2AE2BB17B0D
:10C77000381BB60C9B8ED2920DBED5E5B7EFDC7C94
:10C7800021DFDB0BD4D2D38642E2D4F1F8B3DD68EB
:10C790006E83DA1FCD16BE815B26B9F6E177B06FE6
:10C7A0007747B718E65A0888706A0FFFCA3B0666D3
:10C7B0005C0B0111FF9E658F69AE62F8D3FF6B6160
:10C7C00045CF6C1678E20AA0EED20DD75483044E02
:10C7D000C2B30339612667A7F71660D04D47694990
:10C7E000DB776E3E4A6AD1AEDC5AD6D9660BDF40A3
:10C7F000F03BD83753AEBCA9C59EBBDE7FCFB24756
:10C80000E9FFB5301CF2BDBD8AC2BACA3093B3533A
:10C81000A6A3B4240536D0BA9306D7CD2957DE5443
:10C82000BF67D9232E7A66B3B84A61C4021B685D1C
:10C83000942B6F2A37BE0BB4A18E0CC31BDF055A95
:10C840008DEF022D416C6C207461736B73207374D7
:10C850006F707065640076303730002025732025B6
:10C8600073004D656D6F727920636C6561726564EC
:10C87000004E6F2066726565207461736B20656E73
:10C880007472696573000000D0C80000F958000098
:10C89000DDC8000091550000E9C800002F590000D4
:10C8A000EFC800003F590000F5C800004F590000D4
:10C8B000FBC80000C555000005C900006159000013
:10C8C0000DC900000557000073656E736F72730029
:10C8D000616363656C65726174696F6E0074656D28
:10C8E00070657261747572650074696C7458007457
:10C8F000696C74590074696C745A00746F7563685C
:10C900005265616400693263526561640069326333
:10C9100057726974650000008CC90000E15900007D
:10C920009AC90000E5590000A3C90000F1590000B0
:10C93000ADC90000F5590000B6C90000F959000062
:10C94000BBC90000FD590000C0C90000015A000029
:10C95000CCC90000055A0000D3C90000095A0000E4
:10C96000DCC900000D5A0000E1C90000115A0000A6
:10C97000ECC90000155A0000F6C90000E959000092
:10C9800000CA0000ED59000074667400656E6162B3
:10C990006C65446973706C6179006765745769648C
:10C9A00074680067657448656967687400736574C6
:10C9B000506978656C006C696E650072656374001F
:10C9C000726F756E64656452656374006369726347
:10C9D0006C6500747269616E676C6500746578746B
:10C9E00000746674546F756368656400746674548B
:10C9F0006F7563685800746674546F756368590086
:10CA0000746674546F75636850726573737572657C
:10CA10000057656C636F6D6520746F204D6963729C
:10CA20006F426C6F636B732100705F7370692021BC
:10CA30003D204E554C4C002F686F6D652F62726F14
:10CA40006D61676F73612F2E706C6174666F726DAC
:10CA5000696F2F7061636B616765732F6672616DBB
:10CA600065776F726B2D61726475696E6F6E6F7230
:10CA70006469636E7266352F6C6962726172696592
:10CA8000732F5350492F5350492E637070005350E9
:10CA900049436C6173733A3A535049436C61737301
:10CAA000284E52465F5350495F547970652A2C20B6
:10CAB00075696E74385F742C2075696E74385F7494
:10CAC0002C2075696E74385F742900000000000026
:10CAD00000000000195C0000D55B0000FB5B00005B
:10CAE000055C00000F5C0000F95B00000300000023
:10CAF000020000000100000004000000050000002A
:10CB0000110000000C0000000B00000012000000EB
:10CB10000A000000060000001A00000014000000D7
:10CB200017000000160000001500000010000000B3
:10CB3000FFFFFFFFFFFFFFFF000000001E000000DF
:10CB400019000000180000000700000008000000A5
:10CB5000090000000D0000000E0000000F000000A2
:10CB60001C0000001B0000001D000000130000005E
:10CB70000000000000000000C9600000F96700002C
:10CB8000496100005D61000053610000C560000064
:10CB9000B960000069610000E5600000B560000058
:10CBA000000000000000304300000000000030C31F
:10CBB0007371727400000000FB21F93FFB210940F2
:10CBC0007CD91240FB2119407A6A1F407CD922404F
:10CBD000BBFD2540FB2129403A462C407A6A2F4074
:10CBE0005C4731407CD932409C6B3440BBFD3540C2
:10CBF000DB8F3740FB2139401BB43A403A463C407A
:10CC00005AD83D407A6A3F404C7E40405C474140A4
:10CC10006C1042407CD942408CA243409C6B444003
:10CC2000AC344540BBFD4540CBC64640DB8F47405A
:10CC3000EB584840FB21494083F9A200444E6E0066
:10CC4000FC291500D1572700DD34F50062DBC00058
:10CC50003C999500419043006351FE00BBDEAB0060
:10CC6000B761C5003A6E2400D24D42004906E0008B
:10CC700009EA2E001C92D100EB1DFE0029B11C0018
:10CC8000E83EA700F535820044BB2E009CE98400F5
:10CC9000B4267000417E5F00D6913900538339007D
:10CCA0009CF439008B5F840028F9BD00F81F3B001D
:10CCB000DEFF97000F980500112FEF000A5A8B0036
:10CCC0006D1F6D00CF7E360009CB2700464FB700A1
:10CCD0009E663F002DEA5F00BA277500E5EBC700AE
:10CCE0003D7BF100F739070092528A00FB6BEA00A6
:10CCF0001FB15F00085D8D00300356007BFC4600CD
:10CD0000F0AB6B0020BCCF0036F49A00E3A91D0005
:10CD10005E619100081BE60085996500A0145F0024
:10CD20008D40680080D8FF0027734D000606310053
:10CD3000CA561500C9A873007BE260006B8CC00066
:10CD400000000040FB21F93F000000002D44743E2C
:10CD5000000000809846F83C0000006051CC783B11
:10CD600000000080831BF0390000004020257A3845
:10CD7000000000802282E336000000001DF36935C8
:10CD80000200000003000000040000000600000094
:10CD9000DC8400008684000086840000B4850000E6
:10CDA0008284000082840000AA850000B48500000F
:10CDB00082840000AA85000082840000B4850000FF
:10CDC000B8850000B8850000B8850000C085000067
:10CDD000B88F00002A8E00006E8E0000D28D0000F9
:10CDE0006E8E00005E8F00006E8E0000D28D0000FF
:10CDF0002A8E00002A8E00005E8F0000D28D000077
:10CE0000CA8D0000CA8D0000CA8D00006C8F000022
:10CE1000E0960000E2950000E29500000099000015
:10CE2000DC950000DC950000E89800000099000007
:10CE3000DC950000E8980000DC95000000990000F7
:10CE4000F6980000F6980000F6980000049900009B
:10CE50002C2066756E6374696F6E3A20006173737F
:10CE6000657274696F6E2022257322206661696C79
:10CE700065643A2066696C6520222573222C206C3B
:10CE8000696E65202564257325730A006C000020F7
:10CE9000232D302B2000686C4C00656667454647A3
:10CEA0000030313233343536373839414243444526
:10CEB0004600303132333435363738396162636495
:10CEC0006566000000000000000000000000000097
:10CED0000000000000000000000000000000000052
:10CEE0000000000000000000000000000000000042
:10CEF0000000000000000000000000000000000032
:10CF00000000000000000000000000000000000021
:10CF10000000000000000000000000000000000011
:10CF2000000000004300504F5349580000202020CB
:10CF300020202020202028282828282020202020C9
:10CF40002020202020202020202020202088101099
:10CF500010101010101010101010101010040404F5
:10CF600004040404040404101010101010104141B3
:10CF700041414141010101010101010101010101A1
:10CF800001010101010101011010101010104242B5
:10CF90004242424202020202020202020202020271
:10CFA0000202020202020202101010102000000011
:10CFB0000000000000000000000000000000000071
:10CFC0000000000000000000000000000000000061
:10CFD0000000000000000000000000000000000051
:10CFE0000000000000000000000000000000000041
:10CFF0000000000000000000000000000000000031
:10D000000000000000000000000000000000000020
:10D010000000000000000000000000000000000010
:10D020000000000000000000000000000000000000
:04D0300000000000FC
:08D03400D430FF7F0100000071
:10D03C00FFFFFFFF400600001800000019FCFFFF77
:10D04C00FFFFFFFFFF0000000200000003000000D4
:10D05C00FFFFFFFF000000000100000000000200C5
:10D06C0001000000FFFFFFFF0000000002000000B5
:10D07C000000040002000000FFFFFFFF00000000A2
:10D08C000300000000000800030000000A0000007C
:10D09C0008000000010000006C00002000000000EF
:10D0AC00E4CE000004CF0000C4CE0000000000005D
:10D0BC000000000000000000000000000000000064
:10D0CC000000000000000000000000000000000054
:10D0DC000000000000000000000000000000000044
:10D0EC000000000000000000000000000000000034
:10D0FC0000000000000000000000000043000000E1
:10D10C000000000000000000000000000000000013
:10D11C0000000000000000000000000043000000C0
:10D12C0000000000000000000000000000000000F3
:10D13C0000000000000000000000000043000000A0
:10D14C0000000000000000000000000000000000D3
:10D15C000000000000000000000000004300000080
:10D16C0000000000000000000000000000000000B3
:10D17C000000000000000000000000004300000060
:10D18C000000000000000000000000000000000093
:10D19C000000000000000000000000004300000040
:10D1AC000000000000000000000000000000000073
:10D1BC000000000000000000000000004300000020
:10D1CC000000000000000000000000000000000053
:10D1DC00000000000000000000000000DDB70000AF
:10D1EC00F5B10000000000002CCF00001EBA0000BA
:10D1FC0067BD000067BD000067BD000067BD000093
:10D20C0067BD000067BD000067BD000067BD000082
:10D21C0067BD0000FFFFFFFFFFFFFFFFFFFFFFFFEA
:10D22C00FFFF00000100415343494900000000008A
:10D23C0000000000000000000000000000000000E2
:10D24C000000000000004153434949000000000069
:10D25C0000000000000000000000000000000000C2
:10D26C000000000000000000E9000000A55B0000C9
:0CD27C00ED5E000015640000C100000021
:0400000300005F8911
:00000001FF
